:020000040000FA
:107800005469616E59696E673130300000000000C4
:1078100054593230302E303830303030625F747925
:10782000424154333247313339474B3634464200B4
:1078300043414E5F5354440000000000000000002C
:1078400043414E5F43485F300000000000000000ED
:1078500043414E5F3530304B6270730000000000D2
:107860009407000014070000DF070000000000007C
:020000040000FA
:1080000090330020E9800000F1800000F380000040
:108010000000000000000000000000000000000060
:10802000000000000000000000000000FB800000D5
:108030000000000000000000FF8000007DCC010077
:108040003515010079150100A9150100D9150100A8
:108050000916010039160100691601009916010080
:10806000C9160100F91601002D1701004117010082
:10807000511701008517010095170100A517010090
:10808000D91701001D18010065180100AD18010085
:10809000F51801003D1901004D1901008119010079
:1080A000B5190100E5190100191A01004D1A010066
:1080B0005D1A01006D1A0100A11A0100D51A010014
:1080C000EF72E8FF03B40148019001BD017F002079
:1080D0000448854600F02CFA0048004729110200A8
:1080E000C046C046903300201648804716480047D7
:1080F000FEE7FEE7FEE7FEE7FEE7FEE7FEE7FEE758
:10810000FEE7FEE7FEE7FEE7FEE7FEE7FEE7FEE747
:10811000FEE7FEE7FEE7FEE7FEE7FEE7FEE7FEE737
:10812000FEE7FEE7FEE7FEE7FEE7FEE7FEE7FEE727
:10813000FEE7FEE7FEE7FEE7FEE7FEE7FEE7FEE717
:10814000FEE7000081D20100D180000030B50B466F
:10815000014600202022012409E00D46D5409D4221
:1081600005D31D469540491B2546954040191546A7
:10817000521E002DF1DC30BD70B5002425460028CC
:1081800001DA01244042002901DA01254942FFF7C2
:10819000DDFFAC4200D04042002C00D0494270BD0F
:1081A000F0B51FB40646002082B005464024019178
:1081B00000901BE0019922460F46304600F066F918
:1081C000049A059B801A994110D3104619462246FD
:1081D00000F04CF9361A8F41019722460120002108
:1081E000009F00F043F938184D4100902046641E6E
:1081F0000028DFDC019B00982946324607B0F0BD1D
:10820000F0B51FB486B0002000900190029006984F
:10821000069980B204900798090C020400141143D7
:1082200007900027089D099806913E463C4603901A
:108230000398A9B20204000C039004982D0C154376
:1082400048430021224600F011F9C719714110344A
:108250000E46402CECDB3846029A00F007F9009AF3
:10826000019B8018009059410298019110300290B2
:108270004028CCDB00980BB0F0BD03460B439B07B6
:1082800003D009E008C9121F08C0042AFAD203E08B
:108290000B780370401C491C521EF9D27047D2B2B1
:1082A00001E00270401C491EFBD270470022F6E735
:1082B00010B513460A4604461946FFF7F0FF20465C
:1082C00010BD30B504460020034600E05B1C93421D
:1082D00003D2E05CCD5C401BF8D030BD0321001D13
:1082E000401E037812021A43491EF9D51046704702
:1082F000034603220870000A491C521EFAD518468C
:108300007047024670B54A40D30FDB0740002DD0BE
:108310004A002AD0010E140E000212020919400A66
:10832000520A8418E50104465443000A120A2E0436
:108330005043A4194219200CC543AA18120C012558
:10834000AD03521C521912047F39240400D0521C70
:10835000104301D44000491EC2B20C06C0092018C7
:10836000401C4008802A02D003E0002070BD400875
:108370004000002900DA0020184370BD70B50246A5
:108380004A40D50F40004A00ED0740085208002837
:1083900014D0002A12D0C40DD30D41020120C00513
:1083A0005202490A520AE41A091812187D349142FD
:1083B00001D3641C00E04900002C01DA002070BDEC
:1083C0000023914201D3891A034340084900002841
:1083D000F7D100290AD0914202D10121C90705E055
:1083E000914201D2012101E00121C943E005C018F9
:1083F000401900F05CF870BD10B5002296231146BC
:1084000000F05DF810BDC20FD207400040080BD04D
:10841000C10D0723DB01C91840020905400A1143B9
:10842000C208400711437047002001467047000012
:1084300010B5002904DB0124E40740428C412146A9
:10844000002B04DB1C460123DB075242A341994267
:1084500000D1904210BD00000122D207002800DBAD
:10846000101A002900DB511A8842704710B5202AE3
:1084700004DB0146203A9140002010BD91402023AA
:108480009C1A0346E3401943904010BD10B5202AC2
:1084900004DB0846203AD040002110BD0B46D340F3
:1084A000D0402024A21A91400843194610BD00294B
:1084B00004DA401C490001D140084000704770B404
:1084C0000024050C05D11024000402D1002921D07C
:1084D0001124050E01D100020834050F01D100015D
:1084E000241D850F01D18000A41C002801DB400061
:1084F000641C002908D020252E1B0D46F540A14004
:1085000000D001212943084301061B1B000ADB1D83
:1085100002D5002070BC7047DB05181880180029B0
:10852000F8DA401C4900F5D170BC400840007047A3
:10853000064C0125064E05E0E36807CC2B430C3CB6
:1085400098471034B442F7D3FFF7C6FD80250200E8
:10855000B025020070B58C180578401C6B075B0FC6
:1085600001D10378401C2A1106D10278401C03E097
:1085700006780E70401C491C5B1EF9D12B0705D4F0
:108580000023521E0DD40B70491CFAE70378401CDF
:10859000CB1A921C03E01D780D70491C5B1C521E07
:1085A000F9D5A142D8D3002070BD70B507F01EF9EF
:1085B0000524204618F072FD0025284607F00CF926
:1085C000204618F06BFD0126304607F0E3F8204600
:1085D00018F064FD284607F0DDF8204618F05EFD2F
:1085E000304607F0F9F8204618F058FD70BDB0B5D8
:1085F00007F0FCF80524204618F050FD0125284618
:1086000007F0EAF8204618F049FD284607F0C2F8BE
:10861000204618F043FD002007F0BCF8204618F073
:108620003DFDB0BDF0B581B007F0CEF8052018F0E3
:1086300035FD08270026012007F0ACF80524204668
:1086400018F02CFD204618F029FD07F0B3F8054678
:10865000204618F023FD002007F09CF8204618F073
:108660001DFD76002E437F1E3806E4D1F0B201B026
:10867000F0BD70B50446002007F08CF807F0B6F89E
:10868000052018F00BFD0826E0B2C00907F0A4F899
:108690000525284618F002FD012007F07BF8284642
:1086A00018F0FCFC002007F075F8284618F0F6FCDE
:1086B000284618F0F3FC6400761E3006E4D105204D
:1086C00018F0ECFC012070BDF0B583B001931446A6
:1086D0000E460746012038430290032504E000F0CF
:1086E0008EF86D1E280631D000F067F83846FFF787
:1086F000C0FF00F0A7F80028F1D13046FFF7B9FF1E
:1087000000F0A0F80028EAD100F057F80298FFF72F
:10871000B0FF00F097F80028E1D1019802280BD3B0
:10872000451E0026FFF77EFF2070FFF73EFF641C0A
:10873000761CF0B28542F5DCFFF774FF2070FFF77E
:1087400056FF00F05CF8202003B0F0BD102003B00D
:10875000F0BDF0B583B01C46009201910290032554
:1087600004E000F04CF86D1E280623D000F025F838
:108770000298FFF77EFF00F065F80028F1D101981C
:10878000FFF777FF00F05EF80028EAD1002C0CD04C
:108790000026009F3878FFF76CFF00F053F80028A0
:1087A000DFD1761C7F1CA642F4D300F028F8082005
:1087B00003B0F0BD102003B0F0BDB0B507F016F85F
:1087C0000524204618F06AFC0125284606F0E2FF41
:1087D000204618F063FC284606F0FEFF204618F0FD
:1087E0005DFC0025284606F0F7FF204618F056FCF1
:1087F000284606F0CFFF642018F050FCB0BDB0B59D
:1088000006F0F4FF0524204618F048FC0025284611
:1088100006F0C0FF204618F041FC284606F0DCFFB9
:10882000204618F03BFC0125284606F0B3FF204601
:1088300018F034FC284606F0CFFF642018F02EFC18
:10884000B0BD0000B0B506F0BFFF0524204618F00B
:1088500025FC012006F09EFF204618F01FFC0B4D62
:1088600006F0A8FF044606F08FFF002C02D06D1E14
:108870002804F5D10525284618F010FC002006F044
:1088800089FF284618F00AFC2046B0BD33210000BD
:10889000034801780B2901D8491C01707047C04674
:1088A0007B2F002070B584B00025039502950195BB
:1088B000009506F069FF0F20C6430E4C1036F1B24A
:1088C000A0206A461023FFF744FF204618F0E6FB7D
:1088D000204618F0E3FB912EF0D3A020B0216A4689
:1088E0001023FFF736FF204618F0D8FB024805801A
:1088F00004B070BD581B00006E2F002070B5022917
:1089000002D2EB24E0B270BD891EEB250022134693
:1089100005E0401C5B1CDDB2A94225460EDB047855
:108920006C40154604E034466E1C072D3546F0D2E7
:108930006608E407F7D09A246640F4E7E0B270BD19
:10894000F0B591B00C91417810AA117083781B0298
:108950005918C37804792402E3181B0459180B0E24
:10896000D3700C0C94700D0A55700B910895691812
:10897000099409190A93C9180278D24389184279CF
:1089800083791B029A18C379047A2402E3181B0422
:108990009A188918130A0693C918130C0593C91855
:1089A0000792120E04928918827AC37A1B029A18CF
:1089B000037B0F90447B2402E3181B0498180918CA
:1089C000020A02928918020C019289180D910390F3
:1089D000000E0E9000200346014606E032409A4009
:1089E000D2B211435B1C082B0ED0012635469D40A8
:1089F0000746024602E07F1C042FEFD010ACE45D76
:108A00002542F8D0521CF6E70E9C0D980019C3B20F
:108A10000F98827B934205D0427A914202D1002086
:108A200011B0F0BD1021FFF769FF0C99CC72019ACB
:108A30008A72029A4A72039A0A72049ACA71059A51
:108A40008A71069A4A71079A0A710A9ACA70099A33
:108A50008A70089A4A700B9A0A7011B0F0BDF0B58E
:108A60008DB055220270002747720B784370CA7987
:108A7000059202728A790492C2714A7903928271D4
:108A80000A7902924271CA7A089242738A7A0192F2
:108A900002734E7AC6720C7A84720CAA13704D78E7
:108AA0002D02EB188D78C978090249190904CB18F1
:108AB000190E01711D0CC57009931B0A0B90837070
:108AC00038460A91D170079595700693537031021C
:108AD0000919089A1202019BD21812045118089120
:108AE00003990902029A8918059A1202049BD21866
:108AF0001204511805913D463A4605E02640AE4025
:108B000032436D1C082D0ED001242146A940034696
:108B1000064602E05B1C042BF0D00CAFFF5C394230
:108B2000F8D0761CF6E70B9B5A7209980699401804
:108B3000079940180A994018059A8018110A401898
:108B4000110C4018110E4018089A8018110A40188C
:108B5000110C4018110E4018563898731021184601
:108B6000FFF7CCFE0DB0F0BDF0B58FB00446FF208E
:108B7000E070A07060700F20C04302900F30207032
:108B8000704818F08BFA70490868632801D864208F
:108B900008606E4F002038806D4E0190308008E0F4
:108BA0000B99814222D338881030388080B2A128B6
:108BB0006DD206F0E9FD3978A02003AA1023FFF753
:108BC00083FD30802028EED103AD0BA92846FFF7A6
:108BD000B7FEE97B8842E6D128785528E3D15D4885
:108BE000017800290298DBD10846D9E73888A02807
:108BF0004DD8C0B20021019105E006F0C5FD3988CD
:108C0000C8B2A12943D2C1B2A02003AA1023FFF702
:108C10005BFD3080398810313980202837D103AD91
:108C200007A92846FFF78CFEE97B8842E5D1287822
:108C30005528E2D1474800780028029900D1014622
:108C400007988842D9D240490A68962151430B9A25
:108C5000824208D90818904219D30BA90E22204647
:108C6000FFF70BFBC9E78918814210D307A90E2231
:108C70002046FFF702FB0BA80A99818107980B9009
:108C800008980C9009980D9038880190B5E72078E5
:108C9000617809020818A178E278120251180904D3
:108CA0000818401C24D1002001903880A020B02159
:108CB00003AA1023FFF708FD3080202818D103AD48
:108CC0000BA92846FFF73CFEE97B884210D12878A3
:108CD00055280DD11F480078002800D102900B982C
:108CE0000299884204D20BA90E222046FFF7C5FA4A
:108CF0002078617809020818A178E27812025118E8
:108D000009040818401C0CD10020E072A0726072A7
:108D10002072E071A07160712071E070A0706070CD
:108D20002070019838802078617809020818A178AD
:108D3000E2781202511809040818074908603088BF
:108D40000FB0F0BD70110100682F00206E2F0020C1
:108D5000642F0020672F0020742F0020F0B581B011
:108D600000910646214800250570002A2ED01446A1
:108D7000C036631B71190F2008401022101A83425D
:108D800000D303461A480278102A01D0042A1AD1C7
:108D9000C809FE2707405F2F13D80127B843603862
:108DA000C0B29E3282420CD3009A5219C9B2DFB2CD
:108DB0003B46FFF789FC0F490880ED19A542D8D33F
:108DC00004E0082000E004200A49088009480188DE
:108DD0000020042902D0082900D00120034908708E
:108DE000411E8841400001B0F0BDC0467A2F0020EE
:108DF000662F0020782F00200A4A012313700A4AA8
:108E000010700A4A11600A4A00211160042801D139
:108E100005218901102801D11D208101054801800B
:108E20007047C046672F0020662F0020682F002063
:108E3000742F00206C2F0020F0B587B0994D0026CC
:108E40002E80994B1B688B4224D1994C2188202974
:108E500025D1029000920196964C00272760964DEE
:108E6000964E2878062809D806F08EFC2068401C0B
:108E70002060B042F5D38D48042101802F70904CC2
:108E800020880107029B31D0884820210180854D30
:108E9000019E0BE0012040028449088006E003A8FF
:108EA000FFF762FE20808148802101807F48008892
:108EB0003F2807DD874988420BDC402812D08028F4
:108EC00010D010E004280DD008280AD0202809D09E
:108ED00009E001214A02904204D0C902884201D02F
:108EE00001E002262E80288807B0F0BDA128019E4F
:108EF00000D32780009A012A6A4D1ED1187B0128D1
:108F000056D1DF719F715F711F711F73587B0128EC
:108F100004D1DF729F725F721F725F7303AF3846B6
:108F20001946FFF79CFDF8732088002846D01038BA
:108F3000C1B2A02003AA102344E0002AB6D16148A0
:108F400001780029B2D002701878597809020818FF
:108F50009978DA7812025118090408185A490978E0
:108F6000002901D00F21C943884233D2274603ACE0
:108F700020461946FFF773FDE0733978A0201023CF
:108F80002246FFF7E6FB029A4849088008288DD15F
:108F90003888103038801078517809020818917894
:108FA000D2781202511809040818484908607DE770
:108FB000597B012911D10128A3D0A7E7A02003AA3A
:108FC00010230146FFF7C5FB384908803D4800994A
:108FD00001706BE70120C0025EE73D480078012880
:108FE00012D103AC20461946FFF739FDE073A020EB
:108FF000B02110232246FFF7ACFB2C49088008283B
:10900000E4D133480770E1E7187859780902081865
:109010009978DA7812025118090408182B4909685E
:10902000214A12685118884203D220484021018009
:10903000CCE725490978002901D00F21C94388428E
:109040002DD203AF384619461C46FFF708FDF873CA
:109050001B480178A02010233A46FFF77AFB1349FA
:1090600008800828B2D11649088810300880207876
:10907000617809020818A178E278120251180904EF
:1090800008181249086008490A6815215143FFF77A
:109090005DF800299AD101200D49087096E701205A
:1090A000C00291E7802F0020682F00207E2F002033
:1090B000642F0020842F00207B2F0020818D5B00F7
:1090C0006E2F0020702F0020672F0020742F0020AB
:1090D0007C2F0020FF010000F0B585B00646434C10
:1090E0000027278004921018414A1288904241D2EA
:1090F00001910397404F0020029038603F4C404D53
:109100002078052809D806F03FFB3868401C3860F5
:10911000A842F5D3374804210180029820703948CD
:10912000018839480278102A01D0042A32D18819DE
:109130000346C033049C651A0F2404401020001B12
:10914000854200DB0546DC09603C01263002E7B2BF
:109150007F09052F12D3B443E6B29E32B242234CAC
:10916000039F0DD301984218D9B2EBB23046FFF7F6
:10917000F0FA05E01F482021018011E01B4C039FFD
:109180001C49088008280BD1E8B21E4A118808182B
:10919000108005E00120800216490880134C039FCF
:1091A000144800881F2809DD202813D001210A0255
:1091B00090420FD0890288420CD00CE0042809D0DC
:1091C000082808D10F4800880499884201D3022753
:1091D00000E001272780208802210143022902D1D3
:1091E000084900220A8005B0F0BDC046802F00204B
:1091F0006C2F00207E2F0020842F00207B2F00204A
:10920000818D5B00882F0020662F0020F0B585B08F
:10921000044600200190042C6FD20CF06FF9002856
:1092200001D10CF0EBF90020009000BF0098401C29
:1092300000900CF063F903900398002803D048498C
:1092400000988842F2D30398002856D1042145485B
:109250000CF036F94448454908802101444A515CE4
:109260004900404A505A41490A880121090300F047
:1092700055F902900120049020013D4940184078A2
:10928000002801D100264BE02001394940184078E0
:10929000012802D13548068842E0200134494018AF
:1092A000407802282AD12001401805792901304A46
:1092B000515C49002B4A505A2C490A880121090364
:1092C00000F02CF9064628012A49431828012849AC
:1092D00040180289280140180021C7683046B84765
:1092E00006462801224BC018C2882801C018817880
:1092F000304600F087F8064612E02DE020011C49B8
:1093000040184078032804D02001401840781328E2
:1093100004D1200116494018868801E000200490FD
:109320000498002818D02001124943182001104940
:1093300040180289200140183146C7680298B84792
:10934000019020010A4BC018C2882001C018817802
:10935000019800F057F80190019805B0F0BD0000A9
:1093600050C30000F600002088130000F000002029
:109370001C1C02005C1C0200F8B505460E46144693
:109380000020009001211C4801751C48007888438A
:109390001A490870084680780821084317498870E0
:1093A000002088710846007801210843134908709D
:1093B00008460572002717E010480078802108430E
:1093C0000E49087000BF0E48007D0028FBD0002029
:1093D0000B4908750948C0892080A41C0748C18929
:1093E0000098081800907F1CB742E5D331460098DA
:1093F000FEF7ACFE80B2F8BD406100400050044072
:109400004060004010B50346012908D1094CA41A58
:109410009C4202D99C18A0B20BE0064809E0022940
:1094200006D1934202DD9C1AA0B202E0002000E0C7
:10943000184610BDFFFF000010B504460121202092
:1094400001F0E8FF00203249087001213148017520
:10945000002031490875152017F008FB2C4880784A
:10946000E17808432A4988700846807821780843C3
:10947000274988702078802806D108460079E1794C
:10948000490008432249087121488078E17A08435D
:109490001F498870A078002803D108460079087118
:1094A0000FE0A078012806D119480079602108430F
:1094B0001749087105E016480079802108431449CE
:1094C0000871134880792179084311498871084649
:1094D0008079617908430E498871207AC872607A70
:1094E0008872084600783821884309490870084680
:1094F00000786178C900084305490870A07A0873AC
:1095000008460078012108430149087010BD000099
:10951000005004404061004040600040F8B50446FF
:109520000E461746002E01D100250FE0A64201DCB1
:109530003D460BE00094009C204678430090314665
:109540000098FEF703FE0090009885B22846F8BD0B
:109550000146042904D28A00024BD218508800E048
:1095600000207047342900200146042903D28A00D4
:10957000024B985C00E00020704700003429002076
:10958000FFB587B004460898844203DA0A988068D9
:10959000002802D12448019042E00898001B82B2C2
:1095A0000292002625460A98806800212F463A46F6
:1095B0003346049605910690FEF722FE05460E46B8
:1095C000002328463146029AFEF7EAFD05460E467C
:1095D000304600210A4649405040014302D012481B
:1095E00001901DE003950A98C068039DA84202D32C
:1095F0000020019014E00A98C1680398401A039073
:1096000009990398FEF7A2FD03900398000C00044B
:10961000002802D00448019002E0039880B2019033
:1096200001980BB0F0BD0000FFFF000010B5084826
:10963000007880218843064908700121054801759A
:10964000002005490875152017F010FA10BD00001C
:10965000005004404061004040600040F8B50546BD
:109660000E4614461F4621462846FEF785FD80B269
:10967000F8BD0000FFB587B006460A98406800288C
:1096800001D1029035E00A980168406808180390FB
:10969000002534460021274603980695049105903D
:1096A00038462946049B059AFEF7AAFD04460D4656
:1096B0000A98406802460023019020462946FEF79A
:1096C0006FFD04460D46002320462946099AFEF701
:1096D00067FD04460D4628460749214000235940AE
:1096E0005840014303D00448C043029001E0A0B2B7
:1096F000029002980BB0F0BD0000FFFF10B5FE48CD
:1097000000688079030017F097F907059ED8F5F4F3
:10971000F3F2F100F84800684079030017F08CF983
:109720000805138A2A8A468A638A13F0DFF9002023
:10973000F1490968C873F04800684079401CEE4957
:10974000096848717DE0ED494969EB4A1268D27AAF
:10975000885C13F043FAE84800684079401CE64909
:1097600009684871E44800684079401CE24909688A
:10977000487166E00AF028F9002810D113F02EFA9B
:10978000DD4800684079401CDB4909684871DA48C7
:1097900000684079401CD8490968487105E013F019
:1097A000CFF90020D449096848714AE00AF00CF961
:1097B000002811D1112013F011FACF480068407928
:1097C000401CCD4909684871CB4800684079401C6D
:1097D000C9490968487105E013F0B2F90020C6498B
:1097E000096848712DE00AF0EFF800281BD1C24843
:1097F0000068C07A401CC0490968C872BE48006849
:10980000C07ABE49097888420DDB0020BA49096850
:10981000C872B94909684862B74800688079401C35
:10982000B5490968887113F08BF90020B2490968BD
:10983000487106E013F084F90020AF4909684871C7
:1098400000BF00BF32E3AC480068407C002817D05E
:10985000AA48C068002803D0A848C16819208847D2
:109860000020A54909684862A34800688079401C27
:10987000A1490968887100209F49096848711BE067
:109880009D480068406A282807D29B480068406AC3
:10989000401C9949096848620EE000209649096811
:1098A0004862954800688079401C9349096888712E
:1098B0000020914909684871F8E28F4800684079B2
:1098C000030017F0B9F8080518A42FA44CA480A42D
:1098D00013F00CF9002088490968C87386480068AD
:1098E0004079401C84490968487197E0D4E2C7E296
:1098F00030E25DE194E0814949697F4A1268D27A99
:10990000885C13F06BF97C4800684079401C7A4908
:1099100009684871784800684079401C76490968B0
:1099200048717BE00AF050F8002811D1012013F0B3
:1099300055F9714800684079401C6F4909684871C1
:109940006D4800684079401C6B490968487105E022
:1099500013F0F6F800206849096848715EE00AF0E3
:1099600033F8002828D164490968C97A2422514370
:10997000634A12688918604A1268D27B885C13F0C7
:109980002DF95D480068C07B401C5B490968C873BD
:1099900059480068C07B242814D357480068407990
:1099A000401C554909684871534800684079401C7B
:1099B00051490968487105E013F0C2F800204E498A
:1099C000096848712AE009F0FFFF002818D14A48C9
:1099D0000068C07A401C48490968C8724648006857
:1099E000C07A4649097888420ADB00204249096862
:1099F000C872414800688079401C3F4909688871F5
:109A000013F09EF800203C490968487106E013F005
:109A100097F8002038490968487100BF00BF45E247
:109A2000354800684079030017F006F80A0614B9B3
:109A30002BB948B978B995B913F058F800202E49D8
:109A40000968C8732C4800684079401C2A49096895
:109A50004871ABE029494969274A1268D27A885C83
:109A600013F0BCF8244800684079401C224909687A
:109A70004871214800684079401C1F4909684871B5
:109A800094E009F0A1FF002811D14A2013F0A6F8B4
:109A9000194800684079401C174909684871164800
:109AA00000684079401C14490968487105E013F0CA
:109AB00047F8002010490968487177E009F084FFF1
:109AC000002824D1FF2013F089F80B480068C07BE0
:109AD000401C09490968C87307480068C07B2428EE
:109AE0001BD3054800684079401C03490968487148
:109AF00001480068407905E0E00700204C2F002075
:109B0000DC070020401CEA490968487105E013F0B1
:109B100017F80020E6490968487147E009F054FF4A
:109B2000002811D1FF2013F059F8E148006840796E
:109B3000401CDF4909684871DD4800684079401CD5
:109B4000DB490968487105E012F0FAFF0020D849A6
:109B5000096848712AE009F037FF002818D1D44875
:109B60000068C07A401CD2490968C872D0480068B1
:109B7000C07AD049097888420ADB0020CC490968BC
:109B8000C872CB4800688079401CC949096888714F
:109B900012F0D6FF0020C6490968487106E012F0AD
:109BA000CFFF0020C2490968487100BF00BF7DE1B6
:109BB000BF4800684079030016F03EFF0C0715C34C
:109BC0002CC349C366C382C39FC312F08FFF00201A
:109BD000B7490968C873B64800684079401CB44961
:109BE00009684871B4E0B3494969B14A1268D27A48
:109BF000885C12F0F3FFAE4800684079401CAC4925
:109C000009684871AA4800684079401CA849096859
:109C100048719DE009F0D8FE002811D1772012F09C
:109C2000DDFFA34800684079401CA14909684871DC
:109C30009F4800684079401C9D490968487105E0CB
:109C400012F07EFF00209A490968487180E009F00F
:109C5000BBFE002811D10C2012F0C0FF9448006810
:109C60004079401C924909684871914800684079E0
:109C7000401C8F490968487105E012F061FF00201F
:109C80008B490968487163E009F09EFE002810D1F5
:109C900012F0A4FF864800684079401C8449096896
:109CA0004871834800684079401C814909684871BF
:109CB00005E012F045FF00207D490968487147E042
:109CC00009F082FE002811D1132012F087FF784896
:109CD00000684079401C76490968487174480068FA
:109CE0004079401C72490968487105E012F028FF6C
:109CF00000206F49096848712AE009F065FE0028D4
:109D000018D16B480068C07A401C69490968C8725C
:109D100067480068C07A6749097888420ADB0020F2
:109D200063490968C872624800688079401C6049CC
:109D30000968887112F004FF00205D4909684871C4
:109D400006E012F0FDFE002059490968487100BF85
:109D500000BFABE0564800684079030016F06CFE87
:109D6000080513872A874787638712F0BFFE002004
:109D70004F490968C8734E4800684079401C4C49F7
:109D8000096848717AE04B494969494A1268D27AB0
:109D9000885C12F023FF464800684079401C444923
:109DA00009684871424800684079401C4049096888
:109DB000487163E009F008FE002811D1492012F033
:109DC0000DFF3B4800684079401C394909684871DB
:109DD000374800684079401C35490968487105E0FA
:109DE00012F0AEFE002032490968487146E009F0E1
:109DF000EBFD002810D112F0F1FE2D4800684079EB
:109E0000401C2B4909684871294800684079401C6A
:109E100027490968487105E012F092FE00202449A4
:109E2000096848712AE009F0CFFD002818D12048C0
:109E30000068C07A401C1E490968C8721C48006846
:109E4000C07A1C49097888420ADB00201849096851
:109E5000C872174800688079401C154909688871E4
:109E600012F06EFE002012490968487106E012F0F7
:109E700067FE00200E490968487100BF00BF15E069
:109E800000200B4909688871094909684871062052
:109E900007490968C87009E012F052FE0020044921
:109EA0000968487102490968887100BF00BF10BD88
:109EB000E00700204C2F002010B56A480068407968
:109EC000030016F0B9FD090610C627C644C6608E09
:109ED000C60012F00BFE634800684079401C6149DF
:109EE00009684871BCE0604949695E4A1268D27AE3
:109EF000885C12F073FE5B4800684079401C594949
:109F000009684871574800684079401C55490968FC
:109F10004871A5E009F058FD002811D17F2012F00A
:109F20005DFE504800684079401C4E490968487100
:109F30004C4800684079401C4A490968487105E06E
:109F400012F0FEFD002047490968487188E009F0D9
:109F50003BFD002810D112F041FE424800684079D4
:109F6000401C4049096848713E4800684079401CDF
:109F70003C490968487105E012F0E2FD00203949CA
:109F8000096848716CE009F01FFD002822D13548AE
:109F90000068C07A401C33490968C87231480068BB
:109FA000C07A3149097888420FDB00202D490968C1
:109FB000C8722C4800684079401C2A4909684871D9
:109FC000002028490968486208E0002025490968FE
:109FD000487103E0002023490968487112F0B0FD80
:109FE0003EE020480068407C002816D01E48C0682B
:109FF000002803D01C48C16819208847002019494F
:10A0000009684862174909684871164909688871E2
:10A01000052014490968C8701AE012480068406AAF
:10A02000282807D20F480068406A401C0D4909687B
:10A0300048620DE000200B49096848620949096837
:10A040004871084909688871052006490968C8707F
:10A0500006E012F075FD002002490968487100BF52
:10A0600000BF10BDE00700204C2F002010B50024D9
:10A07000F7480068807A01287ED1F5480068C079E9
:10A0800000287AD0F24800688079002804D001289E
:10A0900074D0022873D191E1ED480068007B242838
:10A0A0006ED2EB480068C07901287AD1002475E0AF
:10A0B000E7480068C07A24214843E6490968401807
:10A0C000E3490968097B415CE1480068C07A2422C1
:10A0D0005043E14A12688018DD4A1268127B805CA6
:10A0E000814229D0DA480068C07A24214843DA49FD
:10A0F00009684018D6490968097B415CD448006862
:10A10000C07A24225043D34A12688018D04A126879
:10A11000127B8154CE480068407B242805D3CC486C
:10A120000068007BCA4909684873C9480068007B19
:10A13000C7490968887308E0C5480068407B24283F
:10A1400003D20120C24909688871C1480068007BB8
:10A15000401CBF4909680873BD480068007B24287B
:10A1600008D3BB480068407B242803D20120B849AB
:10A1700009688871B64805E0D3E1CDE169E0BAE14C
:10A1800038E00EE00068007B242804D2B048006864
:10A190008079012800D103E0601CC4B2242C87D34D
:10A1A00056E0002413E0AA480068C07A24214843FE
:10A1B000A94909684018015DA5480068C07A2422B1
:10A1C0005043A44A126880180155601CC4B2242C64
:10A1D000E9D300209E490968487323209C490968F7
:10A1E000887301209A490968887124209849096870
:10A1F00008732DE0002096490968087394480068A8
:10A20000C07A401C92490968C87291480068C07AB7
:10A2100092490978884217DB8D480068007C012844
:10A2200004D102208A490968887106E00020884923
:10A230000968887186490968C871002084490968DD
:10A24000C872834909680874002081490968487107
:10A2500061E17F4800684079030016F0EDFB0805D6
:10A2600013A62AA651A68EA601207949096808746A
:10A2700012F03CFC764800684079401C744909683B
:10A28000487199E075494969714A1268D27A885CC7
:10A2900012F0A4FC6E4800684079401C6C490968C3
:10A2A00048716B4800684079401C694909684871E9
:10A2B00082E009F089FB00281BD165490968497BC8
:10A2C000491CC8B212F08AFC61480068407B6049B2
:10A2D0000968C8735E4800684079401C5C49096899
:10A2E00048715B4800684079401C594909684871C9
:10A2F00005E012F025FC00205549096848715BE033
:10A3000009F062FB00282BD151490968C97A24223F
:10A310005143504A126889184D4A1268D27B885CB2
:10A3200012F05CFC4A480068C07B401C4849096840
:10A33000C87347480068C07B45490968897B8842E3
:10A340001ADD434800684079401C4149096848715A
:10A350003F4800684079401C3D49096848710BE05E
:10A3600012F0EEFB3A480068407B39490968C8732F
:10A3700000203749096848711EE009F025FB0028D4
:10A380000CD1334909688871242031490968C873A0
:10A390002F49096848732E490968887312F0D0FB69
:10A3A00000202B490968487106E012F0C9FB002023
:10A3B00027490968487100BF00BFACE02448006825
:10A3C0004079030016F038FB08050F8E268E4C8E60
:10A3D000688E12F08BFB1E4800684079401C1C49B7
:10A3E0000968487185E01D494969194A1268D27A9D
:10A3F000885C12F0F3FB164800684079401C144951
:10A4000009684871124800684079401C1049096881
:10A4100048716EE009F0D8FA002811D1492012F0F5
:10A42000DDFB0B4800684079401C09490968487108
:10A43000074800684079401C05490968487105E0F3
:10A4400012F07EFB002002490968487151E00000CB
:10A45000E0070020DC070020D80700204C2F002058
:10A4600009F0B2FA002810D112F0B8FB9C4800683D
:10A470004079401C9A4909684871994800684079B8
:10A48000401C97490968487105E012F059FB00200B
:10A490009349096848712CE009F096FA00281AD10E
:10A4A0008F480068C07A401C8D490968C8728C4882
:10A4B0000068C07A8B49097888420CDB0020884903
:10A4C0000968C872864909688871854909684871B0
:10A4D00083490968C87112F033FB0020804909687C
:10A4E000487106E012F02CFB00207D490968487194
:10A4F00000BF00BF0FE012F023FB0020784909687D
:10A500004871774909688871754909680873744901
:10A510000968C87200BFE2E00020714909688872CA
:10A52000DDE06F480068807A0228F4D16C4800684A
:10A53000007A002879D06A4800684079030016F054
:10A540007BFA0B0711BB25BB41545EBB7590BB006A
:10A5500012F0CCFA624800684079401C60490968F2
:10A560004871B7E05F494969087812F037FB5C48E9
:10A5700000684079401C5A49096848715848006889
:10A580004079401C564909684871A3E009F01CFA5B
:10A59000002810D112F022FB514800684079401C7D
:10A5A0004F49096848714E4800684079401C4C4941
:10A5B0000968487105E012F0C3FA002048490968AB
:10A5C000487187E009F000FA002807D14448006884
:10A5D0004079401C42490968487103E00020404925
:10A5E0000968487112F0ACFA74E012F07FFA3C4846
:10A5F00000684079401C3A49096848716AE0394965
:10A6000049690978491CC8B212F0E8FA3448006870
:10A610004079401C324909684871314800684079E6
:10A62000401C2F490968487154E054E009F0CCF906
:10A6300000280FD112F02CFA2949096888700120EE
:10A6400012F0A0FA264800684079401C24490968A5
:10A65000487105E012F074FA002021490968487138
:10A6600038E01F480068807811280CD100201C4970
:10A6700009680872AA201A490968887000201849D8
:10A680000968487011E0164800684078401C144979
:10A6900009684870124800684078032805D309F01B
:10A6A00033FA00200E490968487012F049FA002078
:10A6B0000B49096848710DE012F042FA0020084980
:10A6C00009684871064909684870AA200449096860
:10A6D000887000BF03E0002001490968887210BD3E
:10A6E000E00700204C2F0020F0B505460C4616462A
:10A6F0001F462088482806DA3A462946304605F0A3
:10A700007DF8012800D0F0BD2088C0002E502088A0
:10A71000401C208000BFF6E710B502469000074BB2
:10A72000C018405C002802D00320C04310BD0120A7
:10A730009300024C1B1958540020F7E7C82A002048
:10A7400070B5002508E06D1C1B48854202D20AF056
:10A7500081FF01E0002503E00AF0D0FE0028F2D1DD
:10A7600000BF022100200AF0D7FE032100200AF0DA
:10A77000D3FE052100200AF0CFFE072100200AF0B9
:10A78000CBFE002408E00020A1000C4A5054A10098
:10A7900089184880601CC4B2042CF4D301200849F5
:10A7A000087000204870052088700020C870054897
:10A7B0000549088070BD000050C300003429002006
:10A7C000F200002088130000F0000020F8B58D484A
:10A7D0000078030016F030F9060405163D5EFDFC16
:10A7E0000EE10AF00BFF00208649C8704870084649
:10A7F0008078002802D10320087002E002208149FD
:10A800000870FDE07F488078002804D07D4880787B
:10A81000401E7C4988700AF071FE00280BD10AF0B6
:10A82000EDFE00207749C8700846807800280FD1D7
:10A83000032008700CE07348C078401C7149C87050
:10A840000846C078052803D3052008700AF002FFE7
:10A85000D6E00AF053FE00280ED104216A480AF01F
:10A860002FFE00206749C870487068486849088012
:10A870000420644908700CE06248C078401C6149BB
:10A88000C8700846C078052803D3052008700AF070
:10A89000E1FEB5E05B49497809015E4A515C490037
:10A8A000594A505A5A490A8801210903FEF736FECF
:10A8B00000900125534840780001564940184078DF
:10A8C000002801D100243CE04E4840780001514965
:10A8D00040184078012802D14D48048831E04948A9
:10A8E000407800014B4940184078022812D1454970
:10A8F00049780901474A89180879FEF729FE044674
:10A90000404949780901434A89180879FEF72CFE25
:10A91000054616E03B48407800013E494018407823
:10A92000032806D0374840780001401840781328A3
:10A9300006D134484078000136494018848800E048
:10A940000025002D2FD02F484078000132494318B0
:10A950002C48407800012F49401802892948407846
:10A96000000140182146C7680098B84706462548A8
:10A9700040780001274BC018C28822484078000167
:10A98000C01881783046FEF73DFD06461D484078E8
:10A99000800022494018468001201A4949788900E0
:10A9A0001E4A50540AE000201649497889001B4A83
:10A9B00089184880134949788900505411484078D3
:10A9C000401C1049487008464078042809D301E02B
:10A9D00013E007E00AF012FE00200A494870032045
:10A9E00008700DE00AF08AFD002803D10120054916
:10A9F000087001E00AF02EFE02E0FFF7A1FE00BFA2
:10AA000000BFF8BDF2000020F6000020881300000F
:10AA1000F00000201C1C02005C1C020034290020F5
:10AA200010B50AF035FD002405E00020A100074A1A
:10AA30005054601CC4B2042CF7D3002004490870A1
:10AA40000520887003480449088010BD342900207F
:10AA5000F200002088130000F000002070B50446CA
:10AA6000002000F0AFF8002000F0DAF8002000F03D
:10AA70009BF8002000F0C4F8002000F087F80020C8
:10AA800000F0AEF800BF012000F08EF8012000F0C9
:10AA9000B7F8002521E0002000F086F8002000F043
:10AAA000AFF880202040002806D0012000F08AF86E
:10AAB000012000F0B5F805E0002000F083F8002048
:10AAC00000F0AEF800BF012000F06EF8012000F0A9
:10AAD00097F86006040E681CC5B2082DDBDB012068
:10AAE00000F054F8012000F07BF870BD70B504460A
:10AAF0000D46012000F066F8012000F091F80020DA
:10AB000000F052F8002000F07BF8002000F03EF842
:10AB1000002000F065F800BF012000F045F801209A
:10AB200000F06EF8002628E0002000F03DF800203C
:10AB300000F066F880202040002803D0012000F0BB
:10AB400041F802E0002000F03DF880202840002875
:10AB500003D0012000F064F802E0002000F060F86B
:10AB600000BF012000F020F8012000F049F8600645
:10AB7000040E6806050E701CC6B2082ED4DB012038
:10AB800000F004F8012000F02BF870BD10B5044669
:10AB9000002C04D0012103200AF05AFE03E000211A
:10ABA00003200AF055FE10BD10B50446002C04D059
:10ABB000012104200AF04CFE03E0002104200AF0E9
:10ABC00047FE10BD10B50446002C04D00121022020
:10ABD0000AF03EFE03E0002102200AF039FE10BD1B
:10ABE00010B50446002C04D0012104480AF030FEC0
:10ABF00003E0002101480AF02BFE10BD0107000010
:10AC000010B50446002C05D00121072000020AF0EF
:10AC10001FFE04E00021072000020AF019FE10BD0B
:10AC200010B50446002C04D0012104480AF010FE9F
:10AC300003E0002101480AF00BFE10BD02070000EE
:10AC400010B5F920FFF70AFF3221424805F018FE3F
:10AC50008820FFF703FF9020FFF700FF9820FFF701
:10AC6000FDFE08210846FFF741FFE820FFF7F6FE4A
:10AC700012210846FFF73AFFA020FFF7EFFE7021F0
:10AC80000846FFF733FFA820FFF7E8FE70210846CB
:10AC9000FFF72CFFB020FFF7E1FE70210846FFF719
:10ACA00025FFB820FFF7DAFE00210846FFF71EFF58
:10ACB000C020FFF7D3FE00210846FFF717FFC8208A
:10ACC000FFF7CCFE00210846FFF710FFD020FFF76A
:10ACD000C5FE2F210846FFF709FFD820FFF7BEFE6B
:10ACE0002F210846FFF702FFE020FFF7B7FE2F21D4
:10ACF0000846FFF7FBFE4020FFF7B0FE00210846A4
:10AD0000FFF7F4FE0A20FFF7A9FE002405E000216A
:10AD10000846FFF7EBFE601CC4B25A2CF7DB002498
:10AD20000AE000200C4908550C4908550C49085503
:10AD30000C490855601CC4B25A2CF2DB8120FFF785
:10AD40008DFE0020084908708870C870087148702E
:10AD500010BD0000204E00005C260020B62600201A
:10AD6000102700206A270020C800002010B580208E
:10AD7000FFF774FE10BD0000002004490870012098
:10AD8000034908700020487070470000CD00002083
:10AD9000C800002010B54848007800287AD04648FE
:10ADA0008078030015F048FE0604434A535A687E33
:10ADB000414800794149085C3F490979404A515C62
:10ADC000884209D13C4800793E49085C3A490979F2
:10ADD0003D4A515C88421BD0374800793749085CAE
:10ADE00035490979364A5054334800793549085C69
:10ADF00031490979344A50542F48C078002803D08B
:10AE000004202D49887011E001202B4988700DE045
:10AE100000202949C87008460079401C087108467E
:10AE200000795A2802DB00200871087041E04020B8
:10AE3000FFF714FE0220204988703AE01E4A11797B
:10AE40001079FFF753FE03201B49887031E00A2078
:10AE5000FFF704FE0420184988702AE0164A127988
:10AE6000194B995C144A1279154B985CFFF73EFE1A
:10AE70000520114988701CE00F480079401C0E49DC
:10AE80000871084600795A2805DB0020087108700F
:10AE9000C87003E00EE001200749C8700020064991
:10AEA000887006E00020044908708870C870087136
:10AEB00000BF00BF10BD0000C80000205C260020BD
:10AEC000B6260020102700206A27002010B512F0B7
:10AED00045FA012812D1072009F0A0FB002806D06E
:10AEE0004B22D2000021012013F066FF0BE07D22EF
:10AEF000D2000021012013F05FFF04E00022114680
:10AF0000012013F059FF10BD00200349087248705A
:10AF10008870486070470000600A00205822115273
:10AF2000704710B504460121022000F073FA002199
:10AF3000022000F06FFA10BD014600205322525C3F
:10AF400010231A40002A08D05322525C0C231A40C6
:10AF50009210032A18D1032016E05422525A0123DA
:10AF6000DB031A40002A0ED05322525C0C231A40F5
:10AF70009210032A05D05322525C9207920F032AA3
:10AF800001D1022000E00120704702460020582332
:10AF90009B5A0B40002B01D0012000E0002070479D
:10AFA000014600226020405AFF231B021840000582
:10AFB000020F1001014BC0187047000000550440FB
:10AFC00010B5002A0AD056231B5A0C0223435624DC
:10AFD000235256231B5A8B43235209E056231B5AF4
:10AFE0000C02A3435624235256231B5A0B432352CD
:10AFF00010BD0000F8B504460D4601270026344870
:10B00000844203D10121022000F004FA2878401E76
:10B01000A0702088FF21013108432080208840084B
:10B0200040002080A878401EC1B25A20015568799E
:10B030000007000CE97909020843A97908435C215B
:10B040000853288981B240200153A868C000C10C70
:10B0500042200153A88981B244200153E868C0000E
:10B06000C10C46200153288A81B248200153286927
:10B07000C000C10C4A200153A88A81B24C20015360
:10B080006869C000C10C4E2001535020005B297933
:10B0900009020843502108535020005B2979884356
:10B0A0005021085300E0761C5020005B4007400F01
:10B0B0002979884202D007488642F4D15020005BAB
:10B0C0004007400F2979884200D000273846F8BD54
:10B0D00000540440FFFF000030B5034600201C89E7
:10B0E0008C4209DD082A05D218244C431D682C190E
:10B0F000A05C02E0002000E0002030BD10B5024658
:10B1000013898B4205DD18234B431468E318987CA0
:10B1100000E0002010BD0146FF22C889C007C00F13
:10B1200000280AD00120C88100E0521EC889C0074B
:10B13000C00F002801D0002AF7D1C889C007C00F6E
:10B1400000280FD10220C8810420C881487A400815
:10B1500040004872487A3823984348720020487269
:10B16000012070470020FCE70246507A0123184373
:10B170005072507A0B78DB0018435072087A01281D
:10B1800008D1888850814868000C0123DB031843EC
:10B19000908108E0087A002805D150814868800035
:10B1A0001A4B18409081487A012804D1507A4023E4
:10B1B0001843507206E0487A002803D1507A4023A1
:10B1C000984350720878002811D1C87A1072087B11
:10B1D0001070487B5070887B9070CB7BD370087C5C
:10B1E00010714B7C5371887C9071CB7CD371887AC1
:10B1F000002803D00120C002D08101E00820D081C6
:10B20000FF200130D081012070470000FC1F0000AA
:10B21000002904D0427A80231A43427203E0427A22
:10B2200080239A434272704730B5024600200F4B8C
:10B230005024A45A0D022C435025AC525024A45A39
:10B240008C43AC5200E05B1E5024A45A6407640F88
:10B250008C4201D0002BF6D15024A45A6407640F0D
:10B26000002C01D0002000E0012030BDFFFF0000D5
:10B27000827A80231A40802A00D0817270470000B1
:10B2800070B5044600250023002D02D00126602061
:10B2900006530420C88188890126F603304000281F
:10B2A00008D0012010728889C004C0084E8930433C
:10B2B000506006E00020107288890F4E30408010E8
:10B2C0005060087AD072002304E0CE5C10460C3047
:10B2D000C6545B1CD07A9842F7DCC88904263040FB
:10B2E000002804D1C889F6023040002801D000208F
:10B2F00070BDD07AFCE70000FC1F0000002002496E
:10B300000880024908807047780000207A000020F9
:10B31000027C80231A40802A00D00174704710B547
:10B320000246FF23D089C007C00F002802D00120A9
:10B33000D0815B1ED089C007C00F002801D000203B
:10B3400010BD507A012420435072507A3824A04313
:10B350005072C87A1072487A00280FD1087B10709A
:10B36000487B5070887B9070CC7BD470087C1071C7
:10B370004C7C5471887C9071CC7CD471FF2001305E
:10B38000D0814000D081107ADAE70000F8B5044699
:10B390000D460020002C00D100BF002A00D100BFC4
:10B3A000012C01D141263043012A01D1122630431C
:10B3B000022C01D1C0263043022A01D1302630436D
:10B3C000134E307076788027BE43114F7E70012C6B
:10B3D00008D1FF2100BF0E4EB3781E460E40334603
:10B3E0008B42F8D10A4E76784027BE43084F7E70D4
:10B3F000012A0BD10026009603E000BF009E761CB8
:10B400000096FF276937009EBE42F6D9F8BD0000BE
:10B4100000040240002905D0054A12780243044B7B
:10B420001A7004E0024A12788243014B1A70704786
:10B4300020040240002905D0054A927E0243044BB5
:10B440009A7604E0024A927E8243014B9A767047D4
:10B450000008024070B5034614460020002B01D1BD
:10B46000C0B202E005468035E8B2012902D1051DCF
:10B47000E8B206E0022903D105460835E8B200E04B
:10B48000C0B2012C02D1851CE8B200E0C0B2084D68
:10B49000A870AD7801263543054EB570002201E055
:10B4A00000BF521C7D252D01AA42F9D970BD0000B4
:10B4B000000C024070B50024244800792021084087
:10B4C000002801D0224D3FE000F046F80546214813
:10B4D000007880210840002836D01E488078084037
:10B4E000002801D01A4D02E000F036F80546194850
:10B4F00080780007840F022C01DBAD0804E0012CEA
:10B5000001D16D0800E000BF124880788007C00FAD
:10B51000002801D02D0101E00C2045430D480078A2
:10B520004007840F002C02D1601CC4B207E0032C3A
:10B5300003D1601C4006040E01E06006040E2146A3
:10B540002846FCF703FE0546284670BD000402406D
:10B5500000127A00000C024000B5C0229178F82257
:10B5600011401C4A12781143EA2923D00ADC0A460A
:10B57000E03A130015F060FA0A181C20242A2A2A3F
:10B580002A161A2AED291FD004DCEB2916D0EC2943
:10B590001CD117E0F02903D0F82917D10E4817E085
:10B5A0000E4815E00E4813E00E4811E00E480FE07B
:10B5B0000E480DE00E480BE00E4809E00E4807E08B
:10B5C0000E4805E00E4803E00E4801E00D4800BFBC
:10B5D00000BF00BD201C02400090D003006CDC02C4
:10B5E0000048E80100366E010024F400001BB7009B
:10B5F00000127A00808D5B0000093D00C0C62D005E
:10B6000080841E0040420F0070B586B004460025BD
:10B61000002620680290A1796846C1736179417360
:10B6200000210173017100BF05E020460830415D33
:10B6300004A841556D1C6846C07BA842F5D80B2272
:10B64000D2010299881A914237D007DC2C48081A97
:10B650001FD023210901401A48D113E0FF386F3869
:10B66000002802D0012841D105E001A92548FFF7B3
:10B6700056FE06463BE001A922484030FFF74FFE48
:10B68000064634E001A91F485030FFF748FE064641
:10B690002DE001A91B482030FFF741FE06461A485D
:10B6A0000088072805DA18480088401C16490880D9
:10B6B00002E000201449088019E005F06BFD002825
:10B6C00013D0124801780078401C104A10700229EB
:10B6D00006DC01A90B486030FFF721FE064604E0B6
:10B6E00000200A4908700A49087000E000BF00BF46
:10B6F000002E02D1012006B070BD0020FBE7000043
:10B7000020020000805504407A00002076000020CE
:10B71000E400002010B5A8211348FCF7C7FD12482B
:10B72000124908601248486007200881002088728A
:10B7300007220F490D4800F0A9FA00210B48FFF736
:10B7400097FDA0210B48FCF7B1FD0A480A49486063
:10B750000A4B05220A49084800F015FC002106485A
:10B76000FFF7D6FD10BD0000800800206008002013
:10B7700038180200280900206C08002009B60000D3
:10B78000AC1702000C4A127812060B4B5B781B04B4
:10B790001A43094B9B781B021A43074BDB781A4369
:10B7A000104642084240D20083085A401146034ADC
:10B7B0005140034A11607047230700200102000036
:10B7C00028070020F8B504460F46A07A4006400E30
:10B7D000002874D10025ACE01820684321680818BF
:10B7E000407C01283CD101211820684322681018B0
:10B7F000017400260CE018206843216808180830FE
:10B80000815D18206843226810188155701CC6B2EB
:10B81000082EF0D300211820684322681018017404
:10B820001820684322681018417418206843226861
:10B8300010184161182068432268101881742C2068
:10B84000684361680818406A002809D018236B43D0
:10B850002268D0182C236B436268D218516A88473B
:10B8600018206843216808184069FF21C9438842AD
:10B870005DD818206843216808184069C11918204C
:10B88000684322681018416118206843216808182D
:10B8900041692C206843626810188069814246D350
:10B8A0001820684321680818807C55283FD055210E
:10B8B00018206843226810188174002624E03CE0B8
:10B8C0001820684321680818805D2C21694362684C
:10B8D00051181031895D08401821694322685118B8
:10B8E00088551820684321680818805D2C21694319
:10B8F000626851180831895D08431821694322683C
:10B9000051188855701CC6B2082ED9D32C20684314
:10B9100061680818806A002809D018236B432268E0
:10B92000D0182C236B436268D218916A8847681C30
:10B9300085B22089A84200DD4EE7F8BD012001490B
:10B94000087070478C00002010B50446002015F0E8
:10B95000D7FB02284DD1FFF7D1FC2D4800780028F5
:10B9600002D101202A49087029480078012823D1F2
:10B9700027484078401C2649487021465A20FCF749
:10B98000E5FB23494978884241D800202049487086
:10B9900008468078401C8870084680780A2803D3BF
:10B9A0000020887002200870FFF7A8FC00F068F8FB
:10B9B000002015F0D5FB2AE015480078022826D192
:10B9C00013484078401C1249487021467D20C00031
:10B9D000FCF7BCFB0E494978884218D800200C4976
:10B9E0004870FFF78BFC00F04BF8002015F0B8FB17
:10B9F0000DE00748C078401C0549C8700846C0786B
:10BA0000042804DB0020C87008704870887010BDDE
:10BA10007200002000B587B0002168460171042142
:10BA200041710C480290411003910B49049105911A
:10BA30000A480690FFF76EFE01A815F0F5FB00F02E
:10BA400059FB00F033F80021054809F001FF07B069
:10BA500000BD0000FFFF1F00FFFFFF1F15BD00001E
:10BA60000205000030B5034600201C898C4204D931
:10BA70004D015C686419626000E0022030BD000086
:10BA800010B5002400BF09E01C20604305494018A0
:10BA9000214682680448FFF7E5FF641C052CF3D3B8
:10BAA00010BD0000AC1702006C08002010B5FF208C
:10BAB000023072494860002008720120087000209E
:10BAC0004872012088726E48FFF725FB6B496C486D
:10BAD000FFF74AFB01216A48FFF79AFB694867496B
:10BAE0004860002008720120087000204872012080
:10BAF000887263481030FFF70EFB604960481030D1
:10BB0000FFF732FB01215E481030FFF781FB5D48F3
:10BB1000401E5A4948600020087201200870002029
:10BB200048720120887256485030FFF7F4FA5349A2
:10BB300053485030FFF718FB012151485030FFF7B0
:10BB400067FB5048C1384D49486000200872012009
:10BB50000870002048720120887249484030FFF781
:10BB6000DAFA464946484030FFF7FEFA01214448D8
:10BB70004030FFF74DFBFF20123040494860002065
:10BB800008720120087000204872012088723C4829
:10BB90006030FFF7C0FA394939486030FFF7E4FAFE
:10BBA000012137486030FFF733FBFF202130334954
:10BBB00048600020087201200870002048720120AF
:10BBC00088722F48A030FFF7A6FA2C492C48A030E5
:10BBD000FFF7CAFA01212A48A030FFF719FB2948CC
:10BBE0008F38264948600020087201200870002024
:10BBF0004872012088722248E030FFF78CFA1F4912
:10BC00001F48E030FFF7B0FA01211D48E030FFF790
:10BC1000FFFA1D4819494860002008720120087089
:10BC2000002048720120887215482030FFF773FA0F
:10BC3000124913482030FFF797FA012110482030AD
:10BC4000FFF7E6FA1048CB300C4948600020087234
:10BC500001200870002048720120887208483030A6
:10BC6000FFF759FA054906483030FFF77DFA012100
:10BC700003483030FFF7CCFA10BD00008C2A0020BA
:10BC8000105504400204000014070000F0B50B46F4
:10BC9000144643600481002136E0002216E02C2582
:10BCA0004D4346687519AD5C18274F430668F61971
:10BCB000B5542C254D4346687519AD5C18274F4384
:10BCC0000668F6190836B554551CEAB2082AE6D3B8
:10BCD000002518274F430668F619357418274F4377
:10BCE0000668F619757418274F430668F619B57477
:10BCF00018274F430668F619F57418274F4306684E
:10BD0000F61975614D1CA9B205898D42C5DC002567
:10BD10008572F0BD70B50446606800F0F1FD05461F
:10BD2000E27A23460C332946094800F0B1FD09495F
:10BD30006068884204D00749CB396068884206D1E0
:10BD4000E17AA28890B222460C3203F097F870BDD7
:10BD500060080020DF070000F8B5054600262C46E5
:10BD6000002C29D000BF03E00020A055701CC6B2F3
:10BD7000082EF9D304F0BCFFC00008210840074694
:10BD80002078884338432070E079E02188430B49CC
:10BD900009884901E02211400843E07104F0A8FF3E
:10BDA000012801D1082000E00020C706FF0EE0793D
:10BDB000400940013843E071F8BD00007A000020DE
:10BDC000F8B5054600260027002000902C46002CE0
:10BDD0005BD000BF03E00020A055701CC6B2082E47
:10BDE000F9D305F083F800280DD005F0C7F9022833
:10BDF00009D106212548FFF781F9552803D005F020
:10BE00006FF8002803D100202070607011E005F069
:10BE100083F892307D21C900884204D805F07CF86F
:10BE2000923087B201E07D27FF003804000E2070B9
:10BE3000677005F05FF900280DD005F0A5F902281C
:10BE400009D106211148FFF759F9552803D005F00B
:10BE50004BF9002803D10020A070E07015E005F038
:10BE60005FF992307D21C900884205D805F058F964
:10BE7000923080B2009002E07D20C00000900098D7
:10BE80000004000EA0700098E070F8BD600800206B
:10BE900070B5054600262C46002C24D000BF03E0D8
:10BEA0000020A055701CC6B2082EF9D305F072F917
:10BEB00001280AD131202070012060705920A07023
:10BEC0000820E070002020710DE005F063F90228E1
:10BED00009D131202070012060705920A070082005
:10BEE000E0700120207170BDFEB5054600260020DF
:10BEF000019001F01DFD074604F02AFF0A21009081
:10BF0000FCF73AF980B201902C46002C18D000BF03
:10BF100003E00020A055701CC6B2082EF9D33802E9
:10BF2000000E60713804000EA071E77105F00AF888
:10BF3000FF2802DDFF20A07002E005F003F8A070EA
:10BF4000FEBDFEB50546002600200190002704F046
:10BF5000F5FC64210090FCF70FF980B201900020FD
:10BF600001F008FD87B22C46002C0BD000BF03E087
:10BF70000020A055701CC6B2082EF9D33804000E5C
:10BF8000A070E770FEBDFFB581B004460F460025E6
:10BF90000026002000902760039820810498E0602C
:10BFA0000020207400BF9DE01C20684321680858D1
:10BFB0006A01616888501C206843216808188068FD
:10BFC0006A016168891848601C2068432168081864
:10BFD00040686A016168891888601C20684321688C
:10BFE0000818C0686A0161688918C8601C20684325
:10BFF00021680818007C6A016168891808741C208F
:10C00000684321680818407C6A016168891848748F
:10C010001C20684321680818807C6A0161688918BF
:10C0200088831C20684321680818C07C6A01616805
:10C030008918887400206A0161688918C8741C20F6
:10C040006843216808184068002813D01C20684302
:10C0500021680818C07C002805D1401E6A0161686B
:10C060008918C8831AE00020C0436A0161688918F2
:10C07000C88313E01C20684321680818C07C00288E
:10C0800005D000206A0161688918C88306E0002095
:10C090006A0161688918C88301200090002607E0C2
:10C0A00000216A016068801814308155701CC6B286
:10C0B000690160684018808BB042F1DC1C20684345
:10C0C00021680818406900280AD06B016268D218FC
:10C0D000104614301C236B432268D21851698847DC
:10C0E000681CC5B22089A84200DD5DE7009805B054
:10C0F000F0BD000000B58BB068480790002108A88B
:10C1000001706846017608A8417000206449887271
:10C11000082108A8C170002004E0002209A90A54DF
:10C12000411CC8B208A9C9788142F6DC5D48FEF717
:10C13000F2FF06A95B48FFF717F85848401C079024
:10C14000002108A801706846017608A84170002007
:10C1500053498872082108A8C170002004E0002219
:10C1600009A90A54411CC8B208A9C9788142F6DC61
:10C170004C484030FEF7CFFF06A94A484030FEF752
:10C18000F3FF452000010790002108A801706846D0
:10C19000017608A84170002041498872082108A84A
:10C1A000C170002004E0002209A90A54411CC8B251
:10C1B00008A9C9788142F6DC3A485030FEF7ABFF57
:10C1C00006A938485030FEF7CFFF112040010790F4
:10C1D000002108A801706846017608A84170002077
:10C1E0002F498872082108A8C170002004E00022AD
:10C1F00009A90A54411CC8B208A9C9788142F6DCD1
:10C2000028482030FEF787FF06A926482030FEF791
:10C21000ABFF0B20C0010790002108A80170684601
:10C22000017608A8417000201D498872082108A8DD
:10C23000C170002004E0002209A90A54411CC8B2C0
:10C2400008A9C9788142F6DC16486030FEF763FF22
:10C2500006A914486030FEF787FF1048A630029008
:10C260000021684601730171417381730821C17314
:10C27000002004E0002204A90A54411CC8B2694607
:10C28000C97B8142F6DC07481030FEF744FF01A964
:10C2900004481030FEF768FF0BB000BDEE0600004A
:10C2A0008C2A002080550440F0B585B004460F4626
:10C2B00000250026207C4006400E55287ED100BF78
:10C2C00076E1690160684018807C002877D16901B7
:10C2D0006068401840686A01616889188968884206
:10C2E00009D26901606840184068C0196A01616834
:10C2F000891848605AE1690160684018C068AF4910
:10C30000884208D8690160684018C068401C6A010A
:10C3100061688918C860690160684018C07C00289D
:10C3200021D1002607E000216A01606880181430DE
:10C330008155701CC6B2690160684018808BB0429C
:10C34000F1DC1C20684321680818406900280AD0E5
:10C350006B016268D218104614301C236B432268AC
:10C36000D218516988476901606840580090690196
:10C3700060684018017C68460171002141716901C3
:10C3800060684018017F68468171690160684018E3
:10C39000417C6846C171002608E069016068401868
:10C3A0001430815D02A88155701CC6B269016068B5
:10C3B0004018808BB042F0DCE06801E0FCE01DE05A
:10C3C000002806D06846E16888476A0161688918D4
:10C3D000C874690160684018C07C002804D16A01F3
:10C3E000616889184860E1E0690160684018406848
:10C3F000C01B6A01616889184860D7E069016068FC
:10C40000401880680028EED0690160684018C08B31
:10C410000028E8D0690160684018C08B6A01616833
:10C420008918C968884207D1690160684018C08BC3
:10C430006249C94388427DD16901606840184068FB
:10C440006A01616889188968884209D2690160684F
:10C4500040184068C0196A01616889184860A5E001
:10C4600000206A01616889184860690160684018A5
:10C47000C0685249884208D8690160684018C0689D
:10C48000401C6A0161688918C860002607E0002125
:10C490006A016068801814308155701CC6B2690149
:10C4A00060684018808BB042F1DC1C206843216832
:10C4B0000818406900280AD06B016268D21810463B
:10C4C00014301C236B432268D218516988476901D4
:10C4D000606840580090690160684018017C6846B7
:10C4E000017100214171690160684018017F68464F
:10C4F0008171690160684018417C6846C1710026FD
:10C5000008E06901606840181430815D02A8815517
:10C51000701CC6B2690160684018808BB042F0DCC4
:10C52000E068002808D06846E16888476A016168C9
:10C53000891800E015E0C874690160684018C07C83
:10C54000002804D16A016168891848602EE06901F9
:10C55000606840184068C01B6A01616889184860BB
:10C5600024E01C20684321680818406800280FD088
:10C570000020C0436A0161688918C8831C20684391
:10C580002168081840686A0161688918886008E0B5
:10C5900000206A0161688918C8836A016168891886
:10C5A000886000206A0161688918C860681CC5B28B
:10C5B0002089A84200DD84E605B0F0BD0000FFFF41
:10C5C0007CB500BF19212C480078FBF7BFFD04465D
:10C5D0002A4860432A4A8118002201200DF096F96A
:10C5E00020460A2250436430001981B20022012003
:10C5F0000FF0FEF901200A2262431219D1B20A2279
:10C60000624312190090D0B201231A4609F034FC9B
:10C61000FF220721002007F06FF801200090019011
:10C620000B20604382B20B20604381B200230120C3
:10C630000EF0FAFE6F20604381B201200FF07EFC05
:10C64000104860430246032101200BF0D9FE00256B
:10C6500005E0012128460BF00DFE681CC5B20F2D28
:10C66000F7DB21460B2251436431C8B20FF0D0FEF4
:10C670000FF0B8FE7CBD00006F000020672B0000AB
:10C68000A0860100FCB101000020054908700549A1
:10C690000870054908700549087005490870704719
:10C6A00070000020710000206F0000206E0000204C
:10C6B0006D000020F0B589B000BF00BF00BF00BF13
:10C6C00000BF00BF00BF00BF00BF00BF5D480078D3
:10C6D0003C2805DA5B480078401C5A49087002E0A3
:10C6E0003C2058490870574800781D2805DC5648FA
:10C6F0000078401C544908700BE05348007800282B
:10C7000002D15149087004E04F480078401E4E495C
:10C71000087003214C480078FBF72EFD4B49484335
:10C720000390052148480078FBF710FD04460321DB
:10C7300045480078FBF720FD0B214843643080B268
:10C740000690414909788A0088180621FBF714FDF4
:10C75000FF21F531484380B2079003213A48007821
:10C76000FBF70AFD0B214843643080B20890032197
:10C7700035480078FBF700FD3549484335494018F6
:10C780000490032130480078FBF7F6FC0B210646A5
:10C790004E4303212C480078FBF7EEFC0B210746A3
:10C7A0004F43032128480078FBF7E6FC6F214843FC
:10C7B00080B2059003210120039A0BF021FEE1B223
:10C7C00001200BF0E9FBE1B201231846069A09F0BB
:10C7D0002DFEFF21F5310798FBF7CEFCC0B20146D4
:10C7E000029001200AF004FB0022012008990FF0BA
:10C7F000FFF80022012004990DF088F80120059926
:10C800000FF09CFB0120F9B20090F0B201231A4610
:10C81000029009F031FBFF220721002006F06CFF97
:10C82000032109480078FBF7A7FC0B21484385B298
:10C830000120009000232A46294601900EF0F4FDC5
:10C8400009B0F0BD7100002070000020FCB10100B3
:10C85000672B0000A0860100002000BF06E0002139
:10C86000044A1154044A1154411CC8B25A28F6DB38
:10C87000704700005C260020102700200348007A43
:10C88000002801D10149487070470000600A00206B
:10C89000FFB581B004460F463D462089A8422DDDF4
:10C8A0001820684321680818007C002826D100263B
:10C8B00009E00498815D1820684322681018083048
:10C8C0008155701CC6B2082EF3D30121182068438D
:10C8D0002268101841742C20684361680818006AA7
:10C8E00000280BD018236B432268D218104608305A
:10C8F0002C236B436268D218116A884705B0F0BDDB
:10C9000001460720124BCA1A994211D008DCCA1FEF
:10C91000FA3A002A14D0102A0CD01F2A14D10DE0A4
:10C92000322A0FD0C02A07D0C12A0DD100200DE035
:10C9300001200BE0022009E0032007E0042005E0CD
:10C94000052003E0062001E0072000BF00BF70477C
:10C950004103000010B504467D21C900614308462B
:10C96000322103F08DFF10BDFF200B49087000201D
:10C97000C0430A4908800A490880FF200949087015
:10C9800009490870094908700020094908600949E7
:10C9900008600949086070475400002056000020D4
:10C9A000580000205A0000205B0000205C0000209E
:10C9B000480000204C000020500000200148006882
:10C9C000704700004C0000200148006870470000DC
:10C9D0004800002010B505490988652251430846E2
:10C9E0006421FBF7C9FB80B210BD00005600002097
:10C9F00001480078704700005B0000200148007883
:10CA0000704700005400002010B510F0A7FC01286A
:10CA10002CD100F063F8012000F066F803F094FFD9
:10CA2000044600F043F804F071F9044600F04AF8B7
:10CA300004F0D2FB012805D100F03EF8012000F0FF
:10CA400047F805E0002000F037F8002000F040F83B
:10CA500000201349086013480068134988421ED219
:10CA600010480068801C0F49086018E000200D493C
:10CA700008600B4800680C49884204D208480068E6
:10CA8000801C07490860002000F028F8012000F011
:10CA90002BF8002000F00AF8002000F013F810BD79
:10CAA0004C00002048000020FFFFFF7F0149088064
:10CAB00070470000560000200149087070470000D0
:10CAC0005B000020014908807047000058000020EA
:10CAD00001490870704700005C000020014908709F
:10CAE00070470000540000200149087070470000A2
:10CAF0005A0000200021014A117170470060004077
:10CB0000002201494A757047006000400022014937
:10CB10004A767047006000400021014A1172704758
:10CB2000006000400021014A11737047006000401E
:10CB30000021014A11747047006000400021014A41
:10CB400011757047006000400021014A117670475E
:10CB500000600040002201494A73704700600040B5
:10CB6000002201494A7470470060004010B51C4C17
:10CB70001C49206888421ED106221B49201DFBF754
:10CB8000A0FB002817D11222184920460A30FBF7D3
:10CB900098FB00280FD10622154920461C30FBF7D0
:10CBA00090FB002807D10622124920462230FBF7CD
:10CBB00088FB00280DD000F001FF0A480E490860EC
:10CBC000074814F0FEFB0C4A2C21054814F024FC05
:10CBD00004E02C2221460848FBF74FFB10BD000063
:10CBE000000250007AA7A55A390700203F0700200D
:10CBF000330700202D070020982E00200020084930
:10CC0000087008490870012007490870002007498A
:10CC100008700748074908600020074908707047F6
:10CC20001B0700201A0700201D07002022070020F4
:10CC300025060000540700202C07002070B504468C
:10CC400000BF9120604305460A212846FBF77EFA83
:10CC50000546284670BD000070B5A8B00546002402
:10CC60000026A0216846FBF721FB00F017FD1E49B6
:10CC70000A6814216943505000211B48026814209F
:10CC8000684310184160184802681420684310185F
:10CC9000816015484068002824D000BF17E0600676
:10CCA000060E282E00D316E00F48016814206043BA
:10CCB0000858B1006A4650500B4801681420604380
:10CCC00008184168701C80001150601CC4B20648EE
:10CCD000007AA042E3DC00BF620003486946436873
:10CCE0000220984728B070BD142F002030B5A9B09D
:10CCF00000240025A02101A8FBF7D8FA00BF25E0F9
:10CD00006006050E00F0CAFC1F490A681421614341
:10CD1000505000211C4802681420604310184160E4
:10CD2000194802681420604310188160282D0BD226
:10CD300015480168142060430858A90001AA505002
:10CD40000021681C80001150601CC4B20E48007A9B
:10CD5000A042D5DC0C484068002813D00A48007A6D
:10CD60004000282806D30848282201A94368022049
:10CD7000984707E00448007A4200034801A9436845
:10CD80000220984729B030BD142F0020FFB585B090
:10CD900006460E9F089C00200490039000250290F8
:10CDA0000190701C80002B49085A0490002E05D079
:10CDB000701E800040184088039003E0B0002549B1
:10CDC000085A03900398874204D30498874201D8F5
:10CDD0003D460AE00698012801D1049D05E0069829
:10CDE000002801D1039D00E03D461B48006805284E
:10CDF00005D219480068401C1749086027E0002048
:10CE00001549086005210798FBF7A0F902900298E0
:10CE100000281BD0AC420CD2281B0190029901982B
:10CE2000FBF794F9019001982418AC420FD92C46D5
:10CE30000DE0601B019002990198FBF787F90190C2
:10CE40000198241AAC4202D22C4600E02C4620461F
:10CE500009B0F0BD8A1B0200C000002008B510F028
:10CE60007DFA01287ED1FFF7AFFD7949884216D2BD
:10CE70000F2078498871C87108468078002801D150
:10CE80000520487073488078052802D10020714938
:10CE9000487000206F4948728872087035E0FA20A7
:10CEA0006C498871C8716C49088803F075FE6A483E
:10CEB000807800280CD16749087008468079C870CE
:10CEC0000846C079487100208870487088721CE05C
:10CED0000120604908700846807A022805D10120A7
:10CEE00088720020C87048710FE05A48807A002884
:10CEF0000BD102205749887208464078887008464E
:10CF00008079C8700846C079487152488078514984
:10CF10004978884229DD504800880A2148434D4914
:10CF20000090C9794B4B5B79CA1A4A4988784B49BA
:10CF30000B680021FFF72AFF484908600020454997
:10CF4000C870087108464079401C4871084640790D
:10CF5000C979884257DB00203E49487108468078ED
:10CF6000401E00E067E088704DE03A48807839491B
:10CF70004978884227DA384800880A2148433549E9
:10CF800000908979334BDB78CA1A32498878334963
:10CF90000B680121FFF7FAFE3049086000202D4997
:10CFA000487108710846C078401CC8700846C078AF
:10CFB0008979884227DB00202649C8700846807896
:10CFC000401C88701FE0002022494871C870084644
:10CFD0000079401C087108460079FA2801DBFA2024
:10CFE00008711D4800880A2148431A4900900979B0
:10CFF000FA235A1A1749887818490B680221FFF753
:10D00000C5FE1649086014488078002803D1012025
:10D01000104948721BE010480088732803DB022087
:10D020000C49487213E00C48008870280FDC00207F
:10D03000084948720BE000200649087008468079CC
:10D04000C8700846C079487100204872887208BDCF
:10D05000B80B000050260020BC000020C4000020B7
:10D060000020044988704870C870487148728872FE
:10D070007047000050260020002006490880887074
:10D08000054988704870FA20C870487100204872BD
:10D0900088727047BC00002050260020F8B500249C
:10D0A00000250026002703F07FFC044603F08EFCD9
:10D0B000054610F053F901282ED105211A48FEF734
:10D0C0001DF8552804D1002018498870088027E0F1
:10D0D000012D04D1002015498870088020E001202E
:10D0E000124988701248844202DB201A84B200E0A0
:10D0F00000240A212046FBF73FF8052901DB601DCB
:10D1000084B20C48844200DD04460A212046FBF725
:10D1100033F80649088003E000200449887008803D
:10D12000FFF79CFEF8BD000060080020BC00002056
:10D13000AA0A0000C60700001CB50020009001905C
:10D1400000F0ACFA0B49086000200B490968086040
:10D150000A48006800280CD00749096808680A21B5
:10D16000FAF7F4FF0090012269460520034B1B6883
:10D1700098471CBDF0070020E4070020EC070020C2
:10D180000020084948800849088008490880084963
:10D190000870084988720849088048800120087191
:10D1A000704700002C0000201C0000201E00002002
:10D1B000200000204408002024000020F8B503F0DF
:10D1C000D5FB074603F0E4FB0090FFF717FC0128AE
:10D1D00060D10521C548FDF791FF552802D0009880
:10D1E000012807D10020C2490870C2490880C249FD
:10D1F000887256E0BE480078002810D10120BC4952
:10D2000008703D462846E917890F091889030D0C57
:10D21000BA48854200DD0546B648058041E0B6487B
:10D22000807A4000B4490F520846867A0EE07000BA
:10D23000B1490D5A701E4000085A7100AE4A505252
:10D24000701E400011460D52701EC6B2002E08DD41
:10D250007000A949095A701E4000A74A105A81421D
:10D26000E5DBA548807A401CA34988720846807A8D
:10D27000052816DB002088720846C5882846E9176D
:10D28000890F09188D109D48854200DD0546994893
:10D29000058006E000209649087096490880964966
:10D2A00088729448058896480088A84257DA9448BE
:10D2B0000088281A84B292480079012827D1904822
:10D2C0004088A0420BDA8E4840880A308C4948805A
:10D2D00008464088A04204DD0846448001E08848B2
:10D2E00044808748448803212046FAF745FF84B2EA
:10D2F000192C00DA19248248008800198049088016
:10D3000008460088A84201DD08460580CDE07C483B
:10D310004088142805DD7A484088143878494880C8
:10D3200002E0002076494880754844880321204661
:10D33000FAF722FF84B2192C03DA01207049087130
:10D34000B3E06F480088A04205DD6D480088001BEF
:10D350006B490880A9E0002069490880A5E0684879
:10D360000088A84259DD66480088401B84B26448A2
:10D370000079012827D162484088142805DD6048DB
:10D38000408814385E49488002E000205C494880AB
:10D390005B48448803212046FAF7EEFE84B2192C3C
:10D3A00003DA0220564908717FE0554800880019C9
:10D3B00053490880084600885049884275DD084670
:10D3C0004F49088071E04E484088A0420BDA4C4833
:10D3D00040880A304A49488008464088A04204DD17
:10D3E0000846448001E0464844804548448803217B
:10D3F0002046FAF7C1FE84B2192C00DA19244048FD
:10D4000000882919884202DA3D4805804DE03C48F1
:10D410000088001B3A49088047E0394844880321C6
:10D420002046FAF7A9FE84B2192C3EDD3448408824
:10D43000142805DD3248408814383149488002E01C
:10D4400000202F4948802E48448803212046FAF7BF
:10D4500093FE84B22A480079012813D1192C03DAEB
:10D4600002202749087120E0254800880019244936
:10D470000880084600882149884216DD0846204970
:10D48000088012E0192C03DA01201D4908710CE014
:10D490001B480088A04205DD19480088001B184978
:10D4A000088002E0002016490880164800885028AD
:10D4B00004DC134800881349088016E010480088EF
:10D4C00010490988884204DD0D4800880D4908800C
:10D4D0000BE00B4800880B490988081A84B2502CCD
:10D4E00003DB0748008807490880F8BD6008002072
:10D4F000200000201C00002044080020E02E000036
:10D50000240000201E00002010B50446642044437F
:10D51000A1212046FAF71AFE0446204610BD00005D
:10D5200010B501200F49087000200F4909680860F4
:10D530000D49096848600C490968886000F07EF967
:10D54000FFF7FAFDFFF7D2FB08480068002807D074
:10D5500001220548016808310020044B1B689847E8
:10D5600010BD0000BD070020B8070020B407002050
:10D5700010B5184800681849884229D11748006832
:10D58000002804D0154800688047154908701548E0
:10D590000068002804D013480068804712490870CA
:10D5A00012480068002804D01048006880471049DD
:10D5B000088010480068002805D00E4800688047A1
:10D5C0000D49088002E00D480B49088000F078F80A
:10D5D00010BD0000C807002078563412A4070020B0
:10D5E000BC070020A8070020BE070020AC070020D1
:10D5F000C0070020B0070020C2070020102700004D
:10D6000010B50023174C2360174C2370174C237060
:10D61000174C2370174C2380174C2380174C237012
:10D62000174C13682360174C53682360164C93689B
:10D630002360164CD3682360154C136923600028BF
:10D640000CD0144B1860134C0B682468A3600023A3
:10D65000104C246823600F4C246863600E4B014C0F
:10D66000236010BDC8070020C4070020BC070020AD
:10D67000BE070020C0070020C2070020BD07002011
:10D68000A4070020A8070020AC070020B007002056
:10D69000B4070020B8070020785634120548006807
:10D6A0000549884203D1054800688068704700201A
:10D6B000C043FBE7C807002078563412B8070020A3
:10D6C00070B50024002500263048007801285CD180
:10D6D0002F480078002858D12E480078012854D1CE
:10D6E0002D4805882D490988694308462C49FAF7D1
:10D6F0002DFD85B2E1200001854207D8192169433B
:10D7000008460921FAF722FD044600E0244C25488A
:10D71000006800680019234909680860214800680A
:10D720000068204909684968884207D31D48006895
:10D7300000681C4909684968461A0AE019480068E7
:10D7400040680021C943081A164909680968401849
:10D75000461C1548864218D3344601462046FAF73F
:10D76000F5FC04460F48006841680F4860430818FC
:10D770000C490968486001200C4908700948006894
:10D780008068001907490968886070BDBC070020DF
:10D79000BD070020BE070020C0070020C2070020F0
:10D7A00010270000B8070020A0860100C407002051
:10D7B00000220C4B1A600C4B0A681A600B4B4A682B
:10D7C0001A600B4B8A681A600A4BCA681A600A4BC7
:10D7D0000A691A60002801D0084A1060084A014B03
:10D7E0001A607047C8070020A4070020A80700207F
:10D7F000AC070020B0070020B4070020B8070020C5
:10D800007856341210B50A48006800280ED009482E
:10D81000007801280AD10020064908700122064834
:10D82000016808310020024B1B68984710BD0000BA
:10D83000B4070020C4070020B80700201CB5002052
:10D84000009001900024FFF729FF04460E4800686D
:10D85000046000200C49096848600B490968886029
:10D860000A48006800280DD007480068006800904A
:10D870000548006840680190022269460120034B78
:10D880001B6898471CBD0000CC070020D007002073
:10D89000F8B505460C4616460027002D17D00E4851
:10D8A0000560FFF7FBFE07462068B84203D90A4827
:10D8B0000068076003E008492068096808600649B5
:10D8C0006068096848600449A0680968C86003483E
:10D8D000066000F005F8F8BDCC070020D007002056
:10D8E00070B500240025FFF7D9FE04460F480068F4
:10D8F0000068A04200D903E00C4800680068251ABF
:10D900000A48006840684019084909688860074863
:10D910000068806805490968C968884205D90348D4
:10D920000068C06801490968886070BDCC070020A4
:10D930000148006880687047CC070020002801D0AB
:10D94000024A1060024A116070470000CC070020B4
:10D95000D00700200549002005E00A1D135C044A99
:10D960001354421CD0B22028F7DB70470006500049
:10D97000C82E0020014610480268142048431018A1
:10D9800082680D480368142048431818C068824212
:10D990000BD909480268142048431018C268064889
:10D9A0000368142048431818826003480268142052
:10D9B0004843101880687047142F002010B50021CC
:10D9C0000022002005E01B4B1C5C1B4B1C54431C1D
:10D9D000D8B20628F7DB1221002006E0174B1C5CAA
:10D9E000154B9B1D1C54431CD8B28842F6DB00200B
:10D9F00006E0134B1C5C104B18331C54431CD8B26C
:10DA00000628F6DB002006E00E4B1C5C0A4B1E339A
:10DA10001C54431CD8B20628F6DB0422002005E083
:10DA20000024054B24331C54431CD8B29042F7DB2E
:10DA300010BD0000390700209C2E00203F07002069
:10DA4000330700202D07002038B504460020009041
:10DA5000009401226946052000F06AFC38BD0000F0
:10DA600008B50020009001226946062000F020FC45
:10DA7000684600780F49087368464078487308463E
:10DA8000007B0D4948730B48407B88730948807BB5
:10DA9000C8730848C07B08740020087307490860F1
:10DAA0000749086007490860074908600749087086
:10DAB00008BD00004C280020C80900207C00002080
:10DAC0008000002084000020880000208C000020BE
:10DAD00008B50020009001226946062000F0E8FB0E
:10DAE00068460078124908736846407848730020F9
:10DAF0001049086048600872487288720C48007BC0
:10DB000048730B48407B88730948807BC87308487A
:10DB1000C07B087400200873074908600749086043
:10DB200007490860074908600749087008BD0000F8
:10DB30004C280020C80900207C0000208000002024
:10DB400084000020880000208C00002038B50024CC
:10DB50000025002000900121FA48FDF7CFFA552852
:10DB60000AD002F077FFF849487302F087FFF649C0
:10DB700088730120087308E0F448007BF249487379
:10DB8000F248407B8873002008730621ED48FDF7BA
:10DB9000B5FA552830D002F0A5FF002808D002F0D1
:10DBA000A1FF401C002803D00120E749087502E0CE
:10DBB0000020E549087502F077FF002808D002F040
:10DBC00073FF401C002803D00120DF49C87402E025
:10DBD0000020DD49C87402F085FF002808D002F05B
:10DBE00081FF401C002803D00120D749087507E0B9
:10DBF0000020D549087503E00020D349C874087592
:10DC0000D148407B00282BD1D1490860D148006819
:10DC1000D149884208D8CF480068401CCD490860E7
:10DC20000020C94948736CE0C848007B022812D024
:10DC3000C648007B03280ED00121C248FDF75EFADA
:10DC4000552803D00320C04948735AE0BF48007BE1
:10DC5000BD49487355E0BD48007BBB49487350E05F
:10DC6000B948407B01282CD10020BA490860B84847
:10DC70000068B949884208D8B5480068401CB449D2
:10DC800008600120B04948733BE0B048007B02289F
:10DC900012D0AE48007B03280ED00121A948FDF721
:10DCA0002DFA552803D00320A749487329E0A74837
:10DCB000007BA549487324E0A448007BA24948732F
:10DCC0001FE0A148407B022805D10020A14908603F
:10DCD0009F49086015E09C48407B032808D100203C
:10DCE0009C4908609A49086003209749487308E0F6
:10DCF000002098490860964908609448007B924942
:10DD000048739148807B00282BD19449086094483F
:10DD100000689149884208D891480068401C9049A1
:10DD200008600020884988736CE08848407B02289E
:10DD300012D08648407B03280ED001218148FDF790
:10DD4000DDF9552803D003207F4988735AE07F48C6
:10DD5000407B7D49887355E07C48407B7A498873D5
:10DD600050E07948807B01282CD100207C49086054
:10DD70007A4800687849884208D878480068401C8A
:10DD8000764908600120704988733BE06F48407B0A
:10DD9000022812D06D48407B03280ED0012169482B
:10DDA000FDF7ACF9552803D003206749887329E0B3
:10DDB0006648407B6449887324E06448407B62493C
:10DDC00088731FE06048807B022805D100206449E9
:10DDD00008606249086015E05B48807B032808D131
:10DDE00000205F4908605D49086003205649887338
:10DDF00008E000205A490860584908605348007BF1
:10DE0000514988735048407B5049097B884205D16D
:10DE10004D48807B4D49497B88424FD04A48407BE2
:10DE20004A49097B884202D001204749C8734648C5
:10DE3000807B4649497B884202D0012042490874D0
:10DE40004148407B022803D03F48407B032816D13D
:10DE50003D48407B3D49097B884210D03A48407B91
:10DE60003A4908730846017B684601703748417B90
:10DE70006846417001226946062000F059FA32488E
:10DE8000807B022803D03048807B032816D12E489F
:10DE9000807B2E49497B884210D02B48807B2B49C0
:10DEA00048730846017B684601702848417B6846F4
:10DEB000417001226946062000F03AFA02F0D4FDD2
:10DEC000044602F0E7FD0546FEF798FD01287BD1E8
:10DED00001211C48FDF712F9552807D100201A49E5
:10DEE00008724872086048608872BAE0FF2C01D05E
:10DEF000FF2D78D1FF2C3FD1FF2D3DD000201249BE
:10DF00000872012048721748086017486843486043
:10DF100048686621FAF71AF90B49486008464068D4
:10DF20001249884202D908460749486003F0E8F8D8
:10DF3000112803DB03F0E4F8192819DD0120024958
:10DF400088728EE060080020C80900204C2800205C
:10DF5000800000207C000020701700008800002056
:10DF600084000020DE030000BE0A0000AC26000092
:10DF700000205D49887274E0FF2C2BD0FF2D29D141
:10DF80000120594908720020487258484860584892
:10DF90006043086008686621FAF7D8F852490860BB
:10DFA000084600685349884202D908464E4908602D
:10DFB00002F0A2FF112803DB02F09EFF192805DD05
:10DFC0000120494988724CE086E00CE00020464977
:10DFD000887246E0474844490860486000208872DB
:10DFE000087248723DE001203F490872487240487B
:10DFF0006043086008686621FAF7A8F83A490860A3
:10E00000084600683B49884202D9084636490860FC
:10E01000374868433449486048686621FAF796F8FB
:10E0200031494860084640683249884202D908466A
:10E030002D49486002F060FF11280BDB02F05CFF05
:10E04000192807DC03F05CF8112803DB03F058F80B
:10E05000192803DD01202449887202E000202249AA
:10E0600088722148407B002802D11F49C87315E0FF
:10E070001D48407B012802D11B49C8730EE01A4895
:10E08000407B022802D11849C87307E01648407B3C
:10E09000032803D11449C873164808601248807BCE
:10E0A000002802D1104908741DE00F48807B012828
:10E0B00002D10D49087416E00B48807B022802D17A
:10E0C000094908740FE00848807B03280BD10649F2
:10E0D00008740848486006E0002003490872487246
:10E0E00008604860887238BDC8090020DE0300005F
:10E0F000BE0A0000AC260000FFB583B006460D4600
:10E10000174600240020029000BF14207843801995
:10E110000190002E57D00198002854D02B4806605B
:10E120002A49069848600846077200BF45E0FFF795
:10E13000B5FA0290200129580298814204D82001A2
:10E140002858401C002806D1204902980A6814214A
:10E150006143505006E0200129581C4802681420F1
:10E1600060431150200140194068401C002807D12D
:10E17000002116480268142060431018416008E02E
:10E1800020014019416811480268142060431018AA
:10E1900041602001401981680C48026814206043E6
:10E1A0001018C16020014019017B08480268142042
:10E1B000604310180161601CC4B20448007AA04298
:10E1C000B5DC00F005F807B0F0BD0000142F00200A
:10E1D00070B5002400250026FFF760FA054600BF51
:10E1E0004EE02A480168142060430858A84239D8F4
:10E1F000264801681420604308582E1A23480168F5
:10E2000014206043081840688119204802681420CF
:10E210006043101881601D4801681420604308188D
:10E2200081681A480268142060431018C06881424F
:10E2300024D9164801681420604308180069002892
:10E2400003D02046FEF708FD18E0104801681420AE
:10E2500060430818C1680D48026814206043101814
:10E2600081600BE009480168142060430818406889
:10E2700006490A681421614351188860601CC4B2C1
:10E280000248007AA042ACDC70BD0000142F0020D0
:10E2900010B500BF14244C432318002805D0002BD0
:10E2A00003D0024C20606260217210BD142F002048
:10E2B000F8B505460E4614462B0012F0BDFB0705C7
:10E2C000131A3131212931001748FAF74DFC17494B
:10E2D00008701548FAF702F807466421F9F736FF87
:10E2E00030601EE0A004020C31462020FAF736FD13
:10E2F00017E0A004020C31466020FAF72FFD10E071
:10E30000A004020C3146FF202130FAF727FD08E077
:10E310006004020C3146FF204130FAF71FFD00E097
:10E3200000BF00BF0020F8BD3E280020D100002023
:10E3300070B505460E4614462B0012F07DFB07050E
:10E340001D243A3A2B323A003068002802D1FAF7FD
:10E35000A9FA10E064223168514308461649F9F7DA
:10E36000C7FF002015490870012264211248FAF7FE
:10E3700063FD124908701DE0A004020C3146202004
:10E38000FAF7AAFE16E0A004020C31466020FAF764
:10E39000A3FE0FE0A2B23146FF202130FAF79CFE27
:10E3A00008E06004020C3146FF204130FAF794FE89
:10E3B00000E000BF00BF70BD30280020D00000206A
:10E3C00000B5AFB050211BA8F9F770FF00201A90DC
:10E3D000142115A8F9F76AFF0020129013901490E9
:10E3E0001190402101A8F9F761FF002000904849F1
:10E3F000086001221BA9FFF75BFF1B98401C002847
:10E4000001D11A9001E01B981A9042481590424899
:10E41000169042481790002018904148199015AA6C
:10E420001AA94048FFF7ECF802221CA90120FFF7C7
:10E430003FFF1C98401C002801D1129001E01C985D
:10E4400012901C98401C002801D1139001E01D98E7
:10E4500013903548149012A93448199AFFF718FA06
:10E4600008221EA90220FFF723FF1E98401C002847
:10E4700001D1019001E01E9801901F9802902C4854
:10E480000390012069460874801E05902949079170
:10E49000012101A80177881E099026490B910121CD
:10E4A00009A80173881E0D9022490F9101210DA822
:10E4B0000173042201A92048199BFFF71DFE0122C8
:10E4C0001BA90520FFF7F4FE1B98401C002807D16C
:10E4D00001201A498860012208310520FFF728FF32
:10E4E00001221BA90620FFF7E3FE1B98401C002811
:10E4F00008D100216846017041700122694606205A
:10E50000FFF716FF0E48024908602FB000BD00005B
:10E51000D4000020FDC90000F1C90000D5C90000E9
:10E5200031E30000C427002076841E00D02700209D
:10E530000F2700009F860100E02700204C280020C4
:10E54000A33AA55A00B585B014216846F9F7AEFE86
:10E5500000200F4908600F4800900F4801900F48B5
:10E560000290002003900E48049069460D48FFF782
:10E570001FF90D480499FFF7E1F904210B48049AAB
:10E58000FFF786FE0A480249086005B000BD00009A
:10E59000D4000020FDC90000F1C90000D5C9000069
:10E5A00031E30000C4270020D0270020E02700200E
:10E5B000A33AA55A00200C4908800C4908800C4950
:10E5C000088001200B49087000200B4908730B4993
:10E5D0000880488001200871002007494880088091
:10E5E0000749086070470000340000203600002012
:10E5F0003C0000203E000020500800204000002089
:10E6000038000020F8B502F0EBF9064602F0F2F906
:10E610000746FEF7F3F9012865D10521AB48FCF761
:10E620006DFD552807D10020A9490870A949088027
:10E63000A94988805FE0012F07D10020A449087014
:10E64000A4490880A449888055E0A14800780028A2
:10E6500008D101209E49087035460A2068439D492B
:10E66000088048E09C48007B42009B48801D865201
:10E67000801F047B11E061009748801D455A601E91
:10E6800041009548801D415A62008152601E410040
:10E690009148801D4552601EC4B2002C0ADD610005
:10E6A0008D48801D415A601E42008B48801D805A53
:10E6B0008142E0DB8848007B401C8749087308469C
:10E6C000007B032807DB00200873084605890A2021
:10E6D0006843804908807F4800887F4988800120FE
:10E6E0007B49087007E00020794908707949088063
:10E6F00079490873888077480088784908607448A9
:10E700000078002815D0084600686C2148437349FA
:10E710000860642171480068F9F718FD6F490860C6
:10E72000084600686E49884206D908466B49086069
:10E7300002E0002069490860684800686949098862
:10E74000884203D2654800680F2804D263480088D5
:10E75000644908800AE06348008860490968401AF3
:10E760000F2803D35D4800885E4908805A48008816
:10E77000401C59490880084600880A282CDB0020E4
:10E7800008805948008857490988884203DA0120DF
:10E790005649087108E0544800885249098888425F
:10E7A00002DD02205149087150480079012840D10A
:10E7B0004C4800884C49098888420DDB494801884B
:10E7C00049480088FF309130814206DD4648008884
:10E7D000FF3073304449088077E04248018842485E
:10E7E00000889630814205DD3F48008878303E49F8
:10E7F00008806AE03B4801883B480088323081420B
:10E8000005DD394800881E30374908805DE035480D
:10E810000188354800880A30814205DD3248008889
:10E820000A303149088050E02E4800882E4908807F
:10E830004BE02E480079022847D12A4800882A490F
:10E840000988884239DA27480088FF309130264904
:10E850000988884206DA24480088FF38733822493C
:10E8600008802AE01F48008896301F49098888429E
:10E8700005DA1D48008878381B4908801DE01948D2
:10E880000088323018490988884205DA164800881D
:10E890001E381549088010E0124800880A301249D5
:10E8A0000988884205DA104800880A380E4908802D
:10E8B00003E00C4800880C4908800B480088084990
:10E8C000884202DB084608490880F8BD600800203D
:10E8D0003E000020340000205008002038000020B6
:10E8E000C60700003C000020360000204000002049
:10E8F00000200849088008490880084908804880A5
:10E9000001200871002006494880088005490860F8
:10E9100070470000360000203C000020400000202E
:10E9200050080020380000200020044908700449E5
:10E930000870002103480176704700008D00002018
:10E940008E000020400A002070B500250024FEF74C
:10E9500055F8012863D103213448FCF7CFFB552833
:10E9600008D100203249087032490870002132482D
:10E97000017659E02F480078002807D102F0D0F83E
:10E980002B49087001202B4908704DE001202949CE
:10E99000087002F0C5F82849097E8900264A603AC5
:10E9A00050502548047E10E0A000234960390D5CDA
:10E9B000601E80000858A1001F4A603A5050601E37
:10E9C000800011460D50601EC4B2002C0ADDA0006C
:10E9D000194960390958601E8000174A603A10587A
:10E9E0008142E1D31448007E401CC1B21248017636
:10E9F000007E1E2818DB00210F4801760146603991
:10EA0000896B0246603AD26B89180246603A126CF2
:10EA100088180321F9F79AFB0549087004E00020E3
:10EA2000034908700349087070BD000060080020A9
:10EA30008D0000208E000020400A0020F0B5A9B013
:10EA400004460E460025002700202890A021684695
:10EA5000F9F72CFCFEF722FE26490A6814216143CF
:10EA6000505024480168142060430818C068B04220
:10EA70000CD220480168142060430818C1681D4862
:10EA80000268142060431018416005E019480168CD
:10EA9000142060430818466016484068002826D0B5
:10EAA000002517E06806070E282F00D316E011484E
:10EAB0000168142068430858B9006A4650500D4850
:10EAC00001681420684308184168781C80001150C0
:10EAD000681CC5B20748007AA842E3DC00BF6A00A0
:10EAE00004486946436802209847012028902898E6
:10EAF00029B0F0BD142F002010B500F0F9FD00F092
:10EB0000D7F810F0B9FE00F00DFB00F001F810BDD1
:10EB100070B541480078912800D070BD00F0BEF873
:10EB2000012876D13D4800883D4908800846807814
:10EB3000F021884320303A498870084680780009DF
:10EB400000013549097A0907090F084334498870DB
:10EB50003148807A401E3049887208460089401C3E
:10EB6000088108460089C988884216DA08202C499D
:10EB7000887200240EE0284841882848001D415C26
:10EB80002748C01C015524484088401C2249488021
:10EB9000601CC4B2072CEEDB2DE01F4800891E4923
:10EBA000C98888421CD11C4800791B498978401AC1
:10EBB000C5B2681C1A49887200240EE016484188C4
:10EBC0001648001D415C1648C01C0155124840887B
:10EBD000401C11494880601CC4B2AC42EEDB0AE024
:10EBE00000F012FD00200C4908700C49088809212A
:10EBF00000F0B8F991E7012000F0C8FC084A917ACA
:10EC00001088921C00F070F905490888002100F076
:10EC1000C1F800BF81E700004C2C0020E82B002049
:10EC2000782B00201B49097E002932D01949897EA2
:10EC30000C225143174A515A174A118000200CE008
:10EC40001449897E0C225143124A8918891C0A5C96
:10EC50001149891C0A54411CC8B20828F0DB0D492F
:10EC6000897E0C2251430B4A8918897A0A4A91728B
:10EC70000121D1720749097E491E064A11761146C3
:10EC8000897E491C91761146897E022901DB00218B
:10EC900091767047442B00206C2B00200349487B61
:10ECA000012802D10021014A517370475C2C0020D9
:10ECB00010B533484068002861D13148007B03001B
:10ECC00011F0BAFE07590512212E3D4A59002D4870
:10ECD0000078002807D000202A4908702A490888AF
:10ECE000012100F03FF947E026480078002809D0CC
:10ECF00000202449087025494A8808880123091DF5
:10ED000000F040F938E01F480078002807D00020C4
:10ED10001C4908701C490888022100F023F92BE0E7
:10ED200018480078002809D00020164908701749B3
:10ED30004A8808880923091D00F024F91CE01148BD
:10ED40000078002807D000200E4908700E49088876
:10ED5000092100F007F90FE00A480078002809D0DF
:10ED600000200849087009494A8808880323091DBA
:10ED700000F008F900E000BF00BF00F045FC10BD46
:10ED80005C2C00204C2C0020E82B0020842B002041
:10ED90007047000070B504460D4634480088A04214
:10EDA00063D1002D61D13248007822284ED004DC96
:10EDB00020283DD0212856D141E0902802D091282A
:10EDC00051D115E02A48C08801280AD100202849DD
:10EDD000087000F019FC27490888002100F0C2F8EB
:10EDE00005E0032000F0D2FBA020214908703BE0A1
:10EDF0001F4800891E49C98888420AD100201C4941
:10EE0000087000F001FC1B490888002100F0AAF8F6
:10EE10000DE01748807A002806D000F0F5FB144971
:10EE2000087B00F095FB02E0032000F0AFFB1BE045
:10EE3000062000F0ABFB11200D49087014E00620FD
:10EE400000F0A4FB11200A4908700DE000200849D9
:10EE5000087000F0D9FB08494A8808880923091D71
:10EE600000F090F800E000BF00BF70BD602B0020F4
:10EE70004C2C0020E82B0020842B002070B503468A
:10EE8000184C247E022C00DB70BD164C647E0C25D1
:10EE90006C43144D2B5300200AE0155C114C647E2A
:10EEA0000C2674430F4EA419A41C2554441CE0B234
:10EEB0008842F2D30B4C647E0C267443094EA4198D
:10EEC000A1723446247E641C35462C762C46647E22
:10EED000641C6C762C46647E022C01DB00246C766C
:10EEE00000BFD1E7442B0020F0B585B007460D46A2
:10EEF00016461A480780002406E031781748801C1F
:10EF00000155761C601CC4B2AC42F6DB2C4605E011
:10EF1000AA211248801C0155601CC4B2082CF7DBE2
:10EF20000E480088019008216846C1720021417294
:10EF300001720170002406E00848801C015D03A8EE
:10EF40000155601CC4B2082CF6DB69460448FCF786
:10EF5000E6F901200149887205B0F0BD602B002060
:10EF60009055044070B504460D462946204610F0E1
:10EF7000A5FB70BD70B504460D462946204610F02D
:10EF8000ABFB70BDF8B504460D4616461F463B4622
:10EF900032462946204610F0A0FBF8BDF8B50746DA
:10EFA0000E4615465C480078002804D009213846F2
:10EFB000FFF7D8FFF8BD002D01D0602D04DD092139
:10EFC0003846FFF7CFFFF5E7544807804580002417
:10EFD00006E031785148001D0155761C601CC4B212
:10EFE000AC42F6DB00204C49487008468580FF2083
:10EFF00088727F2008730846808808282EDA01204E
:10F00000C8800846808848800120088143480088DD
:10F010004349088008468078F02188434049887039
:10F0200008468078000900013B4909790907090F62
:10F0300008433B49887038480079401C8872002496
:10F0400007E03648001D015D3548C01C0155601CB5
:10F05000C4B231488088A042F3DC4AE00721681C32
:10F06000F9F78AF8002907D0072128460830F9F770
:10F0700083F82949C88005E00721681CF9F77CF866
:10F080002549C8800620244948800120088123485A
:10F0900000882349088008468078F0218843103092
:10F0A0001F49887008468078000900011A4989883C
:10F0B0000905090F08431A49887008464088FF214E
:10F0C00009028843144989880902FF22120211406B
:10F0D00008431349488008208872002407E00F483D
:10F0E000001D015D0E48001D0155601CC4B2062CB8
:10F0F000F5DB012000F04AFA094A917A1088921C47
:10F10000FFF7F2FE902004490870054908880021A5
:10F11000FFF740FE00BF4DE74C2C0020E82B0020FD
:10F12000782B002010B5FFF77DFD1448C07A002829
:10F1300022D0124880780009002806D0012807D084
:10F1400002280AD0032810D10CE000F0A7F90FE044
:10F1500000F09EF800F066FA0AE000F011F800F006
:10F1600061FA05E000F000F902E0FFF711FE00BFD0
:10F1700000BF00200149C87210BD00006C2B0020A8
:10F1800010B53F480078112800D010BD3D480088D8
:10F190003D49884200D0F8E73A4880780007000FE0
:10F1A0003749097A0907090F88420CD000203449F1
:10F1B000087000F029FA35494A8808880423091D97
:10F1C000FFF7E0FEE1E72E480089401C2C4908814A
:10F1D0000846807A401E887208460089C98888429D
:10F1E0001BDA2848807A082800D0CEE700240EE0F9
:10F1F0002448C01C015D224842882448001D8154D7
:10F200001F484088401C1E494880601CC4B2072C1F
:10F21000EEDB062000F0BAF930E019488088184982
:10F220004988401A1749897A884203DA1548807A52
:10F23000082800D0A9E700240EE01248C01C015D98
:10F240000F4842881148001D8154601CC4B20C480C
:10F250004088401C0A4948800948408808498988F4
:10F260008842EADB00200649087000F0CDF9074922
:10F270004A8808880023091DFFF784FE00BF84E741
:10F280004C2C00206C2B002014070000842B002045
:10F2900070B53148007880210840802800D170BDC9
:10F2A0002E4800882E49884200D0F8E72B48807A03
:10F2B000082800D0F3E72948807805072D0F2D0294
:10F2C00026484088000A0543082D00DAE7E70020B9
:10F2D0002149487006204880084685800120088121
:10F2E000082088720020C8728988481C0721F8F716
:10F2F00043FF002909D018498988084608300721AA
:10F30000F8F73AFF1449C88007E013498988481C78
:10F310000721F8F731FF1049C880104800881149CB
:10F32000088008464580002407E00C48001D015D68
:10F330000C48001D0155601CC4B2062CF5DB0420EE
:10F3400000F024F9102004490870064A51881088FA
:10F35000FFF710FE00BFA2E74C2C00206C2B002012
:10F3600014070000842B002010B548480078A0281E
:10F3700008D046480078912804D044480078A12855
:10F3800000D010BD42480088424988420AD0424914
:10F3900008880921FFF7E6FD00F036F900203B4917
:10F3A0000870EEE73A48807A08280AD03A49088877
:10F3B0000921FFF7D7FD00F027F900203349087035
:10F3C000DFE7334880780007000F002804D00128C9
:10F3D0002DD002284BD136E02C484078002800D0B0
:10F3E00050E02B48C078002803D1012027494870FD
:10F3F00003E02748C078254988722448007891287E
:10F400000BD023480079002803D101201F4908733D
:10F4100003E01F4800791D49087391201B490870BB
:10F4200000F0F2F81949087B00F092F82AE017483A
:10F430004078002800D025E0A1201449087003205E
:10F4400000F0A4F81EE011484078002800D019E030
:10F450000E480078A02809D10F4908880821FFF735
:10F4600081FD00F0D1F80020084908700AE00A493F
:10F4700008880521FFF776FD00F0C6F80020034953
:10F48000087000BF00BF00BF7BE700004C2C0020CD
:10F490006C2B002014070000E82B002010B5284832
:10F4A000007880210840802800D110BD24480078D1
:10F4B000002805D0234800882349884200D0F4E77B
:10F4C0002048807A1F4989780907090F884203DD9F
:10F4D0001C48807A082800D0E7E71A48807800079F
:10F4E000000F002805D0174880780007000F072874
:10F4F00000DDDAE713480088144908801148807855
:10F500000007000F4880002407E00E48C01C015D82
:10F510000E48001D0155601CC4B20C484088A04232
:10F52000F3DC00200649087000F06EF807494A88AD
:10F5300008880023091DFFF725FD00BFB5E700007F
:10F540004C2C00206C2B002014070000842B002082
:10F550007F2805DC7D21C90041430A4A91600DE006
:10F56000F12808DBF92806DC0107090F6422514362
:10F57000044A916002E00449024A91600221014A72
:10F58000517370475C2C002018F0010000B5030097
:10F5900011F052FA0729050B11171D23290001212B
:10F5A000144A11731449516022E00221114A117367
:10F5B000114951601CE003210E4A11730F4951603B
:10F5C00016E004210B4A11730D49516010E005212A
:10F5D000084A1173002151600AE00621054A11739F
:10F5E0000849516004E00021024A1173516000BFD4
:10F5F00000BF00BD5C2C0020A8610000F8240100C1
:10F6000028230000F04902000020014908737047D8
:10F610005C2C0020024909880918014A11807047B2
:10F620005C2C002010B52E480078102818D12D48E9
:10F63000408860280ADD2C48807800090001801C81
:10F640002949887022202649087025E026488078BC
:10F6500000090001244988702020214908701BE01E
:10F660001F480078112816D11D48807A002800D044
:10F6700010BD1B484078002800D0F9E70820184941
:10F680008872194880780009000117498870202085
:10F690001349087000E0EBE7144813490880084656
:10F6A0008078F021884330300F4988700846C07850
:10F6B0000020C87008460079142008710320887261
:10F6C0000220FFF763FF084A917A1088921CFFF727
:10F6D0000BFC054908880021FFF75CFB00BFC7E76A
:10F6E0004C2C0020842B0020782B00209407000055
:10F6F000244A118852888A4242D0224A52888A4239
:10F7000004DA204A52888A1A90B207E01D4A5288C9
:10F710000023DB439A1A521C521890B2194A5180A6
:10F72000127B002A10D0174A5268002A0CD0154AC2
:10F730005268824205D9134A5268121A114B5A6014
:10F7400002E000220F4B5A600E4A527B022A17D168
:10F750000C4A9268002A0CD00A4A9268824205D963
:10F76000084A9268121A074B9A6002E00022054B81
:10F770009A60044A9268002A02D10122014B5A730E
:10F78000704700005C2C002010B506F03BF910BD5E
:10F7900000BF704710B5044621460320400206F022
:10F7A00057F810BD10B580210320400205F0E4FF9A
:10F7B00010BD000010B50224024806F02DF80446E2
:10F7C000204610BD0106000010B50021014805F0DB
:10F7D000D3FF10BD0106000010B5044621460248C3
:10F7E00006F036F810BD00000106000010B58021BB
:10F7F000014805F0C1FF10BD0106000030B5034609
:10F800000C46002101250D48834201D0002B01D177
:10F81000022030BD012A01D10120FAE7002108E0D1
:10F82000C8002058984202D100252846F1E7481C1C
:10F8300081B29142F4DB2846EBE70000FFFF0000B5
:10F84000002000BF14E00021C200134B9950C200F9
:10F85000D2189180C200114B9950C200D2189180E9
:10F86000C2000F4B9950C200D2189180411C88B23F
:10F870004828E8DB0B490C4A11600C495160002113
:10F8800091600B4911610B49D16000210A4A118036
:10F890000A4A117070470000901F0020D0210020FC
:10F8A00010240020710D01007C1F00200D0E0100AE
:10F8B000B70E0100A90E0100B6000020BA0000201A
:10F8C000F0B585B00646674F384603900290002594
:10F8D000002400200190009063480068002803D0B5
:10F8E00061490868804707465F484068002803D0A0
:10F8F0005D494868804703905B488068002803D0D2
:10F90000594988688047029057480069002803D009
:10F9100055490869804700905348C068002803D0C3
:10F920005149C86880470546482D00DD48250098A4
:10F93000002876D0002D74DD4C480088A8420BDAF0
:10F940002B463A4649494A48FAF7CEFE2B464749E4
:10F950004748039AFAF7C8FE44480088002833DD78
:10F9600042480088A84202D1002040490880002473
:10F9700015E0E0003F490858E1003D4A51588842EF
:10F980000BD0E00011460858E1003A4A5050E00020
:10F9900011460858E100384A5050601C84B2AC420D
:10F9A000E7DB0120354908702C460BE00020E10020
:10F9B000314A5050E1002F4A5050E1002C4A50503B
:10F9C000601C84B2482CF1DB2B4800682549884232
:10F9D00046D0294880882A49884205DA2648808806
:10F9E0008019254988803BE000202349888008460B
:10F9F00000680190012D33DD002408E0601CC00088
:10FA00001D490858E1001C4A5050601C84B2681E11
:10FA1000A042F3DC691EC900174A019850501FE04C
:10FA2000FFE7002015490870002414E00020E100E1
:10FA3000114A5050E10089188880E1000C4A50506A
:10FA4000E10089188880E1000A4A5050E1008918D5
:10FA50008880601C84B2482CE8DB002003490880C1
:10FA600005B0F0BDFFFF00007C1F0020B6000020A5
:10FA7000D021002010240020901F0020BA00002078
:10FA8000881300002E480078401C2D4908702D482E
:10FA90000078401C2B4908702B480078401C2A49EC
:10FAA00008702A480068401C284908600846006819
:10FAB000FF219131884202D9002024490860204862
:10FAC0000078C82802D900201D4908701D48007818
:10FAD000842802D900201B4908701B480078502850
:10FAE00002D9002018490870194818490968405C73
:10FAF00018490870184812490978405C174908707D
:10FB0000174810490978405C1649087016480E4994
:10FB10000978405C15490870154809490978405C26
:10FB200014490870144806490978405C1349087064
:10FB3000134803490978405C124908707047000077
:10FB40006307002064070020650700206807002085
:10FB5000B71F02005C070020472102005D0700205C
:10FB60000F2202005E0700205B23020060070020D6
:10FB7000932202005F070020AB23020061070020F0
:10FB8000732402006207002010B58200054BD218D2
:10FB9000525C012A04D100228300024C1B195A54E2
:10FBA00010BD0000C82A002010B50446204600F011
:10FBB00055FA204600F002F810BD000010B50446CA
:10FBC000B348007800287DD1B2480088B249884205
:10FBD00078DAB248007800284FD0B1480078002881
:10FBE00003D0AC480088AF490880AF4800780028AF
:10FBF00018D1A8480188AB4800880A30814206D352
:10FC00000120A9490870A3480088A6490880A14896
:10FC10000088A449098888421CDA9E480088A149C6
:10FC2000088017E09F4801889A4800880A3081427E
:10FC300006D300209C49087096480088994908809E
:10FC40009448008897490988884203DD91480088D4
:10FC50009449088094480078002858D19348007847
:10FC6000042803D08E480078002807D089480088EF
:10FC7000822803DA05208D490870A3E08B480078BC
:10FC8000032803D086480078002809D081480088DE
:10FC9000FF211931884203DA04208449087091E079
:10FCA00082480078022803D07D48007800280AD0D6
:10FCB00078480088FF21AF31884204DA03207B496D
:10FCC00008707FE0E2E079480078012803D07448AA
:10FCD0000078002809D06F480088AF218900884249
:10FCE00003DA0220714908706CE07048007800283F
:10FCF00003D06B480078002864D066480088E12172
:10FD0000890088425EDA0120684908705AE0664836
:10FD10000078012856D165480078012803D0604852
:10FD20000078002809D05B480088E12189008842DA
:10FD300003DB00205D49087044E05C48007802283D
:10FD400003D057480078002809D052480088AF21D6
:10FD50008900884203DB01205449087032E053488F
:10FD60000078032803D04E480078002809D049487D
:10FD70000088FF21AF31884203DB02204B49087025
:10FD800020E04A480078042803D04548007800283D
:10FD900009D040480088FF211931884203DB032045
:10FDA000424908700EE041480078052803D03C48DD
:10FDB0000078002806D037480088822802DB04201B
:10FDC0003A490870FCF700FE3349643988425DD334
:10FDD0003748006800193649086031480078002823
:10FDE00008D000202E490870314908602F4800785B
:10FDF0003049087000F0A8FD00281FD12C48006889
:10FE00002D49884239D300202949086029480078C3
:10FE100026490978884205DA26480078401C254999
:10FE200008702AE02348007820490978884224DDB8
:10FE300020480078401E1F4908701EE01C480068DA
:10FE40001E49884219D300201949086019480078D2
:10FE500016490978884205DA16480078401C154989
:10FE600008700AE01348007810490978884204DDD8
:10FE700010480078401E0F4908700E4800780B4962
:10FE80000978884202D100200949086010BD0000AD
:10FE90000B000020020000201C0C000012000020BB
:10FEA00008000020040000200A00002006000020B6
:10FEB0001800002007000020C05D0000407E050003
:10FEC00000200B4908700B49087001200A4908708E
:10FED0000A49087000200A4908700A4908700A494E
:10FEE00008800A4908800A4908800A490870704752
:10FEF0000600002007000020080000200900002064
:10FF00000A0000200B0000200C0000200E00002042
:10FF1000100000201200002000200B4908700B493F
:10FF2000087001200A4908700A49087000200A492F
:10FF300008700A4908700A4908800A4908800A4975
:10FF400008800A490870704706000020070000205A
:10FF500008000020090000200A0000200B000020FB
:10FF60000C0000200E0000201000002012000020D5
:10FF7000F8B50646002700240025002000903148EF
:10FF80000078002809D00320F9F7EEFA002804D001
:10FF90000320F9F7DDFA2C4908802C4800880A284C
:10FFA0004AD300202949088029480078282829D2E6
:10FFB0000320F9F7CDFA0746002407E06000254941
:10FFC000085AB84200DD05E0601CC4B22048007841
:10FFD0008442F3DB00BF1E48057808E0681E40003D
:10FFE0001C49085A69001B4A5052681EC5B2A542F6
:10FFF000F4DC600017490F5215480078401C144982
:020000040001F9
:10000000087019E0002000900F2407E060001149FB
:10001000095A009808180090601CC4B2192CF5D336
:100020000A210098F8F792F807490880002008494B
:1000300008700120084908700448008880190349A5
:100040000880F8BD090000200200002016000020F2
:1000500000000020F4070020120000203949098820
:100060001E2928DA0021384A1180384A118038497F
:100070000988384A914207DC37490978002914D0A9
:1000800033490988914210DC0121344A1170002162
:10009000334A1170334A11702F4A11700121324ACC
:1000A00011700021314A11704BE029490988091863
:1000B000274A118045E023490988264A6432914243
:1000C0002ADB0021224A1180204A11801E4909881A
:1000D000204A914207DC20490978002916D01A49A4
:1000E0000988914212DC02211C4A117000211C4A2D
:1000F000117005211B4A11700021174A117001214E
:10010000194A11700021194A11701AE00E49098824
:1001100009180D4A118014E000210D4A11800A4A85
:1001200011800A4909880B4A914205DD00210B4ADA
:100130001170094A117004E0044909880918034A3A
:100140001180704702000020100000200C000020E9
:100150000E000020B80B0000090000200B0000205A
:100160000600002007000020080000200A000020F0
:100170000148007870470000502600200148407A6E
:10018000704700005026002010B50A210248006880
:10019000F7F7DCFF80B210BDC40000200148807872
:1001A0007047000050260020F8B500230025009578
:1001B0000024002200BF94E001259D40ACB20D88D0
:1001C00025400095009DA5426FD11A468D79012DDD
:1001D0000DD1464D03263602AD192D5C0126964001
:1001E0003543424E03273F02F61935540CE03F4D8C
:1001F00003263602AD192D5C01269640B5433B4ED1
:1002000003273F02F6193554CD78002D4ED1374DD6
:1002100060352D5CCE78002E01D1012600E000264D
:100220009640B543314E603635548D78002D2ED131
:100230002E4D19267601AD192D5C8E78002E01D138
:10024000012600E000269640B543284E19277F017D
:10025000F61935540D79002D0ED1244D50352D5CF5
:100260000E79002E01D1012600E000269640B5430C
:100270001E4E5036355423E01C4D50352D5C0E7902
:1002800096403543EEB2194D50352E5418E0174DB7
:1002900019267601AD192D5C8E7896403543134EA4
:1002A00019277F01F61935540AE018E00F4D603523
:1002B0002D5CCE7896403543EEB20C4D60352E5411
:1002C0004D79012D0AD1094D30352D5C012696401E
:1002D0003543EEB2054D30352E5400E000BF5D1CB5
:1002E000ABB2082B00DA67E7F8BD0000000004405D
:1002F000FFB5074615461E4600243846019900F012
:100300001FF8002802D0012004B0F0BD00240CE04A
:100310000A2060430949085CB04204D129462046BE
:1003200000F05EF807E0601C84B20A2060430349D5
:10033000085C0028ECD100BF0020E5E7B8010020F0
:100340000246002A03D1402901DD01207047032A1B
:1003500003D1022901DD0120F8E7042A03D1202975
:1003600001DD0120F2E7052A03D1202901DD01206A
:10037000ECE70C2A03D1102901DD0120E6E70D2A64
:1003800005D1012903DD402901DA0120DEE70E2A2B
:1003900003D1202901D10120D8E70020D6E70000B1
:1003A00010B5064A03231B02D218125C8A43034B82
:1003B000032424021B191A5410BD0000000004403D
:1003C00010B5064A03231B02D218125C0A43034BE2
:1003D000032424021B191A5410BD0000000004401D
:1003E00070B502460020B1E00A2353435A4C1B1952
:1003F0005B1C440004191B199B788B427DD10A2396
:100400005343554C1B195B1C440004191B195B78A2
:10041000082B33D10A2353434F4C1B195B1C440058
:1004200004191B574D4C4E4D6419E35C01242343C2
:100430000A245443484D6419641C45004519645707
:10044000464D474EAD192B550A235343424C1B19B9
:100450005B1C440004191B57404C35466419E35C8F
:10046000022423430A2454433B4D6419641C450071
:1004700045196457394DAD192B5564E00A23534390
:10048000354C1B195B1C440004191B195B78092BA4
:1004900034D10A235343304C1B195B1C440004190C
:1004A0001B572E4C2E4D6419E35C402423430A2431
:1004B0005443294D6419641C450045196457274D60
:1004C000274EAD192B550A235343234C1B195B1C94
:1004D000440004191B57214C35466419E35C802401
:1004E000A3430A2454431C4D6419641C4500451958
:1004F00064571A4DAD192B5525E025E00A235343C7
:10050000154C1B195B1C440004191B57134C144D4C
:100510006419E35C0A2454430F4D6419641C4500BC
:100520004519641965780124AC402343DCB20A23E1
:100530005343094D5B195B1C450045195B57074D3B
:10054000074EAD19EC5404E0431CD8B2032800DA7E
:100550004AE700BF70BD0000B80100200000044061
:1005600075080000F8B50024FCF748FA012861D1AD
:1005700000F0A6FB0446FF220721002003F0BCF890
:10058000012C21D100F09AFC00280ED000F0AAFB2B
:10059000054600F09BFB064601200346024629461D
:1005A0000090304605F068FC50E000F09BFB0546EB
:1005B00000F08CFB064601200023024629460090ED
:1005C000304605F059FC41E0022C21D100F076FCC8
:1005D00000280ED000F086FB054600F077FB0646AB
:1005E00001200346024629460090304605F044FCAF
:1005F0002CE000F077FB054600F068FB0646002083
:1006000001231A4629460090304605F035FC1DE0CE
:1006100000F054FC054600F065FB064600F056FB72
:100620000746012003462A4631460090384605F029
:1006300023FC0BE00020034602460146009005F033
:100640001BFC00220721104603F056F8F8BD0000FD
:10065000FEB5002481480078012827D1FCF7CEF9A7
:10066000012815D1FBF7ACFF00BF0EE0182C0AD013
:10067000152C08D00D2C06D01A2C04D0FF222146B0
:10068000002003F039F8601CC4B2242CEEDBE4E057
:10069000FCF7E2F8002406E000222146104603F0B1
:1006A0002BF8601CC4B2242CF6DBD6E0FCF7A6F9CC
:1006B00001287BD1FCF788F96949884278D300F09A
:1006C0000BFB064600F022FB07460A21F7F73EFD2A
:1006D00005463246294601200BF08AF900F060FDFC
:1006E000064600F0E1FC0A210290F7F72FFD0546CF
:1006F00000F0F2FA07463246294609F007F9FFF7FB
:1007000031FF00F0CBFA05462946012007F044FCF2
:1007100000F0F6FA0646FF21F531F7F72DFDC5B2D8
:100720002946012006F064FBFFF722FD0546FFF78E
:100730002BFD0646FFF732FD07462B46324639466B
:10074000012005F073FE00F005F905462946012059
:100750000BF0F4FB00F0CEFC054600F0C7FB0646AC
:1007600000F0CEFC074600F0C7FB00233A460146E6
:1007700000960195029001200AF056FEFF22032107
:10078000002002F0B9FFFF220421002002F0B4FF94
:1007900000F07EFC054600F075FC064600F07EFC8D
:1007A00007462A46314607F02BFE56E00DE0FFE7EC
:1007B000FF220321002002F09FFFFF2204210020DE
:1007C00002F09AFFFBF776FF47E0FCF745F80022BE
:1007D0000321104602F090FF00220421104602F08F
:1007E0008BFF00222321104602F086FF00222221E7
:1007F000104602F081FF00220721104602F07CFF24
:1008000000220821104602F077FF0022092110463D
:1008100002F072FF00220A21104602F06DFF002252
:100820001321104602F068FF00221121104602F049
:1008300063FF00221221104602F05EFF00220E210B
:10084000104602F059FF00220F21104602F054FF1B
:1008500000221021104602F04FFFFEBDED000020E7
:10086000B80B0000014908607047000090070020A5
:1008700002480068401C0149086070478C0700204E
:10088000F3B581B0064600200E49086000F01EF85E
:10089000044600F01BF805462F1B3046029903F072
:1008A0003DFF00900AE000F011F805462F1B0648B6
:1008B0000068002802D004480068804700988742FA
:1008C000F1D3FEBD8C07002090070020014800688E
:1008D000704700008C0700200B490978012901D1DD
:1008E00001200FE008490978022901D1022009E01E
:1008F00005490978032901D1042003E00121024AB6
:1009000011700120704700001D07002010B5094B31
:100910001B8899B20A12C8B2D3433133064C2370F4
:10092000C3432333637013465633A37003467133B6
:10093000E37010BD54070020230700200148008801
:10094000704700001C00002001480088704700002C
:100950003400002001480078704700008D0000201E
:1009600001480078704700008E00002010B500227A
:1009700005210648FAF7B0FB0402012205210348CD
:10098000FAF7AAFB201880B210BD00006008002012
:1009900010B5062205210348FAF79EFBC006C00FDA
:1009A00010BD00006008002010B504220521064893
:1009B000FAF792FB0402052211460348FAF78CFB72
:1009C000201880B210BD00006008002010B506227B
:1009D00005210248FAF780FBC01110BD6008002015
:1009E00010B5022205210248FAF776FB10BD00007F
:1009F0006008002010B5062205210348FAF76CFBB9
:100A00008006C00F10BD00006008002010B5042251
:100A100002210348FAF760FBC007C00F10BD0000B9
:100A20006008002010B5052202210348FAF754FBA4
:100A3000C007C00F10BD00006008002010B50022E4
:100A400004210348FAF748FB4006400F10BD0000A0
:100A50006008002010B5042201210248FAF73CFB8F
:100A6000801110BD6008002010B50022012102484D
:100A7000FAF732FB10BD00006008002010B5052217
:100A800001210348FAF728FB8007800F10BD000002
:100A90006008002010B5012211460248FAF71CFB3D
:100AA00010BD00006008002010B5002206210C488F
:100AB000FAF712FB0402012206210948FAF70CFB9F
:100AC00020180402022206210548FAF705FB201827
:100AD0000402032206210248FAF7FEFA201810BD8C
:100AE0006008002010B5042206210C48FAF7F4FA39
:100AF0000402052206210948FAF7EEFA201804023A
:100B0000062211460548FAF7E7FA201804020722E0
:100B100006210248FAF7E0FA201810BD600800200C
:100B200010B5022203210248FAF7D6FA10BD0000E0
:100B30006008002010B5032200210248FAF7CCFA21
:100B400010BD00006008002010B5002211460248C8
:100B5000FAF7C2FA10BD00006008002010B50422A8
:100B600000210248FAF7B8FA10BD00006008002022
:100B700010B5012200210248FAF7AEFA10BD0000BC
:100B80006008002010B5052200210248FAF7A4FAF7
:100B900010BD0000600800200146322915DA3E48E9
:100BA0008078012803DD01203B4A507070E03A480C
:100BB0008078002805DD2F296ADC0020364A507035
:100BC00066E00020344A507062E03E2917DA32298C
:100BD00015DB31488078022803DD02202E4A507050
:100BE00056E02D488078012805DD3B2950DC0120A6
:100BF000294A50704CE00120274A507048E05029A3
:100C000017DA3E2915DB24488078032803DD03200A
:100C1000214A50703CE020488078022805DD4D29AB
:100C200036DC02201C4A507032E002201A4A507012
:100C30002EE0622917DA502915DB1748807804283E
:100C400003DD0420144A507022E013488078032802
:100C500005DD5F291CDC03200F4A507018E00320DB
:100C60000D4A507014E073290FDA62290DDB0A482F
:100C70008078042805DD70290ADC0420064A5070BB
:100C800006E00420044A507002E00520024A507039
:100C90000148407870470000502600200148007845
:100CA00070470000070000200148006870470000FE
:100CB000901F00200148007870470000E1000020EC
:100CC0000148007870470000E000002001480078EB
:100CD00070470000E50000200148007970470000DF
:100CE0004C2800200148407870470000E5000020B3
:100CF0000148007A704700004C280020002070470F
:100D000001480088704700001E00002010B5002434
:100D1000FFF7E2FF00280AD10A4800880A49884202
:100D200002DB0846074908800648048808E00548B1
:100D30000088FCF7E9FB84B20448844200DB0446E7
:100D4000204610BD36000020C6070000CE0400007B
:100D5000002005490988054A914202DB1146024AF2
:100D6000118001490888704736000020C60700003E
:100D7000F8B50027002500260024FFF7E5FE05460C
:100D8000FFF7F6FE0646F020284000110A2805DB92
:100D9000F02028400011C01C044303E0F02028404C
:100DA0000011044324022807000F0A2804DB280747
:100DB000000FC01C044302E02807000F0443240274
:100DC000F020304000110A2805DBF02030400011EF
:100DD000C01C044303E0F02030400011044324020F
:100DE0003007000F0A2804DB3007000FC01C044343
:100DF00002E03007000F0443002C01D10248F8BD87
:100E000027463846FBE70000FFFF0000F8B5002743
:100E1000002500260024FFF7A1FE0546FFF7B2FEDD
:100E20000646F020284000110A2805DBF020284063
:100E30000011C01C044303E0F020284000110443CB
:100E400024022807000F0A2804DB2807000FC01C13
:100E5000044302E02807000F04432402F02030403E
:100E600000110A2805DBF02030400011C01C0443AB
:100E700003E0F02030400011044324023007000F4B
:100E80000A2804DB3007000FC01C044302E03007CF
:100E9000000F0443002C01D10248F8BD2746384614
:100EA000FBE70000FFFF000010B50024FFF742FE43
:100EB0000446204610BD012070470000014800781C
:100EC000704700005D07002001480078704700006F
:100ED0005F0700200148C07B70470000C809002060
:100EE0000148C07C70470000C80900200148007A12
:100EF00070470000C809002010B50024054800888C
:100F0000323084B264212046F7F736F984B22046A5
:100F100010BD0000C809002070B50024074908680A
:100F2000FBF78CFE05466421F7F710F984B20448FC
:100F3000844200DD0446204670BD0000C809002040
:100F4000DE03000010B5002400F014F8012800D1E1
:100F50000CE000F00FF8022802D1FF24373405E03E
:100F60000A2103480088F7F707F984B2204610BD2C
:100F70000200002001480078704700000B000020AC
:100F8000002005490968002903D003490968086859
:100F900000E00248704700006C010020307500003E
:100FA00010B50024044804F037FC002801D00124C7
:100FB00000E00024204610BD0407000010B5002406
:100FC000044804F029FC002801D0012400E000249A
:100FD000204610BD0507000010B50024044804F0A9
:100FE0001BFC002801D0012400E00024204610BD95
:100FF0000707000010B50024062004F00DFC0028AF
:1010000001D0012400E00024204610BD10B50024CA
:10101000052004F001FC002801D0012400E0002498
:10102000204610BD10B50024044804F0F5FB00284C
:1010300001D0012400E00024204610BD0607000076
:1010400010B50024044804F0E7FB002801D0012477
:1010500000E00024204610BD0305000010B5002468
:10106000044804F0D9FB002801D0012400E000244A
:10107000204610BD040500000148807A704700003A
:10108000C80900200148807870470000600A0020ED
:101090000148406870470000600A0020014840781D
:1010A00070470000600A002070B50024FFF714FEAE
:1010B000002803D1FCF73CFC04460DE0FFF70CFED2
:1010C000012806D1FCF734FC0546FCF71DFA04465E
:1010D00002E0FCF72DFC0446204670BD0148007C70
:1010E00070470000C80900200148007D70470000DB
:1010F000C80900200148407A70470000C809002054
:1011000010B5002405488088323084B2642120461E
:10111000F7F732F884B2204610BD0000C80900205D
:1011200070B5002407494868FBF788FD054664212F
:10113000F7F70CF884B20448844200DD04462046E8
:1011400070BD0000C8090020DE03000070B50BF080
:1011500003FA05460BF000FA04490860002D01D19E
:10116000012400E00024204670BD0000780100202A
:101170000148007B70470000C80900200148407BFF
:1011800070470000C80900200148807B70470000BC
:10119000C80900200148007870470000E4000020E2
:1011A00070B50024FFF798FD002803D1FCF7E2FB9F
:1011B00004460FE0FFF790FD012807D10020FCF75F
:1011C000D9FB0546FCF7A0F9044603E00020FCF734
:1011D000D1FB0446204670BD0148007870470000EE
:1011E0003E00002070B505460024032D00D170BDDF
:1011F000002D01D0012D1BD181210320800204F09C
:10120000BBFA8021134804F0B7FA32211248FFF7E5
:1012100037FB002409E0A200104BD2189178A200FD
:10122000985A04F0A9FA601CC4B23B2CF3DB0FE01F
:10123000022D0DD1002409E0A200094BD2189178AB
:10124000A200985A04F098FA601CC4B23B2CF3DB5D
:1012500000BFCCE702060000A0860100D415020002
:10126000C0160200F8B5002100240023002200BFB0
:101270000AE001258D40ABB205881D402C469C42FA
:1012800000D10A464D1CA9B21029F2DB0588FF2DBA
:101290001FDC284D6D7E0688B543264E7576354693
:1012A0002D7E0688B543234E357635466D7E86788D
:1012B000F607F60F964035431E4E757635462D7E61
:1012C000867802273E40760896403543194E35769B
:1012D00022E0184DED7E0688B543164EF57635466C
:1012E000AD7E0688B543134EB5768578ED07ED0FD4
:1012F0001646083EB5400F4EF67E35430D4EF57648
:101300008578022635406D081646083EB540094EE0
:10131000B67E3543074EB5760025009505E000BF43
:101320006D462D786D1CEEB200966D462D78012D20
:10133000F5D9F8BD206B0440C107C90F002905D0BD
:101340000021394A1171002238490A7102210140F5
:10135000002905D00021344A1172002233490A7253
:1013600004210140002905D000212F4A11730022D9
:101370002E490A7308210140002905D000212A4A7C
:101380001174002229490A7410210140002905D056
:101390000021254A1175002224490A7520210140A7
:1013A000002905D00021204A117600221F490A7623
:1013B00040210140002904D000221B494A711B49E9
:1013C0004A7180210140002904D0002216494A7246
:1013D00016494A72FF2101310140002904D0002240
:1013E00011494A7311494A730121490201400029F8
:1013F00004D000220C494A740C494A740121890224
:101400000140002904D0002207494A7507494A755E
:101410000121C9020140002904D0002202494A7674
:1014200002494A76704700000060004000610040B9
:10143000C107C90F002905D001223C490A710021CA
:101440003B4A117102210140002905D00122374990
:101450000A720021364A117204210140002905D088
:10146000012232490A730021314A117308210140D7
:10147000002905D001222D490A7400212C4A11743B
:1014800010210140002905D0012228490A750021B8
:10149000274A117520210140002905D00122234946
:1014A0000A760021224A117640210140002905D008
:1014B00001221E494A7100221D494A7180210140C2
:1014C000002905D0012219494A72002218494A729E
:1014D000FF2101310140002905D0012213494A733F
:1014E000002213494A73012149020140002905D015
:1014F00001220E494A7400220D494A7401218902D1
:101500000140002905D0012208494A7500220849F6
:101510004A750121C9020140002905D00122034971
:101520004A76002202494A76704700000061004076
:101530000060004010B50C480078002803D00B4A2A
:1015400050689168884708484078002803D0084AC6
:1015500050689168884704488078002803D0054A7D
:1015600050689168884710BD006000400803002063
:10157000880400200806002010B5084800790028DB
:1015800003D0074A10695169884704484079002808
:1015900003D0044A50689168884710BD006000403D
:1015A000080300209404002010B50848007A0028A1
:1015B00003D0074AD069116A88470448407A002856
:1015C00003D0044A50689168884710BD006000400D
:1015D00008030020A004002010B50848007B002864
:1015E00003D0074A906AD16A88470448407B0028A4
:1015F00003D0044A50689168884710BD00600040DD
:1016000008030020AC04002010B50848007C002826
:1016100003D0074A506B916B88470448407C0028F0
:1016200003D0044A50689168884710BD00600040AC
:1016300008030020B804002010B50848007D0028E9
:1016400003D0074A106C516C88470448407D00283D
:1016500003D0044A50689168884710BD006000407C
:1016600008030020C404002010B50848007E0028AC
:1016700003D0074AD06C116D88470448407E00288B
:1016800003D0044A50689168884710BD006000404C
:1016900008030020D004002010B50848407F00282F
:1016A00003D0074A5068916888470448007F0028A3
:1016B00003D0044A906DD16D884710BD0060004092
:1016C000DC0400200803002010B5084840780028FA
:1016D00003D0074A5068916888470448007800287A
:1016E00003D0044A506E916E884710BD20600040C0
:1016F000E80400200803002010B5094800790028FC
:1017000003D0084A106F516F88470548001D407884
:10171000002803D0044A50689168884710BD000033
:101720002060004008030020F404002010B5034AA4
:10173000D06F78329168884710BD00000803002000
:1017400010B5024A50689168884710BD8C0300208C
:1017500010B50948007C002803D0084A50689168F9
:101760008847054810304078002803D0044A506864
:101770009168884710BD0000206000409803002059
:101780001805002010B5024A50689168884710BDBE
:10179000A403002010B5024A50689168884710BD24
:1017A000B003002010B50948007F002803D0084A84
:1017B00050689168884705481C304078002803D05D
:1017C000044A50689168884710BD000020600040BE
:1017D000BC0300203C05002010B50C480078002810
:1017E00003D00B4A50689168884708484078002821
:1017F00003D0084A506891688847044880780028D8
:1018000003D0054A50689168884710BD4060004089
:10181000C803002048050020C806002010B50D4868
:101820000079002803D00C4A50689168884709481D
:10183000001D4078002803D0084A50689168884706
:101840000448001D8078002803D0054A506891683C
:10185000884710BD40600040D4030020540500209C
:10186000D406002010B50D48007A002803D00C4A99
:10187000506891688847094808304078002803D0AC
:10188000084A5068916888470448083080780028E2
:1018900003D0054A50689168884710BD40600040F9
:1018A000E003002060050020E006002010B50D4890
:1018B000007B002803D00C4A50689168884709488B
:1018C0000C304078002803D0084A50689168884757
:1018D00004480C308078002803D0054A506891688D
:1018E000884710BD40600040EC0300206C050020DC
:1018F000EC06002010B50D48007C002803D00C4AEF
:10190000506891688847094810304078002803D013
:10191000084A506891688847044810308078002849
:1019200003D0054A50689168884710BD4060004068
:10193000F803002078050020F806002010B5024AC0
:1019400050689168884710BD0404002010B509480C
:10195000007E002803D0084A5068916888470548EF
:1019600018304078002803D0044A506891688847AE
:1019700010BD0000406000401004002090050020D1
:1019800010B50948007F002803D0084A50689168C4
:10199000884705481C304078002803D0044A506826
:1019A0009168884710BD0000406000401C04002082
:1019B0009C05002010B508480078002803D0074A8D
:1019C00050689168884704484078002803D0044A4A
:1019D00050689168884710BD60600040280400206E
:1019E000A805002010B509480079002803D0084A4E
:1019F0005068916888470548001D4078002803D04A
:101A0000044A50689168884710BD0000606000403B
:101A100034040020B405002010B50948007A0028DD
:101A200003D0084A506891688847054808304078D4
:101A3000002803D0044A50689168884710BD000010
:101A40006060004040040020C005002010B5024A3C
:101A500050689168884710BD4C04002010B5024AB8
:101A600050689168884710BD5804002010B5094897
:101A7000007D002803D0084A5068916888470548CF
:101A800014304078002803D0044A50689168884791
:101A900010BD00006060004064040020E4050020E8
:101AA00010B50948007E002803D0084A50689168A4
:101AB0008847054818304078002803D0044A506809
:101AC0009168884710BD00006060004070040020ED
:101AD000F005002010B50948007F002803D0084A0F
:101AE00050689168884705481C304078002803D02A
:101AF000044A50689168884710BD0000606000404B
:101B00007C040020FC05002010B5FE4800688079A8
:101B1000002806D001286ED002286DD003286CD191
:101B200004E2F8480068407903000EF085FF0A06D9
:101B300014BC2BBC47BC67BC9BBC0AF0D7FF002081
:101B4000F0490968C873EF4800684079401CED49C6
:101B500009684871AEE0EC490969EA4A1268D27A2C
:101B6000885C0BF03BF8E74800684079401CE54989
:101B700009684871E34800684079401CE1490968F8
:101B8000487197E001F020FF002810D10BF026F8F3
:101B9000DC4800684079401CDA4909684871D94836
:101BA00000684079401CD7490968487105E00AF08F
:101BB000C7FF0020D349096848717BE001F004FFAA
:101BC000002811D101200BF009F8CE4800684079B7
:101BD000401CCC4909684871CA4800684079401CDB
:101BE000C8490968487105E00AF0AAFF0020C54904
:101BF000096848715EE05FE0FEE0A3E101F0E4FE09
:101C0000002828D1BF490968C97A24225143BF4A14
:101C100012688918BB4A1268D27B885C0AF0DEFF22
:101C2000B8480068C07B401CB6490968C873B5480D
:101C30000068C07B242814D3B24800684079401C57
:101C4000B04909684871AF4800684079401CAD4907
:101C50000968487105E00AF073FF0020A949096886
:101C6000487127E001F0B0FE002815D1A5480068B2
:101C7000C07A401CA3490968C872A2480068C07AAB
:101C8000A1490978884207DB00209E490968C8728B
:101C900001209C49096888710AF052FF0020994987
:101CA0000968487106E00AF04BFF00209549096871
:101CB000487100BF00BF4FE19248006840790300BF
:101CC0000EF0BAFE080513912A91479170910AF01F
:101CD0000DFF00208B490968C8738A480068407965
:101CE000401C88490968487184E087490969854A28
:101CF0001268D27A885C0AF071FF824800684079E5
:101D0000401C8049096848717E4800684079401C41
:101D10007C49096848716DE001F056FE002811D138
:101D200026200AF05BFF774800684079401C75491F
:101D300009684871734800684079401C7149096816
:101D4000487105E00AF0FCFE00206E490968487100
:101D500050E001F039FE00281DD101200AF03EFFBD
:101D600068480068C07B401C66490968C8736548BC
:101D70000068C07B242814D3624800684079401C66
:101D80006049096848715F4800684079401C5D49B6
:101D90000968487105E00AF0D3FE00205949096836
:101DA000487127E001F010FE002815D15548006861
:101DB000C07A401C53490968C87252480068C07A0A
:101DC00051490978884207DB00204E490968C872EA
:101DD00002204C49096888710AF0B2FE0020494986
:101DE0000968487106E00AF0ABFE00204549096821
:101DF000487100BF00BFAFE042480068407903006F
:101E00000EF01AFE0805138B2A8B478B638B0AF0A2
:101E10006DFE00203B490968C8733A480068407964
:101E2000401C3849096848717EE037490969354ADC
:101E30001268D27A885C0AF0D1FE32480068407994
:101E4000401C3049096848712E4800684079401CA0
:101E50002C490968487167E001F0B6FD002811D1EE
:101E600025200AF0BBFE274800684079401C254920
:101E700009684871234800684079401C2149096875
:101E8000487105E00AF05CFE00201E4909684871AF
:101E90004AE001F099FD002810D10AF09FFE194890
:101EA00000684079401C1749096848711548006866
:101EB0004079401C13490968487105E00AF040FE6A
:101EC00000201049096848712EE001F07DFD0028CE
:101ED00015D10C480068C07A401C0A490968C872CC
:101EE00008480068C07A08490978884207DB002062
:101EF00004490968C87203200249096888710AF018
:101F00001FFE05E0E00700204C2F0020DC0700202A
:101F1000002012490968487106E00AF011FE00200D
:101F20000E490968487100BF00BF15E000200B4949
:101F300009688871094909684871062007490968D4
:101F4000C87009E00AF0FCFD0020044909684871E6
:101F500002490968887100BF00BF10BDE00700207A
:101F600010B56A480068407903000EF065FD090667
:101F700010C627C644C6608EC6000AF0B7FD634887
:101F800000684079401C614909684871BCE06049BB
:101F900009695E4A1268D27A885C0AF01FFE5B48C3
:101FA00000684079401C59490968487157480068E1
:101FB0004079401C554909684871A5E001F004FDCD
:101FC000002811D14F200AF009FE504800684079DE
:101FD000401C4E49096848714C4800684079401CD3
:101FE0004A490968487105E00AF0AAFD00204749FE
:101FF0000968487188E001F0E7FC002810D10AF078
:10200000EDFD424800684079401C4049096848712C
:102010003E4800684079401C3C490968487105E029
:102020000AF08EFD00203949096848716CE001F022
:10203000CBFC002822D135480068C07A401C3349C7
:102040000968C87231480068C07A31490978884205
:102050000FDB00202D490968C8722C4800684079C0
:10206000401C2A49096848710020284909684862CB
:1020700008E0002025490968487103E00020234951
:10208000096848710AF05CFD3EE020480068407C29
:10209000002816D01E48C068002803D01C48C1681C
:1020A00019208847002019490968486217490968BA
:1020B0004871164909688871052014490968C87073
:1020C0001AE012480068406A282807D20F480068C2
:1020D000406A401C0D49096848620DE000200B4928
:1020E000096848620949096848710849096888719E
:1020F000052006490968C87006E00AF021FD0020A5
:1021000002490968487100BF00BF10BDE007002008
:102110004C2F002010B50024F7480068807A012871
:102120007ED1F5480068C07900287AD0F24800686E
:102130008079002804D0012874D0022873D191E15D
:10214000ED480068007B24286ED2EB480068C07917
:1021500001287AD1002475E0E7480068C07A24217C
:102160004843E64909684018E3490968097B415C2E
:10217000E1480068C07A24225043E14A126880187E
:10218000DD4A1268127B805C814229D0DA480068FF
:10219000C07A24214843DA4909684018D6490968B9
:1021A000097B415CD4480068C07A24225043D34A5A
:1021B00012688018D04A1268127B8154CE48006899
:1021C000407B242805D3CC480068007BCA490968B5
:1021D0004873C9480068007BC7490968887308E0EC
:1021E000C5480068407B242803D20120C249096801
:1021F0008871C1480068007B401CBF4909680873AA
:10220000BD480068007B242808D3BB480068407B99
:10221000242803D20120B84909688871B64805E02E
:10222000D3E1CDE169E0BAE138E00EE00068007B7F
:10223000242804D2B04800688079012800D103E046
:10224000601CC4B2242C87D356E0002413E0AA48B3
:102250000068C07A24214843A94909684018015DF3
:10226000A5480068C07A24225043A44A1268801806
:102270000155601CC4B2242CE9D300209E49096892
:10228000487323209C490968887301209A4909688A
:10229000887124209849096808732DE00020964928
:1022A0000968087394480068C07A401C924909681C
:1022B000C87291480068C07A92490978884217DB51
:1022C0008D480068007C012804D102208A490968F1
:1022D000887106E000208849096888718649096884
:1022E000C871002084490968C87283490968087464
:1022F000002081490968487161E17F4800684079A0
:1023000003000EF099FB080513A62AA651A68EA677
:1023100001207949096808740AF0E8FB76480068EA
:102320004079401C74490968487199E07549096908
:10233000714A1268D27A885C0AF050FC6E480068D4
:102340004079401C6C49096848716B4800684079C5
:10235000401C69490968487182E001F035FB00289A
:102360001BD165490968497B491CC8B20AF036FC93
:1023700061480068407B60490968C8735E4800682E
:102380004079401C5C49096848715B4800684079A5
:10239000401C59490968487105E00AF0D1FB00204A
:1023A0005549096848715BE001F00EFB00282BD10C
:1023B00051490968C97A24225143504A1268891840
:1023C0004D4A1268D27B885C0AF008FC4A480068D3
:1023D000C07B401C48490968C87347480068C07BF7
:1023E00045490968897B88421ADD4348006840797D
:1023F000401C4149096848713F4800684079401CC9
:102400003D49096848710BE00AF09AFB3A480068B8
:10241000407B39490968C873002037490968487109
:102420001EE001F0D1FA00280CD133490968887107
:10243000242031490968C8732F49096848732E4917
:10244000096888730AF07CFB00202B4909684871F1
:1024500006E00AF075FB002027490968487100BFB3
:1024600000BFACE024480068407903000EF0E4FAB5
:1024700008050F8E268E4C8E688E0AF037FB1E489C
:1024800000684079401C1C490968487185E01D4975
:102490000969194A1268D27A885C0AF09FFB1648CB
:1024A00000684079401C1449096848711248006866
:1024B0004079401C1049096848716EE001F084FAC7
:1024C000002811D125200AF089FB0B4800684079CB
:1024D000401C094909684871074800684079401C58
:1024E00005490968487105E00AF02AFB0020024905
:1024F0000968487151E00000E0070020DC07002077
:10250000D80700204C2F002001F05EFA002810D1DF
:102510000AF064FB644800684079401C624909681D
:102520004871614800684079401C5F4909684871FA
:1025300005E00AF005FB00205B49096848712CE0C2
:1025400001F042FA00281AD157480068C07A401CAE
:1025500055490968C87254480068C07A53490978D7
:1025600088420CDB002050490968C8724E4909684E
:1025700088714D49096848714B490968C8710AF06A
:10258000DFFA002048490968487106E00AF0D8FAE5
:10259000002045490968487100BF00BF0FE00AF0FC
:1025A000CFFA00204049096848713F49096888719D
:1025B0003D49096808733C490968C87200BF71E069
:1025C00000203949096888726CE037480068807AD1
:1025D000022867D134480068007A00285ED032486B
:1025E00000684079002804D001280CD0032846D187
:1025F0001BE00AF07BFA2C4800684079401C2A490D
:102600000968487149E000200AF0E8FA26480068A5
:102610004079401C24490968487123480068407982
:10262000401C21490968487137E00AF029FA00285E
:1026300012D11D4800684078401C1B490968487049
:10264000194800684078032812D301F05DFA002091
:102650001549096848700BE00020134909680872A1
:10266000AA2011490968887000200F49096848703C
:102670000AF066FA00200C49096848710DE00AF07A
:102680005FFA0020084909684871074909684870DD
:10269000AA2005490968887000BF03E000200249AC
:1026A0000968887210BD0000E00700204C2F002050
:1026B000F8B504460D4600260C2060431D49085C11
:1026C000002801D00120F8BD0C20604319494018B2
:1026D00085600C20604340188068002801D10120EB
:1026E000F1E701210C206043124A115400222046D8
:1026F000E317DB0E1B185B115B01E31A9B000E4F07
:10270000DB19E717FF0E3F197F11DA550EF0C6F9F6
:1027100000222046E317DB0E1B185B115B01E31A56
:102720009F00064BFB18E717FF0E3F197F11DA5584
:102730003046C8E708030020006000400061004008
:1027400000BFFEE709480088401C08490880084689
:1027500000880749884208DD06480078002804D030
:10276000084602490880012088707047DC0000207C
:10277000DC050000E000002010B515488078012835
:1027800024D11448007801280CD11348007801287E
:1027900008D1002011498870084602F00BFE002085
:1027A0000D4908700B48007802280CD10C480078BD
:1027B000012808D1002009498870084602F0FAFD76
:1027C00000200749087000200249087010BD000071
:1027D000DC000020E0000020E2000020E5000020F6
:1027E000E30000207047000010B500F05DFE0128F6
:1027F00003D1002001490880887010BDDC00002052
:10280000F0B505460E46174600243A46314628469E
:1028100000F058FE00BF42E000202101394A126852
:1028200050522101374A126889184880002120013E
:10283000344A1268801881802001324A1268801858
:10284000C18020012F4A12688018017220012D4A90
:1028500012688018417220012A4A12688018817219
:102860002001284A12688018C17200202101254ADF
:1028700012688918087300212001224A1268801802
:102880004173002021011F4A1268891888730021B2
:1028900020011C4A12688018C173601CC4B21A4817
:1028A0004078A042B8DC64201849096808807D207F
:1028B000C00016490968488015481449096888808D
:1028C0007D20000111490968C88010490968088104
:1028D00010480E49096848810F480C4909688881E9
:1028E00040000A490968C8813220084909680882FD
:1028F000FF20F53005490968488204490968888243
:10290000F0BD0000A0070020940700209C070020D5
:102910004C040000102700003075000038B500247A
:1029200004E0002013490855601C84B2282CF8D319
:1029300001216846417001706A460F490D48FFF752
:102940005FFF7D21C900322000F0ACF90B490C4833
:1029500000F0C6F90948643000F058F90748C8305B
:1029600000F064F9074800F077F9074800F08AF9A9
:1029700038BD00005C280020A81B020028230000AE
:10298000B80B0000542400001027000010B52448A4
:102990000078002803D10120214908703EE020483A
:1029A0000078012810D11F480078012808D10020A4
:1029B0001D498870084602F0FDFC00201949087086
:1029C00002201749087029E015480078022810D124
:1029D00016480078012808D100201349887008465D
:1029E00002F0E8FC00201149087003200C4908702F
:1029F00014E00B480078032803D10520084908702B
:102A00000CE007480078052803D005480078062820
:102A100004D10020024908700549087010BD00006B
:102A2000E0000020E2000020E5000020E30000209C
:102A3000E4000020F8B50024002500263548007881
:102A400000281ED134480078002803D101203249E3
:102A5000087016E030480078012803D102202E4982
:102A600008700EE02C480078022803D103202A4980
:102A7000087006E028480078032802D10020264983
:102A800008702448007801280ED10124172500265B
:102A900022480123324629460090204601F09CFE40
:102AA00001201F49087034E01A48007802280FD12D
:102AB00001243B2500261948401C012332462946A3
:102AC0000090204601F088FE01201649087020E0A1
:102AD0001048007803280DD1FEF7FEF8002803D136
:102AE00001201149087102E000200F4908710DF022
:102AF00075FF0EE007480078052803D10620054938
:102B0000087006E003480078062802D10520014934
:102B10000870F8BDE0000020E1000020E500002082
:102B2000E2000020E30000204C28002010B50446FD
:102B300023000DF081FF095B060E16171819595A6C
:102B40005E00F9F741FF2C49884201D3FFF772FF7D
:102B500050E0F9F739FF2849884201D3FFF716FF03
:102B600048E047E046E045E0F9F72EFF2249884279
:102B700039D301F0E1FD21480078032814D1204821
:102B80000078002810D1FEF7B3F8002806D1012004
:102B90001C4988608868FAF757FF05E0002019494A
:102BA00088608868FAF750FF14480078012805D13A
:102BB00013480078002801D1FAF798F810480078F7
:102BC000052803D10120104908700AE00C4800785C
:102BD000062803D102200C49087002E000200A49AF
:102BE00008700BF09BFC05E004E003E0FFF7AAFD92
:102BF00000E000BF00BF10BDB80B0000E1000020E6
:102C0000E00000204C280020E400002001460020C5
:102C1000054A126852898A4201DC012002E0024A18
:102C200012681181704700009C07002001460020B7
:102C3000084A126812898A4201DB012009E0054A2C
:102C4000126892898A4201DC012002E0014A12687E
:102C5000518170479C07002001460020084A1268F5
:102C600052898A4201DB012009E0054A1268D289B3
:102C70008A4201DC012002E0014A1268918170471A
:102C80009C07002001460020054A126892898A426A
:102C900001DB012002E0024A1268D1817047000086
:102CA0009C070020024600200C4B1B681B8A9342A5
:102CB00001DD012010E08A4201DB01200CE0074B1E
:102CC0001B689B888B4201DC012005E0034B1B68DD
:102CD0001A80024B1B685980704700009C07002037
:102CE000024600200C4B1B681B8A934201DD012029
:102CF00010E08A4201DB01200CE0074B1B685B8877
:102D0000934201DB012005E0034B1B689A80024BD4
:102D10001B68D980704700009C07002070B50446EE
:102D200000250C206043FE490968401840680028CF
:102D300007D00C216143FA4A126889184868804715
:102D400005460C206043F6490968085C002873D1E9
:102D50000C206043F249096840188068002874D04C
:102D60002001F04909684018C07A02280AD1032DD1
:102D700008D10C206043EA4A12688018816801205B
:102D8000884762E02001E74909684018C07A0228B4
:102D90000AD1042D08D10C206043E14A1268801842
:102DA00081680220884750E02001DE490968401808
:102DB000C07A02280AD1052D08D10C206043D84AD8
:102DC000126880188168032088473EE02001D549B9
:102DD00009684018C07A02280AD1062D08D10C20B3
:102DE0006043CF4A126880188168042088472CE02D
:102DF0002001CC4909684018C07A02280AD1072D61
:102E000008D10C206043C64A1268801881680520EA
:102E100088471AE02001C34909684018C07A02288F
:102E20000BD1082D09D10C206043BD4A12688018CF
:102E300081680620884708E00DE00C206043B84A0E
:102E4000126880188168002088472001B549096808
:102E50004018C5720CE30C206043B1490968085C56
:102E6000012873D10C206043AD490968401880687F
:102E7000002874D02001AB4909684018C07A0328A3
:102E80000AD1022D08D10C206043A54A126880188F
:102E900081680120884762E02001A2490968401842
:102EA000C07A04280AD1022D08D10C2060439C4A24
:102EB0001268801881680220884750E020019949F3
:102EC00009684018C07A05280AD1022D08D10C20C3
:102ED0006043934A126880188168032088473EE067
:102EE0002001904909684018C07A06280AD1022DAD
:102EF00008D10C2060438A4A126880188168042037
:102F000088472CE02001874909684018C07A0728C3
:102F10000AD1022D08D10C206043814A1268801822
:102F20008168052088471AE020017E490968401819
:102F3000C07A08280BD1022D09D10C206043784AB1
:102F40001268801881680620884708E00DE00C2090
:102F50006043734A12688018816800208847200106
:102F6000704909684018C57282E20C2060436C49C0
:102F70000968085C0228F7D1002D7DD1200169493C
:102F80000968085A68490968098A884275DA20017F
:102F900064490968085A0A3081B22001614A1268FE
:102FA000115220015F490968085A5F490968098A76
:102FB000884231DB20015B490968401840885A4942
:102FC00009680988884227DB2001564909684018AA
:102FD000408855490968498888421DDC0020210144
:102FE000504A12688918488020014E4909684018E3
:102FF000807A0028B8D10C206043494909684018FC
:1030000080680028B0D00C206043454A12688018C0
:103010008168012088472BE2200142490968085A4B
:1030200041490968098A88429EDB20013D490968B7
:10303000401840883C4909688988884294DB20010F
:10304000384909684018408837490968C988884262
:103050008ADC00202101334A126889184880200147
:10306000304909684018807A0028D4D10C20604388
:103070002B490968401801E063E00BE080680028F4
:10308000C9D00C206043264A12688018816802204B
:103090008847EDE100202101224A12688918488002
:1030A0002101204A12688918C872002120011D4A96
:1030B00012688018C18020011A4A12688018417273
:1030C0002001184A1268801881721848017820017E
:1030D000144A12688018017200202101114A1268F6
:1030E0008918888021010F4A126889180873210104
:1030F0000C4A12688918487321010A4A1268891813
:10310000887300212001074A12688018C1730C20BF
:10311000604303490968401880680028B9D007E077
:1031200098070020A00700209C070020940700209B
:103130000C206043CF4A12688018816800208847BD
:1031400096E1012DA5D12001CB4909684018C07A2C
:10315000A84225D000212001C74A1268801841806A
:1031600000202101C44A12688918C8802001C24980
:1031700009684018C572C14800782101BE4A12682A
:103180008918487200202101BB4A1268891888807A
:10319000BA4801782001B84A12688018017267E1C4
:1031A0002001B54909684018007AB4490978884275
:1031B00020D0B24800782101AF4A126889180872FD
:1031C0002001AD4909684018407AAC490978884225
:1031D00009D02001A8490968401880882101A64A21
:1031E00012688918C88000212001A34A126880183B
:1031F000818012E02001A049096840188088A04918
:1032000088420AD220019C490968401880880A3007
:103210002101994A12688918888020019649096815
:1032200040184088964988420AD22001924909688C
:10323000401840880A3021018F4A12688918488056
:1032400020018D4909684018407A8C4909788842E4
:1032500005D001202101884A12688918887220014E
:103260008549096840184088864909680988884264
:1032700004DB00212001804A1268115220017E499E
:1032800009684018807A00287ED10C206043794973
:10329000096840188068002877D0200176490968BD
:1032A00040184088774909680989884214DB200161
:1032B000714909684018007B00280DD10C2060433B
:1032C0006C4A126880188168032088470120210118
:1032D000694A12688918087320016749096840180B
:1032E0004088684909684989884214DB200162499D
:1032F00009684018407B00280DD10C2060435D4ACE
:1033000012688018816804208847012021015A4AE8
:103310001268891848732001574909684018408885
:10332000584909688989884214DB20015249096893
:103330004018807B00280DD10C2060434D4A126854
:103340008018816805208847012021014A4A1268B7
:1033500089188873200148490968401840884949FC
:103360000968C989884210DB20014349096840186F
:10337000C07B00287CD10C2060433E4A1268801834
:1033800081680620884701E007E03BE00120210139
:10339000394A12688918C8736AE0200136490968F9
:1033A0004018407A01282ED13448007802282AD1CA
:1033B0002001314909684018C08832490968498AA2
:1033C000884255DB20012C490968401880882D4926
:1033D0000968898A88424BDB0C20604325490968CB
:1033E00040188068002843D00C206043214A1268AE
:1033F0008018816807208847002021011E4A126832
:103400008918487234E020011B4909684018407A45
:1034100002282DD119480078012829D12001164908
:1034200009684018C08817490968898A88421FDBE3
:103430002001114909684018808812490968498AA1
:10344000884215DB0C2060430A49096840188068EF
:1034500000280DD00C206043064A1268801881684D
:103460000820884700202101034A12688918487201
:1034700070BD000098070020A007002094070020DE
:10348000F0FF00009C07002010B5002400BF04E0FE
:103490002046FFF743FC601CC4B202484078A042BB
:1034A000F6DC10BD9407002010B50024044802F09B
:1034B000B3F9002800D000E00124204610BD000030
:1034C0000304000010B5074B14781C7054785C702E
:1034D000054B1960054B186003461833044C2360F4
:1034E00010BD000094070020980700209C070020D2
:1034F000A007002010B50446012C09D1FF220C21A1
:10350000002000F0F9F80121022004F0B3FE08E0E9
:1035100000220C21104600F0EFF80021022004F0F8
:10352000A9FE10BD10B5002404210848F7F7E6FDF8
:10353000552801D1012407E0042001F06FF800288C
:1035400001D0002400E00124204610BD60080020C6
:1035500010B50446012C09D1FF221C21002000F0E7
:10356000CBF80121062004F085FE08E000221C2192
:10357000104600F0C1F80021062004F07BFE10BDCB
:1035800010B50024062001F049F8002801D00124DC
:1035900000E00024204610BD10B50446012C09D1DE
:1035A000FF221721002000F0A7F80121042004F0D9
:1035B00061FE08E000221721104600F09DF800216E
:1035C000042004F057FE10BD00200449097A0029A8
:1035D00001D0012000E0002070470000600A0020B8
:1035E00010B50446022C1CD100220D21104600F01B
:1035F00083F8FDF763FC002809D0FF220B2100208F
:1036000000F07AF801210D2004F034FE58E0002289
:103610000B21104600F070F800210D2004F02AFE66
:103620004EE0032C1CD100220B21104600F064F860
:10363000FDF744FC002809D0FF220D21002000F0F6
:103640005BF801210D2004F015FE39E000220D2168
:10365000104600F051F800210D2004F00BFE2FE081
:10366000042C0ED1FF220D21002000F045F800228D
:103670000B21104600F040F801210D2004F0FAFD66
:103680001EE0012C0ED100220D21104600F034F86E
:10369000FF220B21002000F02FF801210D2004F063
:1036A000E9FD0DE000220D21104600F025F8002272
:1036B0000B21104600F020F800210D2004F0DAFD67
:1036C00010BD000010B500240A480078012801D17F
:1036D00001240CE0FCF752FD012801D1032406E08F
:1036E000FCF74CFD022801D1022400E0042420460E
:1036F00010BD0000ED00002010B5064B1B78834282
:1037000007DD242905D224234343034C24681B19D5
:103710005A5410BD4C2F0020D807002010B5744813
:103720000068407903000DF087F90B0711D325D30A
:103730005A6D77D38DA8D30009F0D8F96C4800688A
:103740004079401C6A4909684871CFE06949496974
:10375000087809F043FA664800684079401C6449DB
:1037600009684871624800684079401C60490968EE
:103770004871BBE000F028F9002811D17F2009F042
:103780002DFA5B4800684079401C59490968487126
:10379000574800684079401C5549096848711DE048
:1037A000534800684078401C5149096848705048A7
:1037B0000068407803280BD300204D490968487001
:1037C000AA204B4909688870032049490968C870D4
:1037D00009F0B6F9002046490968487186E000F012
:1037E000F3F8002807D1424800684079401C40495E
:1037F0000968487103E000203D490968487109F0F3
:103800009FF973E009F072F9394800684079401C6B
:1038100037490968487169E0364949690978491C9E
:10382000C8B209F0DBF9324800684079401C3049E1
:10383000096848712E4800684079401C2C49096885
:10384000487153E000F0C0F800280FD109F020F9CA
:10385000274909688870012009F094F92448006814
:103860004079401C22490968487105E009F068F96F
:1038700000201F490968487138E01D4800688078B9
:1038800018280CD102201A4909680870002018492C
:1038900009684870042016490968C87011E0144886
:1038A00000684078401C1249096848701048006858
:1038B0004078032805D300F027F900200C49096857
:1038C000487009F03DF900200949096848710DE088
:1038D00009F036F900200649096848710449096869
:1038E0004870AA2002490968887000BF00BF10BD57
:1038F000E00700204C2F002010B5314800684079C7
:10390000002804D001280CD0032848D11DE009F07C
:10391000EDF82B4800684079401C29490968487136
:103920004BE028490969087809F058F924480068EB
:103930004079401C22490968487121480068407953
:10394000401C1F490968487137E000F03DF8002825
:103950000CD101201A49096808700020184909682B
:103960004870042016490968C87011E014480068BE
:103970004078401C12490968487011480068407836
:10398000032805D300F0C0F800200D4909684870ED
:1039900009F0D6F800200A49096848710DE009F0DD
:1039A000CFF8002006490968487105490968487040
:1039B000AA2003490968887000BF00BF10BD00003D
:1039C000E00700204C2F002010B509F059F80446FC
:1039D0001F4800680078002838D01D480068C0786B
:1039E000042833D3002C09D1002119480068C07A7B
:1039F0008200174800681430815027E0144800689E
:103A0000C07A810012480068143040581149884239
:103A100011D20F480068C07A81000D480068143048
:103A20004058401C0A490968C97A8A00084909684F
:103A3000143188500AE000F067F80021044800685B
:103A4000C07A82000248006814308150204610BDC0
:103A5000E0070020B80B000000B587B001206946E0
:103A600008710848029008480390084804900848E4
:103A700005900848069001A9074800F00FF807B024
:103A800000BD0000C13D0100055A0100C50B020048
:103A9000151C0200141C0200C4280020F8B50646BC
:103AA0000F46002400253946304600F0EFF900BFEC
:103AB00014E000250EE00021242060430B4A126828
:103AC0008018415524206043094A126880184155E6
:103AD000681CC5B2242DEED3601CC4B20548007822
:103AE000A042E6DC00F010F8F8BD0000D807002086
:103AF000DC0700204C2F00200120024909680871D2
:103B000070470000E007002010B500F073F90020B6
:103B100003490968087002490968C87010BD0000AF
:103B2000E007002007480068C078062808D105484B
:103B30000068C079002803D1012002490968C871D2
:103B400070470000E007002010B555480068C078B5
:103B500003000CF071FF08671D1A1714110E05669B
:103B600050484068002803D04E48416800208847EC
:103B700093E000F0E5F890E000F0C6F88DE000F08A
:103B8000D1F88AE0FFF7B8FE87E0FFF7C7FD84E0D1
:103B900044484068002803D04248416801208847D3
:103BA0003F480068407C00281AD03E48C068002882
:103BB00003D03C48C168C8208847002038490968BC
:103BC0004862374800680078002804D0042034494F
:103BD0000968C87024E0022031490968C8701FE0F4
:103BE0002F480068406A401C2D49096848622C48EB
:103BF0000068406A7D21C900884211D3002028490D
:103C000009684862264800680078002804D004202B
:103C100023490968C87003E0022021490968C87077
:103C20003BE000BF1F484068002803D01D484168A2
:103C3000002088471A480068407C002813D01948A3
:103C4000C068002803D01748C168C82088470020F2
:103C500013490968486212480068C078401C10493E
:103C60000968C87018E00E480068406A401C0C499A
:103C7000096848620A480068406A7D21C900884294
:103C80000AD3002006490968486205480068C078E0
:103C9000401C03490968C87000BF00BF10BD000088
:103CA000E00700204C2F002010B515480068C078B0
:103CB000072824D0012012490968487408E01148F7
:103CC0008068002802D00F4988688047FFF73CFFD2
:103CD0000B480068C0780628F1D109480068007ACE
:103CE0000028ECD106480068C0790028E7D10448D4
:103CF0000068807A0028E2D101490968487410BD43
:103D0000E00700204C2F002010B50548006800781F
:103D1000012802D1FDF7F8FE01E0F5F7EFFC10BD38
:103D2000E007002010B5054800680078012802D19E
:103D3000FEF716F901E0F6F7BFF810BDE007002026
:103D400010B51D480068807A002829D11A480068FB
:103D5000007A002803D002201749096888721648A3
:103D60000068C079002803D00120134909688872CF
:103D7000114800680079012812D100200E49096815
:103D800008710D490968887207200B490968C870D5
:103D90000A484068002803D0084841680020884746
:103DA000054800680078012802D1FEF7B3F901E068
:103DB000F6F75CF910BD0000E00700204C2F002052
:103DC00010B504462146084801F042FD0748007836
:103DD000002805D1002C03D032210548FCF750FD06
:103DE0000248047010BD000001030000EE00002036
:103DF00050C300000020244909684870AA202249C5
:103E00000968887000202049096848621E490968CD
:103E100008711D49096848711B49096888711A4968
:103E20000968C871184909680872174909688872D1
:103E300015490968C8721449096808732420124991
:103E4000096848731049096888730F490968C8737D
:103E500000200D49096808740B49096848740A492B
:103E60000968887408490968C8740749096848617D
:103E7000002105480068816103480068C16102486B
:103E80000068016270470000E007002010B50A7862
:103E90000D4B1860034628330C4C236024235343F6
:103EA000044628341B190A4C23600A4C4B68636093
:103EB0008B68A360CB68E3604B6963610B69236126
:103EC0000B78237010BD0000E0070020D807002009
:103ED000DC0700204C2F002007480068C078062827
:103EE00008D105480068007A002803D10120024962
:103EF0000968087270470000E007002010B504460A
:103F0000012C09D1FF2220210020FFF7F5FB012120
:103F1000084604F0AFF908E0002220211046FFF720
:103F2000EBFB0021012004F0A5F910BD10B5002421
:103F3000032000F073FB002801D0012400E00024DE
:103F4000204610BD10B50446032C0ED1FF221521CA
:103F50000020FFF7D1FB002214211046FFF7CCFB15
:103F600001210E2004F086F939E0022C1CD1FCF767
:103F7000A5FF002809D0FF2214210020FFF7BCFB79
:103F800001210E2004F076F908E0002214211046E9
:103F9000FFF7B2FB00210E2004F06CF9002215217E
:103FA0001046FFF7A9FB1AE0012C0ED1FF221421C5
:103FB0000020FFF7A1FB01210E2004F05BF9002295
:103FC00015211046FFF798FB09E000221521104645
:103FD000FFF792FB002214211046FFF78DFB10BD66
:103FE00010B50024F8F7F0FC094988420DD3FCF71E
:103FF000C1FF002807D1FCF751FE012801DD032491
:1040000004E0022402E0022400E00124204610BD66
:10401000B80B000010B50446012C09D1FF221D2168
:104020000020FFF769FB0121002004F023F908E0DC
:1040300000221D211046FFF75FFB0021084604F017
:1040400019F910BD10B50024022000F0E7FA00288D
:1040500001D0012400E00024204610BD10B5044624
:10406000012C09D1FF221E210020FFF745FB012171
:10407000092004F0FFF808E000221E211046FFF797
:104080003BFB0021092004F0F5F810BD70B50024B9
:1040900000250026FCF7BAFC0546FCF7C3FC0646E3
:1040A00002210848F7F72AF8552800D108E0012E28
:1040B00001D1002404E0012D01D1012400E00024FD
:1040C000204670BD6008002010B50446012C09D1BF
:1040D000FF221F210020FFF70FFB0121082004F021
:1040E000C9F808E000221F211046FFF705FB002158
:1040F000082004F0BFF810BD70B500240025FCF7BF
:104100000FFD054603211A48F6F7F8FF552806D19A
:1041100001201849088000201749088023E016482C
:104120000088012811D114490880FCF713FC762877
:1041300003DA01200F49088015E0FCF70BFC782812
:1041400011DB00200B4908800DE001200A4908809E
:10415000FCF700FC762803DA01200649088002E01B
:1041600000200449088003480488204670BD0000F0
:10417000600800200A0100200C01002010B5044650
:10418000012C09D1FF2221210020FFF7B5FA0121DE
:10419000072004F06FF808E0002221211046FFF705
:1041A000ABFA0021072004F065F810BD10B500241B
:1041B000FCF7CCFF012801D1012400E000242046B7
:1041C00010BD10B50446012C09D1FF221621002094
:1041D000FFF792FA0121032004F04CF808E00022D6
:1041E00016211046FFF788FA0021032004F042F858
:1041F00010BD10B50024052000F010FA002801D0F1
:10420000012400E00024204610BD10B50446012C16
:1042100009D1FF2219210020FFF76EFA01210520A4
:1042200004F028F83CE0022C17D1FCF747FE0028E8
:1042300009D0FF2219210020FFF75EFA0121052095
:1042400004F018F82CE0002219211046FFF754FA68
:104250000021052004F00EF822E0032C17D1FCF712
:1042600033FE002809D0FF2219210020FFF744FA6D
:104270000121052003F0FEFF12E000221921104663
:10428000FFF73AFA0021052003F0F4FF08E00022CE
:1042900019211046FFF730FA0021052003F0EAFF4C
:1042A00010BD000010B50024FCF722FD012839D113
:1042B00004214048F6F722FF552803D101203E494A
:1042C000087032E0FCF7BAFB01280BD0FCF7B6FB14
:1042D000022807D0FCF7B2FB032803D0FCF7AEFBA3
:1042E000052803D10120344908701EE0FCF7A6FB25
:1042F000042803D102203049087016E0FCF79EFB29
:10430000062803D103202C4908700EE0FCF796FB29
:10431000002803D0FCF792FB072806D1002026498D
:10432000087002E000202449087024480078022820
:1043300013D123480078002807D1FCF7BFFD0028DF
:1043400003D01D4800781D490870FCF7B7FD1C49D3
:104350000870FCF7B3FD044616E0184800780328FF
:1043600012D117480078002807D1FCF7ADFD0028CE
:1043700003D01148007811490870FCF7A5FD1049D9
:104380000870FCF7A1FD04460C48007802280ED006
:104390000A48007803280AD00748007807490870BF
:1043A00008460078002801D0012400E000242046BF
:1043B00010BD0000600800200E0100200F01002049
:1043C0001001002010B50446012C0ED1FF221B2144
:1043D0000020FFF791F900221A211046FFF78CF90F
:1043E00001210A2003F046FF1EE0022C0ED1FF221D
:1043F0001A210020FFF780F900221B211046FFF749
:104400007BF901210A2003F035FF0DE000221A217B
:104410001046FFF771F900221B211046FFF76CF9D7
:1044200000210A2003F026FF10BD000010B5002473
:1044300010480078012801D1012418E0FCF74AFD5A
:10444000022803D0FCF74AFE02280FD1FCF714FE25
:10445000012809D1FCF744FD012803D0FCF744FEF4
:10446000012801D1012402E0022400E002242046B8
:1044700010BD0000ED00002010B5F8F7BFFA0446AB
:10448000204610BD10B5034B08220349034800F035
:1044900013F910BD79440100B41B020084280020E8
:1044A00070B506465C488068002804D05A49886880
:1044B0008047054600E000250024A6E056484168F4
:1044C0000C20604308184088A84207D05248416831
:1044D0000C2060430818408802287DD14E4841686E
:1044E0000C2060430818806800280CD04A494A68AC
:1044F0000C21614351188868804747490968E200E8
:104500008918487009E0444841680C206043095C00
:1045100041480068E200801841703F480068E100AF
:10452000401840783C490968E200895C88420FD015
:1045300039480068E1004018417837480068E200D7
:104540008154002034490968E200891848605AE023
:1045500031480068E100401841782F4842680C203B
:1045600060431018407881421FD12B480068E10059
:1045700040184168284842680C2060431018808821
:1045800081420BD824480068E10040184068801937
:1045900021490968E2008918486034E001201E4979
:1045A0000968E200891848802DE01B480068E10096
:1045B00040184168184842680C2060431018C088B1
:1045C00081420DD814480068E10040184068811904
:1045D00011480068E20000E009E08018416012E044
:1045E00000200D490968E200891848800BE000208E
:1045F00009490968E20089184880002106480068D6
:10460000E20080184160601C84B203488089A042A7
:1046100000DD53E770BD0000042F00200146064A6C
:1046200092898A4205DD044A1268CB00D21850886C
:1046300000E0002070470000042F0020002000BF91
:1046400014E00D494A680C21414351184988012959
:104650000AD10021084A1268C300D2185180064AC4
:104660001268C300D2185160411C88B2024989897E
:104670008142E6DC70470000042F0020002000BFCC
:1046800013E00C494A680C2141435118498800291C
:1046900009D1084A1268C300D2185180054A12682D
:1046A000C300D2185160411C88B2024989898142F5
:1046B000E7DC7047042F0020F0B504460020164DBB
:1046C000AB6069602C60AA8100BF1FE0124D6E686C
:1046D0000C254543755D104E3668C700F619757098
:1046E0000D4D6E680C254543755D0B4E3668C70051
:1046F000F5550025084E3668C700F6197580064E38
:104700003668C700F6197560451CA8B2024DAD8920
:104710008542DBDCF0BD0000042F002070B50546AB
:104720000E46002E05D031462846F3F70FFD04460D
:1047300000E02C46204670BD10B5FCF707FD0128AF
:1047400017D10C480078012813D00A4800780328B4
:104750000FD00948007800280BD1FCF711FC07495D
:10476000884202D108F075F803E07D20000108F0CE
:1047700077F810BDE1000020E00000208813000061
:1047800008B500200090012269460520F9F790FD48
:1047900005490098886000200449087004490870A1
:1047A0000449087008BD00004C280020E0000020EB
:1047B000E2000020E300002008B500200090012264
:1047C00069460520F9F774FD002002490871009838
:1047D000886008BD4C28002070B5049C2578914263
:1047E00016DD01280AD18D4206DAFF26F61AAE42FE
:1047F0000ED3EE18F5B20BE0154609E0022807D1FA
:10480000954204DD9D4203DBEE1AF5B200E00D4651
:10481000257070BD0D4A4168516081699161C16820
:10482000D160416A5162016A116201681160416997
:10483000516181689160C169D16101691161816AC9
:1048400091620021024A117070470000202F002061
:10485000D407002010B5FFF7F1FEF7F715FF002190
:104860000148F6F755FD10BD6C08002010B5F7F7AC
:104870000BFFFFF703FF0AF0C5F80AF061F9FBF739
:104880001FFBFAF751F8FFF77BFFF8F7E9FBF6F7A4
:104890003BFBF9F7E5F855210548F6F739FDF8F740
:1048A00065F9F9F757F8FAF7CBFFF6F727FD10BDD2
:1048B0006C0800201CB500203349087008F0C6F8C9
:1048C0000020FCF78FFC0CF0DFFBF7F7A3F8F6F7FE
:1048D00015FD55212D48F6F71BFDF9F7F9F8F8F706
:1048E00045F9F9F737F8F5F72BFFF6F7A9F9E120C5
:1048F00040020CF00BF800F071FAF6F705FB08F037
:1049000085FAF7F7C1FEF9F755FEF8F739FCF8F725
:10491000B3FBFFF7B7FDFEF701F8FFF79DF8FFF7D0
:10492000C3F9F9F74DFDFBF7F7FAF9F7FDFF184A60
:10493000FF21913101200AF0C9F90022114601201E
:104940000AF008F907F0F0FF0AF042F80AF0F8F868
:10495000FFF732FF00200F4988714871087101206C
:10496000887048701420087007226846F3F785FCA9
:104970000199009800F0BCFF0221012000F094FE94
:10498000FAF75EFF1CBD0000ED0000206C0800205F
:104990000090D003FE0000207047000010B50446D0
:1049A000552C03D105494869804702E0034908684E
:1049B000804700200249087010BD0000202F002011
:1049C000D407002010B54648007803000CF034F8F6
:1049D0000A06111B26303B465051738141484068FE
:1049E000002802D03F494868804701203C490870B0
:1049F00000BF3C488068002804D03A498868804756
:104A00003749087069E03748C068002802D0354946
:104A1000C868804703203249087000BF31480069E8
:104A2000002804D02F49086980472D49087054E0B8
:104A30002C484069002802D02A4948698047002054
:104A40002749087049E027488069002802D0254995
:104A50008869804706202249087000BF2148C06944
:104A6000002804D01F49C86980471D49087034E0F8
:104A700000BF1B48007807280AD11A48006A00289E
:104A800002D01849086A804709201549087011E0CA
:104A90001348007808280AD11248406A002802D03A
:104AA0001049486A804709200D49087002E000203B
:104AB0000B49087000BF0A480078002808D0094850
:104AC000806A002804D00749886A80470449087032
:104AD00003E000200249087000BF00BF10BD0000C5
:104AE000D4070020202F00207047000010B50020C0
:104AF0000CF086FB09F064F809F0B8F809F0CEF87C
:104B000000F0C6FCF6F732F90220FCF76BFB002040
:104B100007490870FFF7C8F8FEF7EEFFFFF714F833
:104B2000F5F77EFF10200AF0E7FC00F0B1FD10BDA4
:104B3000A401002010B5012408F010FC012801D1C7
:104B4000052407E0F7F73AFF0349884201D2012420
:104B500000E00224204610BD204E000010B50624BF
:104B600008F0FCFB002800D1002408F0FDFB012820
:104B700003D008F0F9FB072800D90924204610BD0E
:104B800010B5F6F7F3F80022114601200AF014F9E7
:104B900000213C48F6F7BCFB00203B49088000247C
:104BA00000BF00F02FFF32217D200001FBF768FEDF
:104BB0000020364908700AE0002234480178104687
:104BC000FEF79AFD31480078401C304908702F48A4
:104BD00000782428F0DB00202D49087009E000212E
:104BE0002B48007809F0FCFC29480078401C284933
:104BF0000870274800780D28F1DBFEF7A5FFF5F7D0
:104C0000E5FD08F0FDFA23480078401C21490870B2
:104C100008460078052812D300200870FEF782FFAE
:104C20001D4800780A2805D300201B490870FFF7AB
:104C300053F904E018480078401C1749087008F040
:104C400093FB0128ADD908F08FFB0728A9D20020DB
:104C50000F49087008E00E48007809F0DBFC0C48AA
:104C60000078401C0A490870094800780D28F2DBDA
:104C7000F5F7E6FF55210348F6F74AFBF7F774FE10
:104C8000204610BD6C0800207A000020070100209B
:104C900005010020060100200801002010B50324B2
:104CA00008E000F0AFFE012000F0B6FD002801D0C2
:104CB000042400E0F5E700BF204610BD10B5002039
:104CC0002A49086007F0C2FE0120FCF78BFAF6F7CC
:104CD000A1FE55212648F6F71BFBF7F747FFF8F72B
:104CE00039FE0CF0D1F9F5F72BFDF9F72BFCF5F7B0
:104CF000A7FF08F095FAF9F75DFCF9F7F9FDF8F769
:104D00003FFAFFF7BFFBFDF709FEFFF7B7FCFFF720
:104D100037FDFEF7A1FEFEF7C7FF00F05FF8E120C8
:104D200040020BF0F3FDF6F7EFF8FBF7F5F8F9F7B3
:104D3000FBFD104AFF219131012009F0C7FF00223D
:104D40001146012009F006FF09F042FE09F0F8FEC5
:104D5000F8F786FE0221012000F0A6FCFAF770FDAC
:104D600007F004FEF6F7CAFA10BD00004C00002060
:104D70006C0800200090D00370B506460D4614461E
:104D80000E4806600E4805600E49206808600E490E
:104D9000606808600D49A06808600D4920690860D6
:104DA0000C49E06808600C496069086005480068C3
:104DB000002802D003480068804770BDA80000208A
:104DC000B0000020900000209400002098000020F7
:104DD0009C000020A0000020A400002000B587B0A7
:104DE0000C4801900C4802900C480390002004905D
:104DF00005900B48069000200A49086048600A495F
:104E00000860486001AA0121C9020848FFF7B4FF01
:104E100007B000BD314E0100D55101005D510100C8
:104E200089500100741200206C0A00207C170020B9
:104E300001207047F3B5C3B00446449E00200090A3
:104E400057E002E0641C761E00BF022E05D32078D6
:104E5000EB28F7D160789028F4D1072E00D24AE0F1
:104E6000A778FD1CB54200D945E0A81E205C0002D1
:104E7000691E615C08434290042D38D9291FA01C8B
:104E80000CF01CF94299884226D11D480068002880
:104E900004D0B91EE01C1A4A1268904719480068ED
:104EA000002824D0E1786846017120798111684694
:104EB000417120798106890E68468171381FC1B21F
:104EC0006846C171C279611D02A8F3F7D6F901A83D
:104ED0000C49096888470AE00020009002E0009829
:104EE000401C00900098A842F9D30020009064195B
:104EF000761B072EA5D200BF4498801B45B0F0BD9D
:104F00009C000020A4000020F7B5C0B01546002684
:104F10000027E81DFF210131884202DD002043B057
:104F2000F0BDEB216846017090214170281DC1B28F
:104F3000684681700021C1704098C1B26846017115
:104F40000524002605E04198805D69460855641CEB
:104F5000761CAE42F7DBA11E00A802300CF0AEF8C2
:104F60000746381269460855641C0F55641C0648EC
:104F70000068002805D021466846034A1268904719
:104F8000CDE70020CBE700009400002070B500249E
:104F9000002500261B4840681A490968884200D14C
:104FA00070BD1848406817490968884205D91548F6
:104FB000406814490968451A07E012480068114919
:104FC0004968401A012189020D1AFF2D01D9FF26D7
:104FD00000E02E4600240DE00A4801680830405CDD
:104FE0000949085507480088401C8005800D05497F
:104FF0000860641CB442EFD3B1B203480BF0E2FC8A
:1050000000BFCDE7741200207C16002070B500258B
:105010001A480068002830D0194A1288FF2301334B
:10502000991A184A1268164B1B88D018134A12682E
:1050300090470546002D20D011480088401910499E
:105040000880084601880F480068FFF7F3FE044611
:10505000002C0DDD0A480088844209DA08480088DF
:10506000021B08480068011906480068F3F705F9B3
:1050700003480088001B0249088070BD980000208A
:10508000AC000020A800002038B5044600200090A5
:10509000A07810280CD120792D4908700846007896
:1050A000012853D1002211462020FFF72DFF4DE0AB
:1050B000A078122803D120792549087246E0A0780B
:1050C000052803D12079224988723FE0A078022880
:1050D0001DD120791E4948720846407A012806D120
:1050E0000090012269460420FFF70EFF2EE01848C9
:1050F000407A02282AD100BFBFF34F8F15481649C6
:10510000C860BFF34F8F00BF00BF00BFFDE7A078AE
:1051100001281BD12079332803D101200C49487084
:1051200005E02079352802D10020094948706079CE
:1051300007498870607A0006217A09040843E179FA
:1051400009020843A17908430149486038BD0000BD
:10515000600A00200400FA0500ED00E070B5034687
:105160000022002400251A484068194E3668B042D3
:1051700001D1002070BD16484068154E3668B04217
:1051800005D913484068124E3668841B07E0104862
:1051900000680F4E7668801B0126F602341AA14281
:1051A00001D9254600E00D4600220CE008480668BB
:1051B0000830805D985406480088401C4005400D2A
:1051C000034E3060521CAA42F0D32846D2E70000BA
:1051D0006C0A002070B50346002200241548406880
:1051E000144D2D68A84208D312484068114D2D680F
:1051F000401B0125AD022C1A04E00E4800680D4D3D
:105200006D68441BA14201D9012070BD00220CE051
:105210009D5C084846680830855508388088401CE1
:105220008005800D034D6860521C8A42F0D3002037
:10523000EBE700007412002010B50248FFF7EAFA0D
:1052400010BD00009C1C02000021014A117570472E
:1052500040600040014600BFF020084000110A23D2
:10526000584302460807000F8018C0B27047014635
:10527000002204E0501CC2B208460A38C1B20A2912
:10528000F8DA1007000E08437047000010B5044616
:1052900001218020F6F7BEF8607A012805D1424846
:1052A000C078102108434049C870607AA22805D10F
:1052B0003E48007F802108433C490877607A3B499B
:1052C000087700203A4948770846407F217808430C
:1052D00037494877E07B002805D00846407F2021E9
:1052E0000843334948773248407FC008C000A17A5C
:1052F00008432F4948770846807FF72108402C490A
:105300008877E078FFF7B3FF29498874A078FFF722
:10531000AEFF2749C8746078FFF7A9FF24490875D4
:105320002078002805D10846007D217908432049CE
:105330000875E079FFF79BFF1D4988756079FFF7D5
:1053400096FF1B494875A079FFF791FF1849C8756A
:10535000207AFFF78CFF164908760846807F4006C2
:10536000400E8877E07A002806D00846807F4021EA
:1053700008430F49887703E00D48807F0C49887700
:10538000A07BFFF774FF0A498876607BFFF76FFF09
:105390000749C876207B08770846807F102188431C
:1053A0000349887710BD00002004024060040440D7
:1053B000404F044010B504461B48807F012108433C
:1053C000194988772078FFF752FF174908756078E8
:1053D000FFF74DFF1449C874A078FFF748FF124942
:1053E000887420780C2806DD0846407F0821084391
:1053F0000D49487709E00C48407F0B49487708463B
:10540000007DE1780843084908750748807F400817
:1054100040000549887700BF0348807F022108408B
:105420000028F9D110BD0000404F044010B5002005
:105430001449087616200BF025FB0021124801764E
:105440001248407F80210843104948770846807FF2
:10545000012108430D49887700BF0C48807F022155
:1054600008400028F9D00948807F400840000749DB
:10547000887700BF0548807F022108400028F9D1C5
:1054800010BD00004060004040610040404F0440BB
:1054900010B500200749087000212020F5F7BAFF59
:1054A00001210548017500200449087515200BF0FD
:1054B000D1FA10BD005004404061004040600040FF
:1054C00070B504460D46002C14D0002D12D0042DCA
:1054D00010D800F013F800280CD1002608E0064987
:1054E000885D22460121F3F747FFA41C701CC6B259
:1054F000AE42F4DB70BD0000181C0200002005491C
:10550000897DC907C90F002901D0012000E00020D2
:10551000704700000050044030B585B005460C4689
:10552000002003900490009001900290072C0BDC67
:105530000120A04081B2684681810121C17303A985
:105540000220FAF731FE3EE0082C01D0092C0BD1E5
:105550000120A04081B2684681810121C17303A965
:105560000120FAF721FE2EE00A2C03D00B2C01D0EB
:105570000D2C0BD10120A04081B268468181012110
:10558000C17303A90020FAF70FFE1CE00C2C01D018
:105590000F2C0BD10120A04081B2684681810121EE
:1055A000C17303A90E20FAF7FFFD0CE00E2C0AD1FF
:1055B0000120A04081B2684681810121C17303A905
:1055C0000C20FAF7F1FD002168460170C1704170AE
:1055D0000121817000210171C1720D218172FF21B1
:1055E000017200214172F3F727FF03491520FDF7EF
:1055F0005FF805B030BD00004952010010B5002031
:105600001049087515200BF025FA00210E48017588
:105610001520002809DB00BF00BFC206D20E012101
:1056200091400A4A116000BF00BF00BF084880795E
:105630008011032805D006480078802108430449DA
:10564000087010BD406000404061004000E100E093
:105650000050044010B5F3F7E9FF10BD10B5012369
:105660001A4600211846F5F791FE01221146104610
:10567000F5F7F0FEF2F726FD03480BF0F7FC0248C1
:105680000249086010BD00000090D00358070020B8
:1056900000BF04480069042108430249086130BF83
:1056A00000BF704700ED00E0F3B585B0054600246B
:1056B00000270026002003900490EEB22804070E75
:1056C0000F2F54DA082E52DA002009E00C21414352
:1056D000284A515AA94201D1044603E0411CC8B2EC
:1056E0001728F3D300BF0120B04086B20C206043DE
:1056F00020494018C3780C20604340188278F8B2E3
:1057000031460190FAF7F4FD6846868101218173E4
:105710000021C17302214174F8B203A9FAF744FDD4
:105720000C216143134A8918C888FBF781FE0C20BD
:10573000604310494018C18868460181694606984F
:10574000887202A8FBF78EFD0C226243094BD21827
:1057500091680C226243D21804201056FCF7A8FF6F
:105760000C216143034A8918C888FBF7E5FD07B09F
:10577000F0BD0000341E0200FEB505460C460020B8
:10578000C0430290EFB22804060E0F2E42DA082F13
:1057900040DA0120B8406946088080202040002877
:1057A00016D101208870A007800F022801D148710E
:1057B00009E0A007800F012802D16946487102E084
:1057C000002069464871F0B26946FAF7EDFC1FE027
:1057D0000020694688700E202040002800D000BFBD
:1057E00010202040002802D16946087102E0012003
:1057F00069460871E007C00F002802D16946887128
:1058000002E0012069468871F0B26946FAF7CCFCE3
:10581000002002900298FEBD30B50146CAB20C04C9
:10582000230E00200F2B0FDA082A0DDA01249440F2
:10583000A2B2064C03252D026419E45C1440002C2E
:1058400001D0012000E0002030BD00000000044035
:10585000F8B504460F460020C0430090E6B220048D
:10586000050E0F2D11DA082E0FDA0120B04086B296
:10587000002F04D1E8B23146FAF792FD03E0E8B216
:105880003146FAF79DFD002000900098F8BD000019
:105890001649897F01221143144A917700BF1349A9
:1058A000897F022211400029F9D01049897C81703A
:1058B0000E49C97C41700D49097D01700B498A7DF3
:1058C0008271497D01710949CA7D42710A7EC271A6
:1058D000897F49084900054A917700BF0349897FBC
:1058E000022211400029F9D170470000404F0440C6
:1058F00003B585B000200190029003900490002130
:1059000068464173817E01A8C1706846417E01A846
:1059100081706846017E4171002101A80171082152
:1059200068460171817D01A8C1716846C17D4172DF
:10593000417D01A881716846017D01A801720021A5
:1059400068468173C17301A881730C2141734121A1
:10595000684601740021C17401A8FFF797FC1D205F
:105960000449888204491620FCF7A2FE00F006F8DC
:1059700007B000BD204F0440B911020010B5FFF779
:1059800055FD10BD70B504460D46601E0D49884298
:1059900000D90124002C00D1012440200A490870BC
:1059A000084600786043094948610321081F0BF04D
:1059B00081F80020054988610720086104480560D6
:1059C00070BD0000FFFFFF008001002000E000E04C
:1059D0007C0100200020C043002809DBC206D20E53
:1059E00001219140054A1160BFF34F8FBFF36F8FC4
:1059F00000BF0020024908618861704780E100E033
:105A000000E000E010B50AF0FBFF10BD1A200849C5
:105A100008722B2048723C2088724D20C8727F206B
:105A2000044909680860AC200349487070470000C9
:105A300000040240840100200010024010B51C4800
:105A40000078012812D11B480078642809DB022065
:105A500019494871087100201649087014490870E6
:105A600004E014480078401C12490870134800787C
:105A700001281CD112480078012804D100201049C7
:105A80000870104908700F48007832280ADBF7F7D1
:105A9000B5F800210C48F5F7EBFB55210B48F5F75D
:105AA00037FC04E007480078401C0649087010BD28
:105AB0002107002020070020100700201A070020DF
:105AC0001C0700201B070020600800206C08002035
:105AD000F8B504460D46002700200090032000037F
:105AE000204000130090102C04D0122C02D011483A
:105AF000844217D122202840222806D127073F0FB1
:105B000039460098F4F708FE06461220284012286D
:105B10000ED12007000F471C39460098F4F7FCFD12
:105B2000064605E02107090F0098F4F7F5FD064643
:105B30003046F8BD10100000F8B504460D460026AA
:105B400000270120000320400713102C04D0122C42
:105B500002D00F48844215D122202840222805D1A6
:105B60002607360F31463846FAF70EF8122028403D
:105B700012280CD12007000F461C31463846FAF790
:105B800003F804E02107090F3846F9F7FDFFF8BDD7
:105B900010100000FFB58BB01C4600200790069047
:105BA00005903848049010210B980840002801D037
:105BB000022707E040210B980840002801D0012768
:105BC00000E00027002C04D01498047001200890F5
:105BD00001E010200890002548E0002C08D0254660
:105BE0006000294A115A0C98F2F7B0FA079006E0C3
:105BF0006800254A115A0C98F2F7A8FA07903E4619
:105C000030E0711C0798F2F7A1FA400806900D9851
:105C1000F2F7F2FB03900D9A0699881AF2F7ECFB63
:105C200018490190F2F76DFB02900399F2F7A6FB79
:105C300005900598F2F7E7FB4900490803910290A7
:105C40000498F2F7E0FB4900490801910090039B9A
:105C5000029AF2F7EDFB03D20A9509960598049093
:105C6000701CC6B27F2ECCDD681CC5B20898854278
:105C7000B3DB14990A98087014990998487004982D
:105C80000FB0F0BD0000C842481F02000246412A82
:105C90002ED010DC212A2AD006DC102A45D0122A68
:105CA0004BD0202A59D11CE0222A26D0232A2AD0E0
:105CB000402A52D116E081235B01D01A9A4228D0A3
:105CC00008DC422A1AD0432A1ED025481018002882
:105CD00043D13AE0012822D020281BD021283CD1F2
:105CE0001EE000BF1F4803890B43038136E000BF5D
:105CF0001C4843890B43438130E000BF1948838926
:105D00000B4383812AE000BF1648C3890B43C3813C
:105D100024E000BF144883880B4383801EE000BF4B
:105D20001148C3880B43C38018E00E4843890B43D6
:105D3000438103890B43038110E00A48C3890B4365
:105D4000C38183890B43838108E00748C3880B43E1
:105D5000C38083880B43838000E000BF00BF70478F
:105D6000F0EFFFFF0011044000140440F0B50546B9
:105D70000E46412D30D010DC212D2CD006DC102D0C
:105D800051D0122D56D0202D62D11CE0222D2AD0C8
:105D9000232D30D0402D5BD116E081214901681AB6
:105DA0008D4230D008DC422D1ED0432D24D02A480D
:105DB000281800284CD144E001282CD0202823D0DA
:105DC000212845D128E000BF244F3888314600F013
:105DD00049F804463DE000BF204F7888314600F086
:105DE00041F8044635E000BF1C4FB888314600F04A
:105DF00039F804462DE000BF184FF888314600F00E
:105E000031F8044625E000BF154F3888314600F0D0
:105E100029F804461DE000BF114F7888314600F094
:105E200021F8044615E00D4F7888314600F01AF845
:105E300004460EE0094FF888314600F013F8044696
:105E400007E0074F7888314600F00CF8044600E080
:105E500000BF00BF2046F0BDF0EFFFFF001104407F
:105E6000001404400246002013460B40002B01D0D2
:105E7000012000E000207047FFB581B00E461746B4
:105E8000012F07D1F748407D00090001C01DF549E9
:105E9000487505E0F348407D00090001F149487567
:105EA000049801287ED10A210198F2F74FF905469E
:105EB000ED48445DE007C00F002807D0E948007CAA
:105EC00000090001C01DE749087405E0E548007CB1
:105ED00000090001E349087402202040002807D08F
:105EE000E048C07BF02188437030DE49C87305E08C
:105EF000DC48C07BF0218843DA49C8730420204085
:105F0000002807D0D748807C00090001C01DD54972
:105F1000887405E0D348807C00090001D149887469
:105F200008202040002807D0CE48407CF02188433C
:105F30007030CC49487405E0CA48407CF021884361
:105F4000C849487410202040002807D0C548407C2C
:105F500000090001C01DC349487405E0C148407CE8
:105F600000090001BF49487420202040002807D0C4
:105F7000BC48007CF02188437030BA49087405E0C1
:105F8000B848007CF0218843B6490874402020407E
:105F9000002808D0B348807CF02188437030B14994
:105FA000887406E08BE0AF48807CF0218843AD49DF
:105FB00088740A210198F2F7C9F80D46AA48445D91
:105FC000E007C00F002807D0A648807BF021884357
:105FD0007030A449887305E0A248807BF021884393
:105FE000A049887302202040002807D09D48807B6C
:105FF00000090001C01D9B49887305E09948807B1A
:10600000000900019749887304202040002807D028
:106010009448007DF021884370309249087505E06E
:106020009048007DF02188438E4908750820204063
:10603000002807D08B48007D00090001C01D894958
:10604000087505E08748007D00090001854908754D
:1060500010202040002807D08248C07CF0218843CF
:1060600070308049C87405E07E48C07CF0218843C8
:106070007C49C87420202040002807D07948C07B84
:1060800000090001C01D7749C87305E07548C07B51
:10609000000900017349C87340202040002807D040
:1060A0007048C07C00090001C01D6E49C87454E0EE
:1060B0006C48C07C000900016A49C8744DE0694819
:1060C000007C00090001674908740846C07BF02184
:1060D00088436449C8730846807C000900018874BD
:1060E0000846407CF02188435E4948740846407C5D
:1060F0000009000148740846007CF0218843594992
:1061000008740846807CF021884356498874084604
:10611000807BF0218843534988730846807B0009BF
:10612000000188730846007DF02188434D490875B9
:106130000846007D0009000108750846C07CF02172
:1061400088434849C8740846C07B00090001C873E9
:106150000846C07C00090001C8740A9801287DD156
:106160000A213046F1F7F2FF05463F48445DE0075B
:10617000C00F002807D03B48407B00090001C01D2C
:106180003849487305E03748407B0009000135492C
:10619000487302202040002807D03248007BF021BD
:1061A000884370302F49087305E02E48007BF021AA
:1061B00088432C49087304202040002807D0294830
:1061C000807DF021884370302649887505E0254898
:1061D000807DF021884323498875082020400028CD
:1061E00007D02048807D00090001C01D1D49887529
:1061F00005E01C48807D000900011A4988751020BF
:106200002040002807D01748407DF0218843703097
:106210001449487505E01348407DF0218843114931
:10622000487520202040002807D00E48407BF021F0
:10623000884370300B49487305E00A48407BF021E1
:106240008843084948734020204000280ED0054864
:10625000C07D00090001C01D024900E092E0C87540
:106260000AE000005C2600206C1902006D48C07D29
:10627000000900016B49C8750A213046F1F766FF35
:106280000D466948445DE007C00F002807D0654807
:10629000C07AF021884370306249C87205E06148D5
:1062A000C07AF02188435F49C8720220204000284C
:1062B00007D05C48C07A00090001C01D5949C87266
:1062C00005E05848C07A000900015649C872042008
:1062D0002040002807D05348407E00090001C01D1F
:1062E0005049487605E04F48407E000900014D497D
:1062F000487608202040002807D04A48007EF02138
:10630000884370304749087605E04648007EF02112
:1063100088434449087610202040002807D041488F
:10632000007E00090001C01D3E49087605E03D4899
:10633000007E000900013B4908762020204000280B
:1063400007D03848007B00090001C01D354908739B
:1063500005E03448007B0009000132490873402001
:106360002040002807D02F48C07DF021884370309E
:106370002C49C87554E02B48C07DF0218843294939
:10638000C8754DE02748407B000900012549487346
:106390000846007BF0218843224908730846807D27
:1063A000F02188431F4988750846807D0009000157
:1063B00088750846407DF02188431A49487508468B
:1063C000407BF0218843174948730846C07D000987
:1063D0000001C8750846C07AF02188431149C87287
:1063E0000846C07A00090001C8720846407E0009CC
:1063F000000148760846007EF02188430949087666
:106400000846007E0009000108760846007B000966
:10641000000108730846C07DF02188430149C87512
:1064200005B0F0BD5C2600206C190200FFB581B0FC
:106430000E461746019801287ED10498002826D1DF
:10644000FA480078012822D0F6F7BEFAF8498842C7
:106450001DD3FAF733FD00280DD0F648807DF021DA
:1064600088437030F34988750846C07C00090001F4
:10647000C01DC87418E0EF48807DF0218843ED49C5
:1064800088750846C07C00090001C8740CE0E94822
:10649000807DF02188437030E64988750846C07CCD
:1064A00000090001C01DC874E248C07CF021884387
:1064B0007030E049C8740846007EF021884370308F
:1064C000DC4908760846807D00090001401C88757B
:1064D0000846407DF02188431030D649487508466B
:1064E000407D00090001401C48750846007DF021F0
:1064F00088431030CF4908750846007D0009000127
:10650000401C087533000AF097FA062E261E140C5C
:10651000042FC848007D00090001C01DC549087549
:1065200000BFC448007DF02188437030C149087520
:1065300000BFC048407D00E0ADE100090001C01D82
:10654000BC49487500BFBB48407DF021884370308E
:10655000B849487500BFB748807D00090001C01DDB
:10656000B449887500BF00E000BF00BF0498002850
:106570005ED1AE48007801285AD0F6F725FAAC492A
:10658000884255D3AB48C07FF0218843A949C877DA
:106590000846807F0009000188770846407FF02187
:1065A0008843A44948770846007FF0218843A149E1
:1065B00008770846C07DF02188439E49C875084683
:1065C000C07F00090001C8770846807FF02188431A
:1065D000984988770846407F00090001C01D487728
:1065E0000846807EF0218843924988760846807E5E
:1065F0000009000188760846407E000900014876BF
:106600000846007E0009000108760846007F000960
:10661000000108770846C07EF02188438549C87686
:106620000846407EF0218843703082494876B8E1C0
:1066300064213846F1F78AFD0546012D07D17D48D2
:10664000C07FF021884370307A49C87705E07948E7
:10665000C07FF02188437749C8770A213846F1F78F
:1066600075FD0A210090F1F771FD0D46642F02D3EC
:106670007148445D01E07148445DE007C00F0028A7
:1066800007D06C48807F00090001C01D69498877E8
:1066900005E06848807F000900016649887702208C
:1066A0002040002807D06348407FF02188437030A5
:1066B0006049487705E05F48407FF02188435D49A5
:1066C000487704202040002807D05A48007FF02156
:1066D000884370305749087705E05648007FF0211D
:1066E00088435449087708202040002807D05148A3
:1066F000C07DF021884370304E49C87505E04D4893
:10670000C07DF02188434B49C875102020400028E7
:1067100007D04848C07F00090001C01D4549C8771F
:1067200005E04448C07F000900014249C8772020A5
:106730002040002807D03F48807FF02188437030F8
:106740003C49887705E03B48807FF0218843394900
:10675000887740202040002807D03648407F000935
:106760000001C01D3349487705E03248407F0009E9
:106770000001304948770A213846F1F7E7FC0D4619
:106780002D48445DE007C00F002807D02948807ECF
:10679000F021884370302749887605E02548807EBF
:1067A000F02188432349887602202040002807D022
:1067B0002048807E00090001C01D1E49887605E042
:1067C0001C48807E000900011A4988760420204078
:1067D000002807D01748407E00090001C01D154958
:1067E000487605E01348407E0009000111494876CB
:1067F00008202040002807D00E48007E0009000134
:10680000C01D0C49087605E00A48007E0009000119
:106810000849087610202040002811D00548007F44
:1068200000090001C01D034908770FE0ED000020BA
:10683000B80B0000302700206C1902007F190200FD
:106840005948007F0009000157490877202020405F
:10685000002807D05448C07EF02188437030524948
:10686000C87605E05048C07EF02188434E49C8767E
:1068700040202040002807D04B48407EF02188432C
:106880007030494948768CE04748407EF021884383
:106890004549487685E04448807D00090001424929
:1068A00088750846407DF02188433F494875084671
:1068B000407D0009000148750846007DF0218843AD
:1068C000394908750846007D000900010875084629
:1068D000C07C00090001C8740846807DF02188430F
:1068E000314988750846C07CF02188432E49C87418
:1068F0000846007EF02188432B4908760846C07F71
:10690000F02188432849C8770846807F00090001A4
:1069100088770846407FF021884323494877084616
:10692000007FF0218843204908770846C07DF02188
:1069300088431D49C8750846C07F00090001C87713
:106940000846807FF0218843174988770846407FB2
:106950000009000148770846807EF02188431249EB
:1069600088760846807E0009000188760846407EC9
:106970000009000148760846007E000900010876FB
:106980000846007F0009000108770846C07EF02114
:1069900088430549C8760846407EF021884302496D
:1069A000487605B0F0BD00003027002010B5014644
:1069B000002200200A0EFE4B985CC307DB0F002B61
:1069C00007D0FC4BDB7FF024A3437033F94CE37713
:1069D00005E0F84BDB7FF024A343F64CE37702237A
:1069E0000340002B07D0F34BDB7F1B091B01DB1D92
:1069F000F04CE37705E0EF4BDB7F1B091B01ED4C0F
:106A0000E37704230340002B07D0EA4B9B7F1B094D
:106A10001B01DB1DE74CA37705E0E64B9B7F1B09C1
:106A20001B01E44CA37708230340002B09D0E14B62
:106A300020335B781B091B01DB1DDE4C20346370A7
:106A400007E0DC4B20335B781B091B01D94C203459
:106A5000637010230340002B09D0D64B20331B78E2
:106A6000F024A3437033D34C2034237007E0D14B80
:106A700020331B78F024A343CE4C203423702023F2
:106A80000340002B09D0CB4B20331B781B091B0183
:106A9000DB1DC84C2034237007E0C64B20331B7825
:106AA0001B091B01C34C2034237040230340002BDF
:106AB00007D0C04B9B7FF024A3437033BD4CA3771A
:106AC00005E0BC4B9B7FF024A343BA4CA377FF2384
:106AD0001B040B401A0CB64B985CC307DB0F002B52
:106AE00007D0B44B1B7F1B091B01DB1DB14C237767
:106AF00005E0B04B1B7F1B091B01AE4C2377022323
:106B00000340002B07D0AB4BDB7EF024A343703354
:106B1000A84CE37605E0A74BDB7EF024A343A54C0D
:106B2000E37604230340002B07D0A24B9B7EF02486
:106B3000A34370339F4CA37605E09E4B9B7EF024CD
:106B4000A3439C4CA37608230340002B07D0994B0A
:106B50005B7FF024A3437033964C637705E0954B3D
:106B60005B7FF024A343934C637710230340002BF7
:106B700007D0904B5B7F1B091B01DB1D8D4C63779E
:106B800005E08C4B5B7F1B091B018A4C637720233C
:106B90000340002B07D0874B1B7FF024A3437033A7
:106BA000844C237705E0834B1B7FF024A343814C67
:106BB000237740230340002B07D07E4BDB7E1B094D
:106BC0001B01DB1D7B4CE37605E07A4BDB7E1B096A
:106BD0001B01784CE376FF231B020B401A0A744B0F
:106BE000985CC307DB0F002B07D0724B1B7EF02491
:106BF000A34370336F4C237605E06E4B1B7EF0246D
:106C0000A3436C4C237602230340002B07D0694B2F
:106C10001B7E1B091B01DB1D664C237605E0654BC3
:106C20001B7E1B091B01634C237604230340002BAE
:106C300007D0604BDB7D1B091B01DB1D5D4CE37541
:106C400005E05C4BDB7D1B091B015A4CE3750823F7
:106C50000340002B07D0574B9B7E1B091B01DB1DFC
:106C6000544CA37605E0534B9B7E1B091B01514CF2
:106C7000A37610230340002B07D04E4B5B7EF024FD
:106C8000A34370334B4C637605E04A4B5B7EF024A4
:106C9000A343484C637620230340002B07D0454B89
:106CA0005B7E1B091B01DB1D424C637605E0414BFB
:106CB0005B7E1B091B013F4C637640230340002B86
:106CC00007D03C4BDB7DF024A3437033394CE37594
:106CD00005E0384BDB7DF024A343364CE375CAB2A4
:106CE000334B985CC307DB0F002B07D0314B1B7D68
:106CF000F024A34370332F4C237505E02D4B1B7DEF
:106D0000F024A3432B4C237502230340002B07D010
:106D1000284B1B7D1B091B01DB1D264C237505E041
:106D2000244B1B7D1B091B01224C237504230340AC
:106D3000002B07D01F4BDB7C1B091B01DB1D1D4CEF
:106D4000E37405E01B4BDB7C1B091B01194CE3744E
:106D500008230340002B07D0164B9B7CF024A34351
:106D60007033144CA37405E0124B9B7CF024A343B6
:106D7000104CA37410230340002B07D00D4B5B7DF8
:106D8000F024A34370330B4C637505E0094B5B7D26
:106D9000F024A343074C637520230340002B0BD042
:106DA000044B5B7D1B091B01DB1D024C637509E075
:106DB0006C190200102700200C4B5B7D1B091B0186
:106DC0000A4C637540230340002B07D0074BDB7C44
:106DD000F024A3437033054CE37405E0034BDB7CE4
:106DE000F024A343014CE37410BD000010270020E1
:106DF00000B501287ED1FE4AD278F0239A43703242
:106E0000FB4BDA701A46127912091201D21D1A715F
:106E10001A461279F0239A437032F54B1A711A46CA
:106E2000527912091201D21D5A711A465279F02371
:106E30009A437032EE4B5A711A46D27912091201F6
:106E4000D21DDA711A46D279F0239A437032E84B98
:106E5000DA711A46527A12091201D21D5A721A4672
:106E6000527AF0239A437032E14B5A721A46927A60
:106E7000F0239A437032DE4B9A721A469278F023CE
:106E80009A437032DA4B9A701A46D27A120912017A
:106E9000D21DDA721A46527812091201D21D5A70A6
:106EA0001A46D27AF0239A437032D14BDA721A46DC
:106EB000203AD27FF0239A437032CD4B203BDA77D1
:106EC000CB4A127B12091201D21D20331A731A46C3
:106ED000203A927F12091201D21D203B9A77C44AB0
:106EE000127BF0239A437032C14B1A731A46203A30
:106EF000127F00E0F2E1F0239A437032BC4B203B5A
:106F00001A77BB4A527B12091201D21D20335A73E1
:106F10001A46203AD27E12091201D21D203BDA769F
:106F2000B44AD278F0239A437032B24BDA701A46E0
:106F3000127B12091201D21D1A731A461279120914
:106F40001201D21D1A711A46927AF0239A437032B6
:106F5000A84B9A721A461279F0239A437032A54BC5
:106F60001A711A46527912091201D21D5A711A4623
:106F7000927912091201D21D9A711A46127A1209D7
:106F80001201D21D1A721A46127AF0239A437032F5
:106F9000984B1A721A46527A12091201D21D5A726D
:106FA000934A927912091201521C914B9A711A4616
:106FB0009279F0239A4310328D4B9A711A46127AC5
:106FC00012091201521C1A721A46127AF0239A43BD
:106FD0001032874B1A721A46927A12091201521C09
:106FE0009A721A46D27812091201521CDA701A46A5
:106FF000927812091201521C9A701A465278F023A4
:107000009A4310327A4B5A701A461278F0239A43F8
:107010001032774B1A701A46127812091201521C5C
:107020001A701A46203AD27F12091201521C203BD4
:10703000DA771A46927FF0239A4310326C4B203B4A
:107040009A771A46527FF0239A431032684B203BBE
:107050005A771A46527F12091201521C5A771A4661
:10706000127F12091201521C1A771A46D27EF0239F
:107070009A4310325E4B203BDA761A46927EF0231A
:107080009A4310325A4B203B9A765A4A127BF0238D
:107090009A431032574B1A731A46D27AF0239A4306
:1070A0001032544BDA721A46D27A12091201521C6B
:1070B000DA721A46927A12091201521C9A721A4610
:1070C000527AF0239A4310324A4B5A721A46527936
:1070D000F0239A431032474B5A711A46D279F02363
:1070E0009A431032434BDA710B0009F0A5FC19F3F7
:1070F000E9DFD5CBC1B7ADA3998F87786E645A50BD
:10710000463E362E261E160EF5003A4AD279F02358
:107110009A437032374BDA7100BF364A5279F02306
:107120009A437032334B5A7100BF324A527AF0237D
:107130009A4370322F4B5A7200BF2E4A927A12092C
:107140001201D21D2B4B9A7200BF2A4AD27A120921
:107150001201D21D274BDA7200BF264AD27AF023E1
:107160009A437032234BDA7200BF224A127BF0231B
:107170009A4370321F4B1A7300BF1D4A203A927E09
:10718000F0239A4370321A4B203B9A7600BF184A7C
:10719000203AD27EF0239A437032154B203BDA76A8
:1071A00000BF134A203A127F12091201D21D104B60
:1071B000203B1A7700BF0E4A203A527F1209120173
:1071C000D21D0B4B203B5A7700BF094A203A527F11
:1071D000F0239A437032064B203B5A7700BF044A93
:1071E000203A927FF0239A437032014B203B03E018
:1071F0007C260020502700209A7700BFDC4AD27FEF
:1072000012091201D21DDA4BDA7700BFD84A2032B8
:10721000127812091201D21DD54B20331A7000BF0B
:10722000D34A20321278F0239A437032D04B203365
:107230001A7000BFCE4A20325278F0239A4370323F
:10724000CB4B20335A7000BFC94A203292781209C2
:107250001201D21DC64B20339A7000BFC44A20329F
:10726000D27812091201D21DC14B2033DA7000BF4F
:10727000BF4A2032927A12091201D21DBC4B203330
:107280009A7200BFBA4A2032127AF0239A437032BF
:10729000B74B20331A7200BFB54A2032127A120956
:1072A0001201D21DB24B20331A7200BFB04A2032F5
:1072B0009279F0239A437032AD4B20339A7100BF1C
:1072C000AB4A2032927912091201D21DA84B203309
:1072D0009A7100BF01E0FFE700BF47E1A44A2032F6
:1072E000D278F0239A43A24B2033DA701A461279EF
:1072F000120912011A711A461279F0239A439C4B13
:1073000020331A711A465279120912015A711A461B
:107310005279F0239A43964B20335A711A46D27908
:1073200012091201DA711A46D279F0239A43904B6E
:107330002033DA711A46527A120912015A721A4629
:10734000527AF0239A438A4B20335A721A46927A21
:10735000F0239A43864B20339A721A469278F02390
:107360009A43834B20339A701A46D27A120912013B
:10737000DA721A465278120912015A701A46D27AF3
:10738000F0239A437A4B2033DA72794AD27FF02382
:107390009A43774BDA771A462032127B1209120190
:1073A00020331A73724A927F12091201203B9A7796
:1073B0001A462032127BF0239A436D4B20331A7306
:1073C0006B4A127FF0239A43694B1A771A46203290
:1073D000527B1209120120335A73654AD27E120978
:1073E0001201203BDA76634AD278F0239A43614B4C
:1073F000DA701A46127B120912011A731A461279B0
:10740000120912011A711A46927AF0239A43594BC3
:107410009A721A461279F0239A43564B1A711A46F9
:107420005279120912015A711A46927912091201FF
:107430009A711A46127A120912011A721A46127AAF
:10744000F0239A434B4B1A721A46527A12091201D0
:107450005A72474A2032927912091201444B203362
:107460009A711A469279F0239A43414B20339A71CC
:107470001A46127A120912011A721A46127AF02367
:107480009A433B4B20331A721A46927A1209120120
:107490009A721A46D27812091201DA701A46927854
:1074A000120912019A701A465278F0239A43304B0F
:1074B00020335A701A461278F0239A432C4B20330B
:1074C0001A701A461278120912011A70284AD27FCD
:1074D00012091201203BDA771A46927FF0239A4371
:1074E000234B9A771A46527FF0239A43204B5A77C0
:1074F0001A46527F120912015A771A46127F120950
:1075000012011A771A46D27EF0239A43184BDA7684
:107510001A46927EF0239A43154B9A76154A127BAF
:10752000F0239A43134B1A731A46D27AF0239A43E4
:10753000104BDA721A46D27A12091201DA721A461E
:10754000927A120912019A721A46527AF0239A43D9
:10755000084B5A721A465279F0239A43054B5A71D6
:107560001A46D279F0239A43024BDA7100BD00002B
:107570005C26002050270020F7B582B0064617464B
:10758000002500200190002E7ED1F9F799FB0528F7
:107590005FD1F9F793FC00280DD0FA484079F0212B
:1075A00088437030F7494871084680780009000127
:1075B000C01D88700AE0F3484079F0218843F14902
:1075C000487108468078000900018870ED48C0794C
:1075D00000090001EB49C8710846807900090001E3
:1075E0008871084640790009000148710846007A10
:1075F000F0218843E34908720846007A0009000137
:1076000008720846C079F0218843DE49C8710846EF
:10761000C07800090001C87008468078F0218843CE
:10762000D849887008464078F0218843D549487089
:1076300008464078000900014870084600790009B2
:10764000000108710846C078F0218843CD49C87010
:1076500029E2CC484079F02188437030C94948710B
:107660000846807800090001C01D88700846C0796E
:1076700000090001C871084680790009000188717D
:1076800008464079000900E034E0000148710846EE
:10769000007AF0218843BB4908720846007A000945
:1076A000000108720846C079F0218843B549C871C5
:1076B0000846C07800090001C87008468078F021AB
:1076C0008843B049887008464078F0218843AD4926
:1076D0004870084640780009000148700846007963
:1076E0000009000108710846C078F0218843A549C7
:1076F000C870ADE7012E5FD1F9F7E0FB00280DD08F
:10770000A0484079F021884370309E49487108466E
:10771000807800090001C01D88700AE0994840790E
:10772000F021884397494871084680780009000194
:1077300088709448C079000900019249C8710846D0
:10774000807900090001887108464079000900012C
:1077500048710846007AF02188438A490872084631
:10776000007A0009000108720846C079F0218843B8
:107770008449C8710846C07800090001C8700846ED
:107780008078F02188437F49887008464078F0214E
:1077900088437C49487008464078000900014870D9
:1077A000084600790009000108710846C078F021F8
:1077B00088437449C870EAE3022E7DD1F9F780FA54
:1077C00005287AD1F9F77AFB002877D0012F76D1F6
:1077D0000A210398F0F7BAFC0546F9F78FFA00285A
:1077E00002D16948445D01E06848445DE007C00F8C
:1077F000002807D06348C07900090001C01D614915
:10780000C87105E05F48C079000900015D49C87191
:1078100002202040002807D05A4880790009000142
:10782000C01D5849887105E056488079000900015B
:107830005449887104202040002807D051484079DD
:1078400000090001C01D4F49487105E04D484079CD
:10785000000900014B49487108202040002807D04A
:107860004848007AF021884370304649087205E0A4
:107870004448007AF0218843424908721020204091
:10788000002807D03F48007A00090001C01D3D498B
:10789000087205E03B48007A000900013949087286
:1078A0002020204000280BD03648C079F0218843A2
:1078B00070303449C87109E0AEE242E1F4E0A4E07E
:1078C0003048C079F02188432E49C87140202040BB
:1078D000002807D02B484079F0218843703029498F
:1078E000487105E027484079F021884325494871CF
:1078F0000A210398F0F72AFC0D462348445DE0076F
:10790000C00F002807D01F48C07800090001C01D23
:107910001C49C87005E01B48C078000900011949DE
:10792000C87002202040002807D016488078F02137
:10793000884370301349887005E012488078F02140
:1079400088431049887004202040002807D00D4843
:107950004078F021884370300A49487005E00948B2
:107960004078F021884307494870082020400028CB
:107970000ED00448407800090001C01D014948703C
:107980000CE000009C2600206C1902007F19020008
:10799000FE48407800090001FC4948701020204052
:1079A000002807D0F948007900090001C01DF749F7
:1079B000087105E0F548007900090001F3490871F4
:1079C00020202040002807D0F048C078F0218843CC
:1079D0007030EE49C87005E0EC48C078F02188436B
:1079E000EA49C87040202040002807D0E748807846
:1079F00000090001C01DE5498870C8E2E3488078AD
:107A000000090001E1498870C1E2E0484079F021B5
:107A100088437030DD4948710846807800090001CC
:107A2000C01D88700846C07900090001C871084669
:107A30008079000900018871084640790009000139
:107A400048710846007AF0218843D04908720846F8
:107A5000007A0009000108720846C079F0218843C5
:107A6000CA49C8710846C07800090001C8700846B4
:107A70008078F0218843C549887008464078F02115
:107A80008843C249487008464078000900014870A0
:107A9000084600790009000108710846C078F02105
:107AA0008843BA49C87072E2B8484079F0218843E7
:107AB000B649487108468078000900018870084678
:107AC000C07900090001C8710846807900090001E9
:107AD0008871084640790009000148710846007A1B
:107AE000F0218843A94908720846007A000900017C
:107AF00008720846C079F0218843A449C871084635
:107B0000C07800090001C87008468078F0218843D9
:107B10009E49887008464078F02188439B49487008
:107B200008464078000900014870084600790009BD
:107B3000000108710846C078F02188439349C87055
:107B400025E2012F73D10A210398F0F7FFFA0546C9
:107B5000F9F7D4F8002802D18D48445D01E08D4842
:107B6000445DE007C00F002807D08848C0790009AD
:107B70000001C01D8549C87105E08448C07900092D
:107B800000018249C87102202040002807D07F48A8
:107B9000807900090001C01D7C49887105E07B489F
:107BA000807900090001794988710420204000286B
:107BB00007D07648407900090001C01D734948711B
:107BC00005E07248407900090001704948710820B9
:107BD0002040002807D06D48007AF021884370309B
:107BE0006A49087205E06948007AF02188436749CC
:107BF000087210202040002807D06448007A00094D
:107C00000001C01D6149087205E06048007A000962
:107C100000015E49087220202040002808D05B48FF
:107C2000C079F021884370305849C87106E09DE062
:107C30005648C079F02188435449C87140202040FB
:107C4000002807D051484079F021884370304F49CF
:107C5000487105E04D484079F02188434B4948710F
:107C60000A210398F0F772FA0D464948445DE0078F
:107C7000C00F002807D04548C07800090001C01D8A
:107C80004249C87005E04148C078000900013F49F9
:107C9000C87002202040002807D03C488078F0219E
:107CA000884370303949887005E038488078F02181
:107CB00088433649887004202040002807D0334884
:107CC0004078F021884370303049487005E02F48F3
:107CD0004078F02188432D49487008202040002832
:107CE00007D02A48407800090001C01D2749487084
:107CF00005E026484078000900012449487010201A
:107D00002040002807D02148007900090001C01D4B
:107D10001E49087105E01D480079000900011B4952
:107D2000087120202040002807D01848C078F02192
:107D3000884370301549C87005E01448C078F021B8
:107D400088431249C87040202040002807D00F48BF
:107D5000807800090001C01D0C49887017E10B48AC
:107D60008078000900010949887010E107484079CE
:107D7000F021884370300549487108468078000931
:107D80000001C01D88700846C07905E09C260020CF
:107D90006C1902007F19020000090001C871084631
:107DA00080790009000188710846407900090001C6
:107DB00048710846007AF0218843764908720846DF
:107DC000007A0009000108720846C079F021884352
:107DD0007049C8710846C07800090001C87008469B
:107DE0008078F02188436B49887008464078F021FC
:107DF0008843684948700846407800090001487087
:107E0000084600790009000108710846C078F02191
:107E100088436049C870BAE0032E9FD1F8F750FF3D
:107E200005285FD1F9F74AF800280DD05948407964
:107E3000F02188437030574948710846807800091E
:107E40000001C01D88700AE052484079F021884343
:107E500050494871084680780009000188704D48F3
:107E6000C079000900014B49C871084680790009B2
:107E700000018871084640790009000148710846F0
:107E8000007AF0218843434908720846007A0009C5
:107E9000000108720846C079F02188433D49C87145
:107EA0000846C07800090001C87008468078F021B3
:107EB00088433849887008464078F021884335491E
:107EC000487008464078000900014870084600796B
:107ED0000009000108710846C078F02188432D4947
:107EE000C87054E02B480079F0218843703029494C
:107EF000087108464079F02188437030254948715F
:107F00000846807800090001C01D88700846C079C5
:107F100000090001C87108468079000900018871D4
:107F2000084640790009000148710846007AF021AE
:107F30008843184908720846007A0009000108724F
:107F40000846C079F02188431249C8710846C078B4
:107F500000090001C87008468078F02188430D4967
:107F6000887008464078F02188430A4948700846DE
:107F700040780009000148700846007900090001B6
:107F800008710846C078F02188430249C87005B0DE
:107F9000F0BD00009C26002070B505460C46012D62
:107FA0007ED1B148407D00090001C01DAE49487531
:107FB0000846007DF02188431030AB49087508461B
:107FC000007D00090001401C08750846C07CF021B6
:107FD00088431030A449C8740846807CF021884347
:107FE0001030A14988740846807C00090001401CBB
:107FF0008874F8F7BFFF022803D0F8F7BBFF012809
:108000006CD19A480078012868D0F4F7DDFC9849D3
:10801000884263D3F8F752FF00282FD09248007DA2
:10802000F02188437030904908750846007D0009AA
:108030000001C01D08750846C07CF02188437030DF
:108040008949C8740846807CF0218843703086498D
:1080500088740846807C00090001C01D88740846A9
:10806000407DF021884370307F4948750846407C48
:10807000F021884370307C494874F4E07A48007DF0
:10808000F02188431030784908750846007D0009C2
:108090000001401C08750846C07CF021884300E0C0
:1080A000B4E010307049C8740846807CF0218843E1
:1080B00010306D4988740846807C00090001401C1E
:1080C00088740846407DF021884367494875084612
:1080D000407CF021884364494874C4E0F8F7DEFD31
:1080E000002824D1F4F770FC614988421FD3F8F7C7
:1080F000E5FE00280ED05C48407DF02188437030BA
:10810000594948750846407CF021884370305649EB
:1081100048741AE05448407DF0218843524948751C
:108120000846407CF02188434F4948740DE04E4892
:10813000407DF021884370304B4948750846407CAB
:10814000F0218843703048494874F8F7A7FD0128AA
:108150002AD146480078012826D0F4F735FC444956
:10816000884221D34048407DF021884370303E4909
:1081700048750846407CF021884370303A4948747D
:10818000F8F79CFE002807D03748007DF02188438F
:1081900070303549087566E03348007DF02188432A
:1081A0001030314908755EE0230008F045FC062CCC
:1081B000241C140C042D2C48807C00090001C01DD7
:1081C0002949887400BF2848807CF021884370309A
:1081D0002549887400BF2448C07CF0218843703052
:1081E0002149C87400BF2048007D00090001C01D5E
:1081F0001D49087500BF1C48007DF0218843703080
:108200001949087500BF00E000BF2CE01648407D0A
:10821000F0218843144948750846007DF0218843C1
:10822000114908750846007D0009000108750846D7
:10823000C07CF02188430C49C8740846807CF0213A
:108240008843094988740846807C000900018874C5
:108250000846407D0009000148750846407CF02131
:1082600088430149487470BD7C260020ED00002041
:10827000B80B000030B50246002901D1002000E013
:108280000720130008F0D8FB0F09141F2B374350A9
:108290005D67727C88929FA9B500574B5B7EF02486
:1082A000A3430401F0252C402343534C6376A1E003
:1082B000524B9B79F024A3430401F0252C40234327
:1082C0004E4CA37196E04D4B2033DB791B091B010B
:1082D0000407240F2343494C2034E3718AE0464BC2
:1082E0002033DB7C1B091B010407240F2343424C72
:1082F0002034E3747EE0404B40331B781B091B01A4
:108300000407240F23433C4C4034237072E03A4B63
:108310002033DB7FF024A3430401F0252C402343CA
:10832000354C2034E37765E0334B20335B7BF0241E
:10833000A3430401F0252C4023432F4C20346373C6
:1083400058E02E4B9B791B091B010407240F234384
:108350002A4CA3714EE0294B9B7CF024A3430401DB
:10836000F0252C402343254CA37443E0234BDB7EB4
:108370001B091B010407240F2343204CE37639E03B
:108380001D4B2033DB7F1B091B010407240F2343F4
:10839000194C2034E3772DE0174B9B7E1B091B0102
:1083A0000407240F2343144CA37623E0134B2033FC
:1083B0009B79F024A3430401F0252C4023430F4C68
:1083C0002034A37116E00D4BDB7D1B091B01040754
:1083D000240F2343094CE3750CE0074B20335B7CEF
:1083E0001B091B010407240F2343034C203463742F
:1083F00000E000BF00BF30BD5C2600203027002019
:10840000F7B582B00746154600260024FE480078DE
:10841000012804D0F4F7D8FAFC49884279D2FC4804
:10842000407CF02188437030F94948740846807CCC
:1084300000090001C01D88740846007D0009000184
:10844000C01D08750846007DF02188437030F04952
:1084500008750846807CF02188437030EC498874A8
:108460000846C07C00090001C01DC8740846C07CD5
:10847000F02188437030E649C8740846407C000902
:108480000001C01D48740846407D00090001C01D60
:1084900048750846407DF02188437030DC494875B6
:1084A0000846007CF02188437030D949087408469A
:1084B000007C00090001C01D08740846C07BF02143
:1084C00088437030D249C873FF220A210020FBF78D
:1084D00013F9FF2213210020FBF70EF9FF221121CF
:1084E0000020FBF709F9FF2212210020FBF704F915
:1084F000FF220E210020FBF7FFF8FF220F210020B2
:10850000FBF7FAF8FF2210210020FBF7F5F8F4E35F
:10851000FFE7039836283DD019DC08287ED007DC19
:10852000801E030008F088FA0635A8FCFBFAF97EE5
:10853000102874D006DC092872D00D2871D00E28BE
:1085400070D1FDE333286ED03428F9D170E13F2893
:108550006AD00FDC3738082864D243007B449B88FC
:108560005B009F448A009702FF025F005F00650383
:10857000CB0318004E287BD006DC402879D0412858
:1085800078D04D28DCD1BBE14F2874D05028D7D10A
:108590004FE100BF00BF9E48407CF02188439C49CA
:1085A00048740846807C0009000188740846007DF4
:1085B00000090001C01D08750846007DF0218843B0
:1085C0007030934908750846807CF02188439049B3
:1085D00088740846C07C00090001C01DC8740846A4
:1085E000C07CF02188438A49C8740846407C000951
:1085F000000148740846407D00090001487508469E
:10860000407DF0218843824948750846007CF0216E
:1086100088437F4908740846007C06E0A1E2FDE338
:1086200037E2D2E3FBE394E028E00009000108749C
:108630000846C07BF02188437549C873FF220A2190
:108640000020FBF759F8FF2213210020FBF754F814
:1086500000220E211046FBF74FF800220F21104692
:10866000FBF74AF8002210211046FBF745F877E2A5
:10867000ABE110E2DDE26DE000BF00BF6448407C8A
:10868000F0218843624948740846807C0009000153
:1086900088740846007D00090001C01D0875084661
:1086A000007DF02188437030594908750846807C68
:1086B000F0218843564988740846C07C00090001AF
:1086C000C8740846C07CF02188435149C8740846E4
:1086D000407C0009000148740846407D0009000103
:1086E000C01D48750846407DF021884348494875BB
:1086F0000846007CF0218843454908740846007C00
:108700000009000108740846C07BF02188434049F5
:10871000C873FF220A21002003E055E1EFE086E064
:1087200016E0FAF7E9FFFF2213210020FAF7E4FF31
:1087300000220E211046FAF7DFFF00220F2110461B
:10874000FAF7DAFF002210211046FAF7D5FF8EE77C
:1087500000BF00BF2E48407CF02188432C4948745C
:108760000846807C00090001C01D88740846007D11
:1087700000090001C01D08750846007DF0218843EE
:108780007030234908750846807CF021884370309A
:108790001F4988740846C07C00090001C874084657
:1087A000C07CF02188431A49C8740846407C0009FF
:1087B000000148740846407D0009000148750846DC
:1087C000407DF0218843124948750846007CF0211D
:1087D00088430F4908740846007C000900010874AA
:1087E0000846C07BF02188430949C873FF220A214B
:1087F0000020FAF781FFFF2213210020FAF77CFF07
:1088000000220E21104605E0ED000020B80B00000C
:108810009C260020FAF770FF00220F211046FAF77D
:108820006BFF002210211046FAF766FF1FE700BF1A
:1088300000BFFE48407CF0218843FC49487408464C
:10884000807C00090001C01D88740846007D000975
:108850000001C01D08750846007DF0218843703076
:10886000F24908750846807CF0218843EF498874F6
:108870000846C07C00090001C8740846C07CF0218D
:108880008843EA49C8740846407C00090001C01DBD
:1088900048740846407D0009000148750846407D3F
:1088A000F0218843E14948750846007CF02188435F
:1088B000DE4908740846007C000900010874084677
:1088C000C07BF0218843D949C873FF220A210020C8
:1088D000FAF712FFFF2213210020FAF70DFF002202
:1088E0000E211046FAF708FF00220F211046FAF772
:1088F00003FF002210211046FAF7FEFEF6E300BF48
:10890000CA48407CF0218843C84948740846807CA6
:108910000009000188740846007D000900010875FF
:108920000846007DF02188437030C049087508462C
:10893000807CF0218843BD4988740846C07C0009CA
:108940000001C8740846C07CF02188437030B749E4
:10895000C8740846407C0009000148740846407D00
:108960000009000148750846407DF0218843AF4961
:1089700048750846007CF0218843AC4908740846D5
:10898000007C0009000108740846C07BF021884380
:10899000A649C873FF220A210020FAF7ADFEFF2284
:1089A00013210020FAF7A8FE00220E211046FAF744
:1089B000A3FE00220F211046FAF79EFE002210218E
:1089C0001046FAF799FE91E300BF9848407CF021E9
:1089D0008843964948740846807C000900018874E1
:1089E0000846007D0009000108750846007DF02159
:1089F000884370308D4908750846807CF021884393
:108A00008A4988740846C07C00090001C874084679
:108A1000C07CF02188438549C8740846407C000921
:108A2000000148740846407D000900014875084669
:108A3000407DF021884370307C4948750846007CB1
:108A4000F0218843794908740846007C0009000138
:108A500008740846C07BF02188437449C873FF221C
:108A60000A210020FAF748FEFF2213210020FAF71E
:108A700043FE00220E211046FAF73EFE00220F218F
:108A80001046FAF739FE002210211046FAF734FE9C
:108A90002CE300BF00BF6548407CF0218843703064
:108AA000624948740846807C00090001C01D887432
:108AB0000846007D00090001C01D08750846007DBC
:108AC000F02188437030594908750846807CF021B0
:108AD0008843564988740846C07C00090001C87460
:108AE0000846C07CF02188435049C8740846407C41
:108AF0000009000148740846407D000900014875DE
:108B00000846407DF0218843484948750846007C66
:108B1000F0218843454908740846007C000900019B
:108B200008740846C07BF02188434049C873FF227F
:108B30000A210020FAF7E0FDFF2213210020FAF7B6
:108B4000DBFD00220E211046FAF7D6FD00220F2190
:108B50001046FAF7D1FD002210211046FAF7CCFD9D
:108B6000C4E200BF3148407CF02188432F4948745B
:108B70000846807C0009000188740846007D0009D1
:108B8000000108750846007DF021884370302749B0
:108B900008750846807CF02188432449887408467B
:108BA000C07C00090001C8740846C07CF0218843DD
:108BB00070301E49C8740846407C000900014874A2
:108BC0000846407D0009000148750846407DF021B7
:108BD0008843164948750846007CF02188431349AC
:108BE00008740846007C0009000108740846C07B30
:108BF000F02188430D49C873FF220A210020FAF7AB
:108C00007BFDFF2213210020FAF776FD00220E21C2
:108C10001046FAF771FD00220F211046FAF76CFD9D
:108C2000002210211046FAF767FD5FE29C26002023
:108C300000BFFC48407CF0218843FA49487408464C
:108C4000807C0009000188740846007D000900014D
:108C500008750846007DF02188437030F149087599
:108C60000846807CF0218843EE4988740846C07C21
:108C700000090001C8740846C07CF0218843E94916
:108C8000C8740846407C0009000148740846407DCD
:108C90000009000148750846407DF0218843703086
:108CA000E04948750846007CF0218843DD49087496
:108CB0000846007C0009000108740846C07BF021CA
:108CC0008843D849C873FF220A210020FAF714FD0F
:108CD000FF2213210020FAF70FFD00220E2110467B
:108CE000FAF70AFD00220F211046FAF705FD0022CF
:108CF00010211046FAF700FDF8E1F8E1C948407C80
:108D0000F02188437030C74948740846807C0009C8
:108D10000001C01D88740846007D00090001C01DC7
:108D200008750846007DF0218843BE49087508464D
:108D3000807CF0218843BB4988740846C07C00E0F1
:108D4000A9E000090001C8740846C07CF0218843EE
:108D5000B449C8740846407C0009000148740846BC
:108D6000407D0009000148750846407DF021884398
:108D7000AC4948750846007CF0218843A94908742D
:108D80000846007C0009000108740846C07BF021F9
:108D90008843A449C873FF220A210020FAF7ACFCDB
:108DA000FF2213210020FAF7A7FC00220E21104613
:108DB000FAF7A2FC00220F211046FAF79DFC0022D0
:108DC00010211046FAF798FC90E19648407CF0217B
:108DD0008843944948740846807C000900018874DF
:108DE0000846007D0009000108750846007DF02155
:108DF00088438C4908750846807CF021884389495E
:108E000088740846C07C00090001C8740846C07C0C
:108E1000F02188438349C874084601E09EE003E1DD
:108E2000407C0009000148740846407D00090001AB
:108E300048750846407DF02188437A4948750846C0
:108E4000007CF0218843774908740846007C0009BB
:108E5000000108740846C07BF021884370307149D6
:108E6000C87300220A211046FAF746FC002213219B
:108E70001046FAF741FCFF220E210020FAF73CFCD5
:108E800000220F211046FAF737FC0022102110466D
:108E9000FAF732FC2AE16348407CF02188436149BB
:108EA00048740846807C0009000188740846007DEB
:108EB0000009000108750846007DF02188435949E2
:108EC00008750846807CF021884356498874084616
:108ED000C07C00090001C8740846C07CF0218843AA
:108EE0005049C8740846407C00090001487408468F
:108EF000407D0009000148750846407DF021884307
:108F0000484948750846007CF02188434549087463
:108F10000846007C00090001C01D08740846C07B9B
:108F2000F02188433F49C87300220A211046FAF70E
:108F3000E3FB002213211046FAF7DEFB00220E218C
:108F40001046FAF7D9FBFF220F210020FAF7D4FBD5
:108F5000002210211046FAF7CFFBC7E03148407CD1
:108F6000F02188432F4948740846807C000900019D
:108F700088740846007D0009000108750846007DD8
:108F8000F0218843274908750846807CF0218843F2
:108F9000244988740846C07C00090001C87408464A
:108FA000C07CF02188431F49C8740846407C0009F2
:108FB000000148740846407D0009000148750846D4
:108FC000407DF0218843174948750846007CF02110
:108FD00088437030134908740846007C000900017A
:108FE00008740846C07BF02188430E49C8730022EC
:108FF0000A211046FAF780FB002213211046FAF7E7
:109000007BFB00220E211046FAF776FB00220F218F
:109010001046FAF771FBFF2210210020FAF76CFBD3
:1090200064E000009C260020FD48407CF02188433D
:10903000FB4948740846807C000900018874084692
:10904000007D0009000108750846007DF021884375
:10905000F34908750846807CF0218843F0498874FC
:109060000846C07C00090001C8740846C07CF02195
:109070008843EB49C8740846407C000900014874E5
:109080000846407D0009000148750846407DF021F2
:109090008843E34948750846007CF0218843E0494D
:1090A00008740846007C0009000108740846C07B6B
:1090B000F0218843DA49C87300220A211046FAF7E2
:1090C0001BFB002213211046FAF716FB00220E218B
:1090D0001046FAF711FB00220F211046FAF70CFB9D
:1090E000002210211046FAF707FB00BF00BF002F37
:1090F00003D0CC48007A002808D1F3F765FCCA49B0
:10910000884203D3C9480078012872D1FF22112177
:109110000020FAF7F1FAFF2212210020FAF7ECFA08
:10912000C2480078012804D0F3F74EFCBE498842BB
:1091300016D2BF48807BF02188437030BC498873C9
:10914000084640300078F02188437030B8494031FB
:1091500008700846007800090001C01D08702DE065
:109160007D20C000854214D2B148807BF021884325
:10917000AF498873084640300078F021884370304A
:10918000AB494031087008460078000900010870BA
:1091900014E0A748807BF02188437030A44988738D
:1091A000084640300078F0218843A14940310870DA
:1091B0000846007800090001C01D08707D20C0002D
:1091C000854205D201462846EEF7C0FF064604E078
:1091D00098492846EEF7BAFF0646944800780128D9
:1091E00004D0F3F7F1FB9049884203D29248845DA2
:1091F00002E0A0E29148845DE007C00F002809D09A
:109200008B484030C07800090001C01D88494031BA
:10921000C87007E086484030C078000900018449E2
:109220004031C87002202040002807D08048C07913
:1092300000090001C01D7E49C87105E07C48C07965
:10924000000900017A49C87104202040002807D095
:109250007748807900090001C01D7549887105E0D3
:109260007348807900090001714988710820204005
:10927000002807D06E484079F021884370306C494F
:10928000487105E06A484079F0218843684948718F
:1092900010202040002807D06548407900090001CF
:1092A000C01D6349487105E061484079000900012B
:1092B0005F49487120202040002807D05C48007991
:1092C000F021884370305A49087105E05848007908
:1092D000F02188435649087140202040002807D0DB
:1092E00053488079F021884370305149887105E0F6
:1092F0004F488079F02188434D4988717D20C00016
:10930000854213D264212846EEF720FF06464748DF
:109310000078012804D0F3F757FB4349884202D272
:109320004548845D23E04548845D20E0642128466B
:109330003230EEF70BFF7D21C9000090EEF706FFFB
:10934000019164210198EEF701FF06463C488542F1
:1093500008D236480078012804D0F3F735FB3249AB
:10936000884202D23448845D01E03448845DE007DD
:10937000C00F002809D02E4840308078F021884363
:1093800070302B494031887007E0294840308078A0
:10939000F02188432649403188700220204000286F
:1093A00007D02348807A00090001C01D2049887237
:1093B00005E01F48807A000900011D4988720420D9
:1093C0002040002807D01A48407A00090001C01D3B
:1093D0001749487205E01648407A0009000114490F
:1093E000487208202040002807D01148007AF02158
:1093F000884370300E49087205E00D48007AF0216C
:1094000088430B4908721020204000281AD00848D1
:10941000007A00090001C01D0549087218E000002B
:109420009C260020600A0020B80B0000ED00002000
:1094300010270020A08601006C1902007F1902008D
:1094400010270000FE48007A00090001FC4908725C
:1094500020202040002807D0F948C079F021884317
:109460007030F749C87105E0F548C079F0218843AC
:10947000F349C87140202040002807D0F048407AC6
:10948000F02188437030EE49487205E0EC48407A9C
:10949000F0218843EA4948727D20C000854219D2F4
:1094A0000A212846EEF752FE0A210190EEF74EFE01
:1094B0000E460A2D08D2E3480078012804D0F3F7BD
:1094C00083FAE149884202D2E048845D12E0E04834
:1094D000845D0FE0642128463230EEF737FE0A2122
:1094E0000090EEF733FE0A210190EEF72FFE0E46B4
:1094F000D6498C5DE007C00F002809D0D048403025
:10950000807800090001C01DCD494031887007E016
:10951000CB484030807800090001C949403188704B
:1095200002202040002807D0C548807B00090001A8
:10953000C01DC349887305E0C148807B0009000154
:10954000BF49887304202040002807D0BC48407BD6
:1095500000090001C01DBA49487305E0B848407BC6
:1095600000090001B649487308202040002807D0B0
:10957000B348007BF02188437030B149087305E09F
:10958000AF48007BF0218843AD490873102020408C
:10959000002807D0AA48C07A00090001C01DA849C8
:1095A000C87205E0A648C07A00090001A449C87243
:1095B00020202040002807D0A148807AF02188434D
:1095C00070309F49887205E09D48807AF021884379
:1095D0009B49887240202040002807D09848407B53
:1095E000F021884370309649487305E09448407BE9
:1095F000F0218843924948737D20C000854207D2FC
:109600000A212846EEF7A2FD0E469048845D0BE045
:10961000642128463230EEF799FD0A210190EEF7D9
:1096200095FD0E4689498C5DE007C00F002809D0E2
:10963000834840304078F021884370308049403181
:10964000487007E07E4840304078F02188437C49EC
:109650004031487002202040002809D0784840302E
:10966000407800090001C01D75494031487007E08D
:10967000734840304078000900017149403148701A
:1096800004202040002807D06D48007CF02188434A
:1096900070306B49087405E06948007CF02188430C
:1096A0006749087408202040002807D06448007CDF
:1096B00000090001C01D6249087405E06048007C93
:1096C000000900015E49087410202040002807D0DE
:1096D0005B48C07BF021884370305949C87305E06E
:1096E0005748C07BF02188435549C873202020404B
:1096F000002807D05248C07B00090001C01D504916
:10970000C87305E04E48C07B000900014C49C8738E
:1097100040202040002807D04948407C0009000133
:10972000C01D47494874ECE04548407C00090001F1
:1097300043494874E5E000220A211046F9F7DCFFAE
:10974000002213211046F9F7D7FF002211211046FD
:10975000F9F7D2FF002212211046F9F7CDFF0022BF
:109760000E211046F9F7C8FF00220F211046F9F725
:10977000C3FF002210211046F9F7BEFF30484030E9
:10978000C078000900012E494031C8702C48C079CA
:10979000000900014039C8710846807900090001BC
:1097A000887108464079F021884325494871084668
:1097B000407900090001487108460079F02188438A
:1097C0001F49087108468079F02188431C49887137
:1097D000084640308078F02188431949403188702C
:1097E0001748807A00090001403988720846407A9B
:1097F0000009000148720846007AF02188431049A8
:1098000008720846007A0009000108720846C0790B
:10981000F02188430A49C8710846407AF0218843FC
:1098200007494872084640308078000900014031FD
:1098300088700348807B000900014039887309E083
:1098400010270020ED000020B80B00006C1902006A
:109850007F1902000846407B000900014873084652
:10986000007BF0218843284908730846C07A000924
:109870000001C8720846807AF02188432249887224
:109880000846407BF02188431F4948730846403012
:109890004078F02188431C494031487008464078A0
:1098A0000009000148701848007CF02188431649DF
:1098B00008740846007C0009000108740846C07B53
:1098C000F02188431049C8730846C07B0009000195
:1098D000C8730846407C0009000148740846807B34
:1098E000F021884308498873084640300078F02109
:1098F0008843054940310870084600780009000196
:10990000087005B0F0BD000010270020F7B582B048
:1099100007460E460121FF200830FBF799FF012181
:10992000FC48FBF795FFFC48007801287ED0F3F750
:109930004BF8FA49884279D3F7F7C2F9032843D1A3
:10994000F7F7B8F9002803D0F7F7B4F901283BD1AD
:10995000002F1CD1F7F7B2FA00280CD0F048407C59
:10996000F0218843EE4948740846807C00090001D4
:10997000C01D8874EEE0EA48407CF0218843E84945
:1099800048740846807C000900018874E2E0F7F71B
:1099900095FA00280CD0E248407CF02188437030D2
:1099A000DF4948740846807C000900018874D1E0D2
:1099B000DB48407CF0218843D94948740846807CC4
:1099C000000900018874C5E0F7F774F9002803D096
:1099D000F7F770F9012865D1002F0CD1D048407CF1
:1099E000F0218843CE4948740846807C0009000174
:1099F000C01D88740BE0CA48407CF0218843703059
:109A0000C74948740846807C000900018874F7F74C
:109A100051F9002821D1C2482030C078F021884374
:109A20007030BF492031C870BD4800E064E0807DDF
:109A300000090001203988750846807DF02188439F
:109A4000B7498875FF2223210020F9F755FE00222F
:109A500022211046F9F750FE7CE0F7F72BF9012898
:109A600078D1AF482030C078F0218843AC4920310C
:109A7000C870AB48807D00090001C01D2039887581
:109A80000846807DF02188437030A5498875002202
:109A900023211046F9F730FEFF2222210020F9F79A
:109AA0002BFE57E09E48407CF02188439C49487437
:109AB0000846807C00090001887408462030C07880
:109AC000F021884396492031C8709548807D00096F
:109AD0000001203988750846807DF021884390492F
:109AE0008875002223211046F9F706FE0022222164
:109AF0001046F9F701FE2DE08948407CF0218843AB
:109B00007030874948740846807C00090001C01DF8
:109B1000887408462030C078F0218843703080492E
:109B20002031C8707E48807D00090001C01D2039A9
:109B300088750846807DF0218843703078498875A3
:109B4000FF2223210020F9F7D7FDFF222221002048
:109B5000F9F7D2FDF7F7AEF8002808D06E48007884
:109B6000012804D0F2F730FF6C49884276D26D4864
:109B7000864209D96A4820304079F0218843703004
:109B800067492031487107E0654820304079F0216D
